:100000000C94891B0C94BA1B0C94BA1B0C94BA1B4D
:100010000C94BA1B0C94BA1B0C94BA1B0C94BA1B0C
:100020000C94BA1B0C94BA1B0C94BA1B0C94BA1BFC
:100030000C94BA1B0C94BA1B0C94BA1B0C94BA1BEC
:100040000C94BA1B0C94C8A40C94BA1B0C94BA1B45
:100050000C94BA1B0C94BA1B0C94868B0C942677C8
:100060000C94BA1B0C94D4EF0C94CAEF0C94BA1BEA
:100070000C94BA1B0C94BA1B0C94BA1B0C94BA1BAC
:100080000C94CDC50C94BA1B0C94BA1B0C94BA1BDF
:100090000C94BA1B0C94BA1B0C94BA1B0C94BA1B8C
:1000A0000C94BA1B0C94BA1B0C949FC50C94BA1BED
:1000B0000C94BA1B0C94BA1B0C94BA1B0C94BA1B6C
:1000C0000C94BA1B0C94BA1B0C94BA1B0C9482C6E9
:1000D0000C944CC60C94BA1B0C94BA1B0C94BA1B0F
:1000E0000C94BA1B084AD73B3BCE016E84BCBFFDC3
:1000F000C12F3D6C74319ABD56833DDA3D00C77FF8
:1001000011BED9E4BB4C3E916BAAAABE0000008090
:100110003F05A84CCDB2D44EB93836A9020C50B91F
:10012000918688083CA6AAAA2ABE000000803F004B
:100130000D94321A0D94231F0D94DD2B0D94490C50
:100140000D94640B0C94BC720C94D4740C947AF0DF
:100150000D94AC0E0C949D720C94F4450C94DE73CB
:100160000C94BF430C941CC70C94AE720C94CA73CD
:100170000D94EF150D944E170D940B1A0D942A1033
:100180000C9485F00C9498F00D94541A0C94EFC6CE
:100190000C9450F00C94B3450C94B8720C94DB6F33
:1001A0000C9475740C945C760C9414C70C9433C73F
:1001B0000C94A8720D94C8160C947C750D94FB2BAE
:1001C0000C9418C70D940A140C94C0C60C946EF0CD
:1001D0000C941D750C949D730D94631A0D945D160B
:1001E0000C9461750C9428C70D948D140C94D473E1
:1001F0000C94C0730C9412F00D9459140C94CE729C
:100200000C94FEC60C940C760C9458730C94997252
:100210000C94CA720C94E8730C9439760C94F273B3
:100220000D9429150C948B730D94381A0C94BB43C0
:100230000D94801B0C9466F00C9465730C945E70A6
:100240000D943B1A0C943EC70C9446C70D94811A2A
:100250000D94430A0C945FF00C9482720D946D1A05
:100260000C9483730C94C6720D94F9160C945D7003
:100270000D943D140C942CC70C94A7730C9476F039
:100280000C940DC70C946F730C9460730C9424C77A
:100290000D94FE170D9480160D94B9150C94FA75F3
:1002A0000C9479730C94A1720C9458740C94B173DF
:1002B0000C9487720C946C430C947EF00C942C4636
:1002C0000C94A5720D94E7160C94D4720C946AF0F9
:1002D0000C94C0720D94DB0D0C9472F00C9441F0F0
:1002E0000D948E1A0D94730C0C9490F00D94431C85
:1002F0000C94B2720D946F1B0C94D8720C948745B9
:100300000C9493730D94A9160C9420C70D943B176D
:100310000D94C4124E414E494E495459494E46CD52
:10032000CCCC3D0AD7233C17B7D13877CC2B3295AC
:1003300095E6241FB14F0A000020410000C842008A
:10034000401C4620BCBE4CCA1B0E5AAEC59D740054
:10035000407A10F35A00A0724E18090010A5D4E894
:100360000000E87648170000E40B54020000CA9A27
:100370003B000000E1F50500008096980000004079
:10038000420F000000A086010000001027000000BE
:1003900000E803000000006400000000000A000004
:1003A0000000000100000000002C76D888DC674FB8
:1003B0000823DFC1DFAE59E1B1B796E5E3E453C6E8
:1003C0003AE651997696E8E6C28426EB898C9B62E0
:1003D000ED407C6FFCEFBC9C9F40F2BAA56FA5F48A
:1003E00090055A2AF75C936B6CF9676DC11BFCE0B2
:1003F000E40D47FEF520E6B500D0ED902E03009405
:100400003577050080841E080000204E0A00000099
:10041000C80C333333330F986E12831141EF8D21A3
:1004200014893BE65516CFFEE6DB18D1844B381B0A
:10043000F77C1D901DA4BBE424203284725E2281CF
:1004400000C9F124ECA1E53D27434F4D4D554E49E0
:10045000434154494F4E0044525952554E00455263
:10046000524F525300494E464F004543484F004FAC
:100470004646004F4E0020204D61783A2000200073
:1004800020204D696E3A2000536F667420656E64BB
:1004900073746F70733A20003D3D4F6E506F7765F7
:1004A000724C6F7373526573756D653D3D004D32CF
:1004B000342053256C642054256C64004739322E57
:1004C00039204525730047312046256400473932DD
:1004D0002E39205A2573004731205A3020463230B9
:1004E000300047312058257320592573204633307A
:1004F0003030004D34323020532569205A257300A6
:100500004D3130362050256920532569004D323059
:10051000302044257300473238523058590047394B
:10052000322E39204530205A300A47315A2573007F
:100530004D31303920532569004D31393020532554
:1005400069004D343230205330205A300020496E3B
:1005500076616C69642065787472756465722000D8
:1005600047322F47332062616420706172616D658C
:10057000746572730A00536C6565702E2E2E005AD6
:100580002050726F62652050617374204265640A66
:10059000005A2050726F626520506173742042656A
:1005A00064004732384C30004D3131372050726F83
:1005B0006265206661696C65642E0A4732380A00FC
:1005C00070726F62655F7265776970650047323976
:1005D000205265747279696E670050726F62696E3D
:1005E00067204661696C6564004D31313720426592
:1005F00064206C6576656C696E67206661696C6500
:10060000642E0A4730205A31300A4D3330302050A2
:10061000323520533838300A4D33303020503530A1
:100620002053300A4D333030205032352053383883
:10063000300A4D333030205035302053300A4D339E
:1006400030302050323520533838300A4D33303076
:10065000205035302053300A473420533100707217
:100660006F62655F6661696C6564004D313137208A
:10067000426564206C6576656C696E6720646F6E98
:10068000652E00205A3A200020593A200042656425
:1006900020583A20004D65736820706F696E742091
:1006A0006F7574206F662072616E67650A004D3049
:1006B0002053746F70004D312053746F7000436F7E
:1006C0006E74696E756500436C69636B20746F208E
:1006D000526573756D652E2E2E004E6F204D6F7610
:1006E000652E00456E642066696C65206C697374C4
:1006F0000A00426567696E2066696C65206C6973E3
:10070000740A004E6F206D656469610A005265735A
:10071000756D696E6720534400286E6F2066696CA2
:1007200065290043757272656E742066696C653A5E
:1007300020005072696E742074696D653A20000A59
:1007400053746174733A2046696C616D656E7420F0
:10075000757365643A20002C204C6F6E6765737466
:10076000206A6F623A2000546F74616C2074696D66
:10077000653A200053746174733A20002C2046615E
:10078000696C65643A20002C2046696E697368655F
:10079000643A20005072696E74733A200053746199
:1007A00074733A2000436F6F6C696E672E2E2E00B3
:1007B00048656174696E672E2E2E00452025530012
:1007C0006F6B006F6666006A0465045E0457044937
:1007D0000444454255473A004D31313320530042DD
:1007E000656420436F6F6C696E672E2E2E00426524
:1007F000642048656174696E672E2E2E00544D3357
:100800004420453520506C7573204F46462E002FEE
:100810002F004D32303620580046523A0020466CA8
:100820006F773A20003A200020536572766F2000DF
:10083000206F7574206F662072616E67650A0053C1
:100840006572766F200020643A0020693A002070BB
:100850003A00496E76616C696420657874727564DB
:1008600065720A0020643A0020693A0020703A005C
:1008700064697300656E0043290A0061626C6564F7
:1008800020286D696E2074656D702000436F6C6464
:1008900020657874727564657320617265200050FC
:1008A0004944204175746F74756E65005049442049
:1008B0004175746F74756E65206661696C6564213D
:1008C00020426164206865617465722069640A0071
:1008D00046696C616D656E742072756E6F757420FB
:1008E00064697374616E636520286D6D293A200018
:1008F00046696C616D656E742072756E6F757420DB
:10090000004D34323120696E636F727265637420FA
:10091000706172616D657465722075736167650AD7
:10092000004D65736820706F696E74206F75742058
:100930006F662072616E67650A004F666673657444
:1009400073204170706C696564004572723A20547E
:100950006F6F206661722100546F6F206661722094
:1009600066726F6D207265666572656E6365207074
:100970006F696E740A00454550524F4D204F4B0A27
:10098000002E0A002028302D313029002076616C9D
:100990007565206F7574206F662072616E676500E3
:1009A000416476616E6365204B3D00506F776572E0
:1009B0002D6C6F7373207265636F7665727920009A
:1009C0004D383400446F6E65207072696E74696EC4
:1009D000672066696C650A004D3737004D3331007A
:1009E0004361703A004D4541545041434B00434FE1
:1009F0004F4C45525F54454D504552415455524518
:100A0000004348414D4245525F54454D5045524187
:100A10005455524500424142595354455050494E55
:100A2000470041524353004D4F54494F4E5F4D4F85
:100A300044455300544845524D414C5F50524F5429
:100A4000454354494F4E004C4F4E475F46494C4535
:100A50004E414D45004155544F5245504F52545F01
:100A600053445F5354415455530053445F575249C4
:100A7000544500524550454154005344434152446B
:100A80000050524F4D50545F535550504F525400E8
:100A9000454D455247454E43595F5041525345528B
:100AA00000434153455F4C494748545F42524947D0
:100AB00048544E45535300544F47474C455F4C49AB
:100AC0004748545300534F4654574152455F504F87
:100AD000574552004255494C445F50455243454E9C
:100AE00054004C4556454C494E475F4441544100E3
:100AF0005A5F50524F42450052554E4F5554004197
:100B000055544F4C4556454C005052494E545F4A3F
:100B10004F420050524F4752455353004155544F96
:100B20005245504F52545F54454D5000564F4C550E
:100B30004D455452494300454550524F4D0042499E
:100B40004E4152595F46494C455F5452414E5346BF
:100B500045520053455249414C5F584F4E5F584FE4
:100B60004646004649524D574152455F4E414D451C
:100B70003A4D61726C696E20322E302E375F4457C9
:100B8000372E3320544D334420453550534D444285
:100B900042202841707220323420323032312031EC
:100BA000393A35333A31382920534F555243455F4E
:100BB000434F44455F55524C3A68747470733A2FF2
:100BC0002F6769746875622E636F6D2F496E73614C
:100BD0006E6974794175746F6D6174696F6E2F4DB4
:100BE00061726C696E2F747265652F437265616CFA
:100BF0006974794477696E5F322E302050524F54B9
:100C00004F434F4C5F56455253494F4E3A312E3069
:100C1000204D414348494E455F545950453A544D43
:100C2000334420453520506C757320455854525537
:100C30004445525F434F554E543A3120555549442F
:100C40003A63656465326132662D343161322D3428
:100C50003734382D396231322D633535633632669B
:100C600033363766660A0050726F6265204F6666DB
:100C7000736574205A0050726F6265204F66667308
:100C80006574205A00290A0020746F20003F5A2002
:100C90006F7574206F662072616E67652028002969
:100CA0000A0020746F20003F59206F7574206F6612
:100CB0002072616E676520282D00290A0020746F5C
:100CC00020003F58206F7574206F662072616E6738
:100CD0006520282D0050726F6265204F666673652F
:100CE0007420580043616E6E6F74206F70656E20C3
:100CF00073756264697220002569730025696D202F
:100D0000256973002569682025696D2025697300B0
:100D1000256964202569682025696D20256973008F
:100D200025697920256964202569682025696D2059
:100D3000256973003D3D4477696E20496E697420D2
:100D4000436F6D706C6574653D3D002A2A2A4E6FB5
:100D50007A7A6C6554656D705374617475735B3227
:100D60005D203D003D3D48656174696E6720446FBC
:100D70006E65204368616E67652046696C616D65CC
:100D80006E743D3D002020737461727470726F67E1
:100D90007265737320003D3D7761697477617920D6
:100DA000353D3D003D3D7761697477617920343D83
:100DB0003D003D3D7761697477617920333D3D00A9
:100DC0003D3D7761697477617920313D3D003D3D5E
:100DD0006F6E5072696E7454696D657253746F7082
:100DE0007065643D3D003D3D6F6E466163746F729A
:100DF0007952657365743D3D00270A0A000027207B
:100E000027002027002D006E6F7469666963617486
:100E1000696F6E200063616E63656C005072696E6D
:100E2000742041626F72746564004469736D697304
:100E3000730055492041626F727465640072657376
:100E4000756D65004D3234002A2A2A43506C617951
:100E500020546F6E652A2A2A003D3D6F6E507269DC
:100E60006E7454696D65725061757365643D3D00C3
:100E7000486F6D696E67204661696C6564006F70CC
:100E8000656E00545249474745524544003A200098
:100E900066696C616D656E74007A5F6D696E00796C
:100EA0005F6D617800785F6D6178005265706F7278
:100EB00074696E6720656E6473746F7020737461FB
:100EC0007475730A0020746F6F206C6F6E672065F5
:100ED0007874727573696F6E2070726576656E7462
:100EE00065640A0020636F6C6420657874727573A2
:100EF000696F6E2070726576656E7465640A00486D
:100F00006F6D652025732573257320466972737490
:100F1000005761726E696E673A20486F6D696E673F
:100F20002042756D702044697669736F72203C2091
:100F3000310A000202040000B0430000B443000084
:100F400000000000B0430000B4430000C8430000AC
:100F5000004100000041000000400101FF000000CE
:100F600001000000010000800055555500000040C0
:100F70000033333300AAAA2A00499224000000203B
:100F800000C7711C0099991900D1451700555515D6
:100F9000003BB11300244912001111110000001090
:100FA000000F0F0F00E3380E0043790D00CCCC0C7E
:100FB00000C3300C00E8A20B0064210B00AAAA0AAF
:100FC00000703D0A009DD80900427B090092240967
:100FD00000DCD308008888080010420800000008E0
:100FE00000F0C107008787070075500700711C07D4
:100FF000003EEB0600A1BC0600699006006666068E
:1010000000703E06006118060017F4050074D10553
:10101000005BB00500B290050062720500555505F1
:101020000078390500B81E0500050505004EEC04E2
:101030000087D40400A1BD040090A70400499204D5
:1010400000C17D0400EE690400C756040044440456
:10105000005C320400082104004110040000000478
:10106000003FF00300F8E0030026D20300C3C303EF
:1010700000CCB503003AA803000A9B0300388E0396
:1010800000C08103009F750300D0690300505E0318
:10109000001D53030034480300913D030033330324
:1010A0000016290300381F030097150300300C03B6
:1010B00000030303000BFA020049F10200BAE80240
:1010C000005CE002002DD802002DD0020059C802B9
:1010D00000B0C0020031B90200DAB10200AAAA02CF
:1010E00000A0A30200BC9C0200FA9502005C8F02E3
:1010F00000DF88020082820200457C02002776021F
:101100000027700200436A02007C640200D05E0285
:10111000003F590200C8530200FFFDFCFAF8F6F444
:10112000F2F0EEECEAE9E7E5E3E1E0DEDCDAD9D77C
:10113000D5D4D2D0CFCDCBCAC8C7C5C3C2C0BFBD1E
:10114000BCBAB9B7B6B4B3B2B0AFADACAAA9A8A691
:10115000A5A4A2A1A09E9D9C9A99989795949392DC
:10116000908F8E8D8B8A8988878684838281807F09
:101170007E7D7B7A797877767574737271706F6E15
:101180006D6C6B6A696867666564636261605F5E07
:101190005D5C5B5A595858575655545352515050EC
:1011A0004F4E4D4C4B4A4A494847464645444342B8
:1011B0004241403F3E3E3D3C3B3B3A393838373672
:1011C0003535343332323130302F2E2E2D2C2B2B1F
:1011D0002A292928272726252524232322212120BF
:1011E000201F1E1E1D1C1C1B1B1A19191818171650
:1011F00016151514131312121111100F0F0E0E0DD8
:101200000D0C0C0B0A0A0909080807070606050554
:101210000404030302020100003D3D6F6E50726939
:101220006E7454696D6572537461727465643D3D8A
:10123000000000B0430000B4430000C843000000B9
:101240000000000000000000003D3D6F6E53746F11
:10125000726553657474696E67733D3D003D3D6F03
:101260006E436F6E66696775726174696F6E5374F1
:101270006F72655772697474656E3D3D0053657495
:1012800074696E67732053746F726564000A206915
:101290006E6974207A70726F62655F7A6F666673CA
:1012A0006574203D20003D3D6F6E436F6E6669673B
:1012B00075726174696F6E53746F726552656164A3
:1012C0003D3D00454550524F4D20496E697469615E
:1012D0006C697A65640A003B20003A0A0020204DC0
:1012E000363033200020440020204D34313220534A
:1012F0000046696C616D656E742072756E6F7574F1
:101300002073656E736F723A002055004C00466979
:101310006C616D656E74206C6F61642F756E6C6F9F
:101320006164206C656E677468733A0020204D39E3
:101330003030204B004C696E6561722041647661EB
:101340006E63653A0020204D3835312058005A2D03
:1013500050726F6265204F66667365740020204D81
:10136000343133205300506F7765722D4C6F737397
:10137000205265636F766572793A002044002049F7
:101380000020204D333034205000204400204900FC
:1013900020204D3330312050005049442073657473
:1013A00074696E67733A00204A0020204732392062
:1013B0005720490020204D343230205300417574AD
:1013C0006F20426564204C6576656C696E673A00F3
:1013D00020204D323036205800486F6D65206F66F2
:1013E000667365743A0020580020530020204D3267
:1013F0003035204200416476616E6365643A204274
:101400003C6D696E5F7365676D656E745F74696D61
:10141000655F75733E20533C6D696E5F66656564FC
:10142000726174653E20543C6D696E5F74726176C2
:10143000656C5F66656564726174653E20583C6DDD
:1014400061785F785F6A65726B3E20593C6D6178A8
:101450005F795F6A65726B3E205A3C6D61785F7A96
:101460005F6A65726B3E20453C6D61785F655F6ABF
:1014700065726B3E0020540020520020204D323017
:1014800034205000416363656C65726174696F6EEE
:101490002028756E6974732F7332293A20503C707E
:1014A00072696E745F616363656C3E20523C726565
:1014B00074726163745F616363656C3E20543C7455
:1014C000726176656C5F616363656C3E0020204DE0
:1014D0003230312058004D6178696D756D2041635F
:1014E00063656C65726174696F6E2028756E6974CE
:1014F000732F7332293A0020204D323033205800A8
:101500004D6178696D756D2066656564726174659D
:10151000732028756E6974732F73293A00537465AC
:1015200070732070657220756E69743A00204400F3
:1015300020204D3230302053002044697361626CAA
:1015400065640A0046696C616D656E74207365742C
:1015500074696E67733A0020286D6D29002020475A
:101560003231202020203B20556E69747320696E33
:10157000206D6D003D3D6F6E4C6F616453657474FA
:10158000696E67733D3D0000803B4400803B440032
:10159000002041000096420000A0420000A042004E
:1015A0000048440080CC43D0070000D0070000640E
:1015B0000000004B00000024F4D43050C38E20C241
:1015C000A24017828B7011127A910D816CD90AA8F2
:1015D00061E108C7586607615143061E4B5D05C1AE
:1015E00045A7041A411104093D980371393103409C
:1015F00036DB0265339102D4305402802E1D026323
:101600002CEE01752AC501B028A001102781018F99
:101610002564012B244B01E0223401AC211F018DF4
:10162000200D01801FFC00841EED00971DDF00B817
:101630001CD200E61BC600201BBC00641AB200B21C
:1016400019A8000A19A0006A189900D11791004042
:10165000178B00B516840031167E00B31579003A59
:10166000157300C7146F0058146A00EE13660088E3
:1016700013630025135E00C7125B006C1257001540
:10168000125400C111510070114F0021114B00D6AE
:101690001049008D1047004610440002104200C05F
:1016A0000F4000800F3E00420F3C00060F3B00CB76
:1016B0000E3800930E37005C0E3500270E3400F311
:1016C0000D3200C10D3100900D3000600D2E003242
:1016D0000D2D00050D2C00D90C2B00AE0C2900851A
:1016E0000C29005C0C2700350C27000E0C2600E8A6
:1016F0000B2400C40B2400A00B23007D0B23005AF5
:101700000B2100390B2100180B2000F80A1F00D90B
:101710000A1E00BB0A1E009D0A1D00800A1D0063F0
:101720000A1C00470A1B002C0A1B00110A1A00F7AA
:10173000091A00DD091900C4091900AB0919009242
:101740000917007B091800630917004C09160036B9
:10175000091600200916000A091500F5081500E011
:10176000081400CC081400B8081400A40814009051
:101770000813007D0812006B081300580812004679
:10178000081200340811002308110012081100018A
:10179000081100F0071000E0071000D0071000C08B
:1017A000071000B0070F00A107100091070E00837B
:1017B000070F0074070F0065070E0057070E00495A
:1017C000070E003B070D002E070E0020070D00132B
:1017D000070D0006070D00F9060C00ED060D00E0F0
:1017E000060C00D4060C00C8060C00BC060C00B0A9
:1017F000060C00A4060B0099060C008D060B008257
:10180000060B0077060B006C060B0061060A0057FA
:10181000060B004C060A0042060A0038060A002E93
:10182000060A0024060A001A060A00100609000724
:10183000060A00FD050900F4050900EB050900E2B0
:10184000050900D9050900D0050900C7050900BE32
:10185000050900B5050800AD050800A50509009CAF
:10186000050800940508008C050800840508007C24
:10187000050800740508006C050700650508005D93
:10188000050700560508004E0507004705070040FC
:1018900005080038050700310507002A0507002361
:1018A0000507001C050600160507000F05070008C0
:1018B00005060002050700FB040600F5040700EE1C
:1018C000040600E8040600E2040700DB040600D575
:1018D000040600CF040600C9040600C3040600BDC8
:1018E000040600B7040600B1040500AC040600A617
:1018F000040600A00405009B040600950405009062
:101900000406008A04050085040500800406007AA8
:1019100004050075040500700405006B04050066ED
:10192000040500610405005C04050057040500522D
:101930000405004D04050048040500430405003E6D
:101940000404003A04050035040500300404002CAA
:1019500004050027040400230405001E0404001AE3
:1019600004040016040500110404000D0404000919
:101970000405000404040000040400FC030400F84F
:10198000030400F4030400F0030400EC030400E883
:10199000030400E4030400E0030400DC030400D8B3
:1019A000030400D4030400D0030400CC030400C8E3
:1019B000030300C503030024F404D9201BC40C5CFA
:1019C0000E9804C4095F0265077101F405F900FB74
:1019D00004B30048048700C103690058035500039D
:1019E000034500BE023A008402310053022A002956
:1019F00002250004022000E4011C00C8011900AF08
:101A00000117009801140084011300710110006196
:101A100001100051010E0043010D0036010B002B97
:101A2000010B0020010B00150109000C0109000346
:101A3000010800FB000800F3000800EB000700E4C9
:101A4000000600DE000600D8000600D2000600CC2A
:101A5000000500C7000500C2000500BD000400B974
:101A6000000400B5000400B1000400AD000400A9AA
:101A7000000400A5000300A20003009F0004009BD7
:101A800000030098000300950002009300030090FB
:101A90000003008D0002008B000300880002008616
:101AA00000020084000300810002007F0002007D2C
:101AB0000002007B0002007900020077000100763E
:101AC0000002007400020072000100710002006F49
:101AD0000002006D0001006C0002006A0001006954
:101AE000000200670001006600010065000100645B
:101AF0000002006200010061000100600001005F5F
:101B00000002005D0001005C0001005B0001005A62
:101B10000001005900010058000100570001005663
:101B20000001005500010054000100530000005363
:101B30000001005200010051000100500001004F5F
:101B40000001004E0000004E0001004D0001004C5D
:101B50000001004B0000004B0001004A0001004959
:101B60000001004800000048000100470001004655
:101B7000000000460001004500000045000100444F
:101B80000001004300000043000100420000004249
:101B90000001004100000041000100400001003F41
:101BA0000000003F0001003E0000003E0001003D3B
:101BB0000000003D0001003C0000003C0000003C33
:101BC0000001003B0000003B0001003A0000003A29
:101BD0000001003900000039000100380000003821
:101BE0000000003800010037000000370001003617
:101BF000000000360000003600010035000000350E
:101C00000000003500010034000000340000003402
:101C100000010033000000330000003300010032F7
:101C200000000032000000320001003100000031ED
:101C300000000031000100300000003000000030E2
:101C40000001002F0000002F0000002F0000002FD7
:101C50000001002E0000002E0000002E0001002DCB
:101C60000000002D0000002D0000002D0001002CC0
:101C70000000002C0000002C0000002C0001002BB4
:101C80000000002B0000002B0000002B0001002AA8
:101C90000000002A0000002A0000002A000100299C
:101CA0000000002900000029000000290000002990
:101CB0000001002800000028000000280000002883
:101CC0000000002800010027000000270000002776
:101CD0000000002700000027000100260000002669
:101CE000000000260000002600000026000100255C
:101CF0000000002500000025000000250000002550
:101D00000000002500010024000000240000002441
:101D10000000002400000024000100230000002334
:101D20000000002300000023000000230000002327
:101D30000000002300010022000000220000002219
:101D4000000000220000002200000022000100210B
:101D500000000021000000210000002100000021FF
:101D600000000021000000210001002000000020F0
:101D700000000020000000200000002000000020E3
:101D800000000020000000200001001F0000001FD4
:101D90000000001F0000001F0000001F0000001FC7
:101DA0000000001F0001001E0000001E0000001EB9
:101DB0000000001E000000232C0000B82200005686
:101DC0001800003A0F0000B8080000B104000071CC
:101DD0000200003E01000020436F756E7420583AE7
:101DE0000023646566696E652044454641554C5440
:101DF0005F0000626564004B6420004B6920004B6B
:101E0000702000504944204175746F74756E6520D0
:101E100066696E6973686564212050757420746802
:101E200065206C617374204B702C204B6920616EAF
:101E300064204B6420636F6E7374616E74732066EC
:101E4000726F6D2062656C6F7720696E746F2043CE
:101E50006F6E66696775726174696F6E2E680A00CD
:101E6000504944204175746F74756E6520666169D0
:101E70006C6564212074696D656F75740A00504942
:101E800044204175746F74756E65206661696C6578
:101E900064212054656D706572617475726520747B
:101EA0006F6F20686967680A00204B643A20002041
:101EB0004B693A2000204B703A200020436C61733C
:101EC00073696320504944200A00204E6F206F76CA
:101ED000657273686F6F740A002054753A20002091
:101EE0004B753A2000206D61783A2000206D696EB4
:101EF0003A200020643A200020626961733A200091
:101F0000504944204175746F74756E652073746117
:101F100072740A00504944204175746F74756E657F
:101F2000206661696C6564212054656D706572611D
:101F30007475726520746F6F20686967680A004263
:101F4000656400453100626564002C207379737408
:101F5000656D2073746F70706564212048656174CD
:101F600065725F49443A200048656174696E672074
:101F70004661696C65640048656174696E672066D6
:101F800061696C6564004D31313220536875746449
:101F90006F776E001000C90210012C014001220170
:101FA00070011801B0010E01F00104015002FA00A5
:101FB000B002F0003003E600D003DC009004D20051
:101FC0007005C800A006BE000008B400B009AA0051
:101FD000D00BA000600E960060118C0000158200EE
:101FE00020197800C01D6E00A0226400B0275A009E
:101FF000902C500000314600E0343C001038320094
:10200000903A2800603C1E00A03D1400803E0A006B
:10201000203F0000544845524D414C2052554E41FE
:1020200057415900546865726D616C2052756E613C
:10203000776179004572723A204D415854454D50B0
:10204000004D415854454D50207472696767657260
:102050006564004572723A204D494E54454D50001A
:102060004D494E54454D50207472696767657265DD
:102070006400202F002042403A0020403A002057C0
:102080003A0020573A00496E76616C6964206578A1
:102090007472756465720A007C3C3E5E2B3D3F2F76
:1020A0005B5D3B2C2A225C0043616E6E6F74206F77
:1020B00070656E2073756264697220005344204914
:1020C0006E6974204661696C0053442063617264D8
:1020D000206F6B0A006F70656E526F6F74206661BF
:1020E000696C65640A00766F6C756D652E696E6942
:1020F00074206661696C65640A004E6F2053442049
:10210000636172640A000A4D3234004D3233202577
:1021100073002E0A006F70656E206661696C6564DD
:102120002C2046696C653A200046696C6520736511
:102130006C65637465640A002053697A653A20000F
:1021400046696C65206F70656E65643A2000454E87
:102150004420535542524F5554494E450A002220BF
:10216000706F73002220706172656E743A220053A2
:102170005542524F5554494E452043414C4C2074D2
:1021800061726765743A220053756263616C6C20FA
:102190004F766572666C6F77004578636565646538
:1021A00064206D617820535542524F5554494E4535
:1021B0002064657074683A002E0A0044656C65748A
:1021C000696F6E206661696C65642C2046696C6578
:1021D0003A200046696C652064656C657465643AF4
:1021E000005344207072696E74696E67206279745E
:1021F0006520004E6F74205344207072696E7469BC
:102200006E670A0057726974696E6720746F206682
:10221000696C653A2000667265736800646F696E68
:1022200067002066696C653A20004E6F7720002FAA
:102230006175746F25632E67002020506C616E6E8F
:10224000657242756666657242797465733A2000FC
:102250002046726565204D656D6F72793A200043A6
:102260006F6D70696C65643A204170722032342061
:10227000323032310A00204C617374205570646131
:102280007465643A20323032312D30342D313820AB
:102290007C20417574686F723A2054696E794D6183
:1022A0006368696E657333440A00322E302E375FDF
:1022B0004457372E330A004D61726C696E0020530B
:1022C0006F6674776172652052657365740A0020C9
:1022D0005761746368646F672052657365740A00A0
:1022E0002042726F776E206F75742052657365742B
:1022F0000A002045787465726E616C2052657365C2
:10230000740A00506F77657255700A0073746172B9
:10231000740A004732385859004D31303031006569
:1023200072726F722077726974696E6720746F20A1
:1023300066696C650A00446F6E6520736176696E2C
:10234000672066696C652E0A004D323900456E645F
:1023500073746F7073002553202563202563202537
:102360006320256300205A3A0020593A0020583A49
:1023700000656E6473746F7073206869743A20002E
:1023800000000A0B02090C0D0E08070304010000EF
:10239000000000000000000000000000000000003D
:1023A00000000000000000000000000012111000FA
:1023B000000000000000000000000000000000001D
:1023C0000000000000004572726F7220777269741D
:1023D000696E6720746F20454550524F4D210A00A9
:1023E00053544F505045442E20005072696E74650E
:1023F000722073746F707065642064756520746FEB
:10240000206572726F72732E204669782074686539
:10241000206572726F7220616E6420757365204D45
:1024200039393920746F20726573746172742E208B
:102430002854656D706572617475726520697320CA
:1024400072657365742E205365742069742061660B
:102450007465722072657374617274696E67290A9B
:10246000004E6F20436865636B73756D20776974E8
:1024700068206C696E65206E756D6265722C204CEB
:10248000617374204C696E653A20004E6F2043687A
:1024900065636B73756D2077697468206C696E6510
:1024A000206E756D6265722C204C617374204C69CE
:1024B0006E653A2000636865636B73756D206D69A6
:1024C000736D617463682C204C617374204C696E69
:1024D000653A20004C696E65204E756D626572200C
:1024E0006973206E6F74204C617374204C696E6543
:1024F000204E756D6265722B312C204C61737420F7
:102500004C696E653A20004D313130005365726977
:10251000616C20737461747573206D69736D61747F
:1025200063680A00776169740A0053442072656128
:1025300064206572726F720A002121204B494C4C55
:102540002063617573656420627920746F6F206DFC
:1025500075636820696E6163746976652074696D5E
:1025600065202D2063757272656E7420636F6D6DCA
:10257000616E643A2000486F74656E642049646C33
:10258000652054696D656F757400486F74656E647D
:102590002049646C652054696D656F75740A003D4F
:1025A0003D6F6E46696C616D656E7452756E6F75C8
:1025B000743D3D007061757365004D36303000200C
:1025C00066696C616D656E745F72756E6F7574208F
:1025D0000066696C616D656E745F72756E6F75749F
:1025E00020540046696C616D656E7452756E6F752E
:1025F000742054002A2A2A496E6974696E67206320
:10260000617264206973204F4B2A2A2A004D656449
:10261000696120496E736572746564004D65646913
:10262000612052656D6F766564004D3130303053F6
:1026300000627573793A2070617573656420666F06
:102640007220696E7075740A00627573793A207031
:10265000617573656420666F7220757365720A0018
:10266000627573793A2070726F63657373696E6710
:102670000A002A2A2A6B696C6C2A2A2A00706F7752
:1026800065726F6666004B494C4C45442E200050E5
:1026900072696E7465722068616C7465642E206B5B
:1026A000696C6C28292063616C6C6564210A005395
:1026B000544F505045442E20005072696E7465721C
:1026C0002073746F707065642064756520746F206A
:1026D0006572726F72732E20466978207468652067
:1026E0006572726F7220616E6420757365204D395A
:1026F000393920746F20726573746172742E2028CA
:1027000054656D70657261747572652069732072AD
:10271000657365742E205365742069742061667436
:1027200065722072657374617274696E67290A003C
:102730006563686F3A004572726F723A0042696C65
:10274000696E656172204C6576656C696E672047BD
:102750007269643A0A0021212053544F502063616A
:102760006C6C65642062656361757365206F6620BB
:10277000424C546F756368206572726F72202D2011
:10278000726573746172742077697468204D393989
:10279000390A0021212053544F502063616C6C652D
:1027A000642062656361757365206F6620424C54D6
:1027B0006F756368206572726F72202D2072657369
:1027C000746172742077697468204D3939390A0050
:1027D0002F2F616374696F6E3A0070726F6D707441
:1027E0005F00656E640053656E64204D31303820A3
:1027F000746F20726573756D650A00496E7365723A
:10280000742066696C616D656E7420616E642073FE
:10281000656E64204D3130380A0052656865617418
:102820002066696E69736865642E0052656865612B
:102830007420446F6E6500526568656174696E67E7
:102840002E2E2E00526568656174004865617465BE
:10285000722054696D656F75740053656E64204D08
:1028600031303820746F2068656174206E6F7A7A19
:102870006C650A004E6F7A7A6C65205061726B65E8
:102880006400486F74656E6420746F6F20636F6CB2
:10289000640A00706175736564005061757365004A
:1028A00044697361626C6552756E6F757400507522
:1028B0007267654D6F726500506175736564007372
:1028C000686F7700627574746F6E00626567696E19
:1028D000004C6F61642046696C616D656E74004CDC
:1028E0006F61642046696C616D656E7420540049A7
:1028F0006E736572742066696C616D656E742061BB
:102900006E642073656E64204D3130380A00726544
:1029100073756D656400526573756D696E670057F8
:10292000616974696E6720666F722068656174758D
:10293000702E0A004C656176696E6720473236005A
:102940003F53706563696669656420582C5920633C
:102950006F6F7264696E617465206F7574206F6645
:1029600020626F756E64732E0A003F2852296570CD
:102970006561742076616C7565206E6F7420706C73
:1029800061757369626C653B206D75737420626557
:10299000206174206C6561737420312E0A003F2819
:1029A00052296570656174206D75737420626520AD
:1029B000737065636966696564207768656E206E0B
:1029C0006F74207573696E6720616E204C43442ECE
:1029D0000A003F537065636966696564206E6F7AAB
:1029E0007A6C652074656D706572617475726520AE
:1029F0006E6F7420706C61757369626C652E0A006D
:102A00003F5370656369666965642066696C616DD2
:102A1000656E742073697A65206E6F7420706C61C6
:102A2000757369626C652E0A003F53706563696651
:102A3000696564207072696D65206C656E67746885
:102A4000206E6F7420706C61757369626C652E0AFC
:102A5000003F5072696D65206C656E677468206D0B
:102A60007573742062652073706563696669656457
:102A7000207768656E206E6F74207573696E6720AD
:102A8000616E204C43442E0A003F537065636966B3
:102A9000696564206E6F7A7A6C652073697A652047
:102AA0006E6F7420706C61757369626C652E0A00BC
:102AB0003F52657472616374696F6E204D756C74FA
:102AC00069706C696572206D75737420626520731E
:102AD00070656369666965642E0A003F53706563BB
:102AE00069666965642052657472616374696F6EAA
:102AF000204D756C7469706C696572206E6F7420FE
:102B0000706C61757369626C652E0A003F53706565
:102B1000636966696564206C6179657220686569BE
:102B2000676874206E6F7420706C61757369626C75
:102B3000652E0A0043292E0A003F537065636966BB
:102B4000696564206265642074656D706572617486
:102B5000757265206E6F7420706C61757369626C3C
:102B600065202834302D004732362073746172742A
:102B7000696E672E2E2E0A004F46460A0046616493
:102B800065204865696768742000426564204C656B
:102B900076656C696E6720004661696C65642074B7
:102BA0006F20656E61626C6520426564204C6576BD
:102BB000656C696E670A00496E76616C6964206DA8
:102BC0006573682E0A0050726F62696E6720506FDD
:102BD000696E740025532025692F2569002E0A008F
:102BE0002F0050726F62696E67206D657368207088
:102BF0006F696E742000202844525952554E2900A6
:102C0000473239204175746F20426564204C6576E7
:102C1000656C696E67003F20284C2C522C462C4274
:102C200029206F7574206F6620626F756E64732E35
:102C30000A003F2856296572626F7365206C6576BD
:102C4000656C20696D706C61757369626C652028B4
:102C5000302D34292E0A00426164205A2076616C9E
:102C600075650A004E6F2062696C696E656172203D
:102C7000677269640A004163637572616379204415
:102C8000656372656173696E67210044656372658F
:102C90006173696E67204163637572616379204473
:102CA000657465637465642E0A00473238004732E4
:102CB000385A0041636375726163793A2000206F6E
:102CC00066200044696420004733342061626F72DB
:102CD0007465642E0A0041636375726163792041F3
:102CE0006368696576656400546172676574206124
:102CF0006363757261637920616368696576656491
:102D00002E0A004469666673205A312D5A323D25D9
:102D100073000A444946464552454E4345205A31C0
:102D20002D5A323D0050726F62696E6720466169AC
:102D30006C65640050726F62696E67206661696CD1
:102D400065640A0047333420497465726174696FA1
:102D50006E3A202569000A47333420497465726150
:102D600074696F6E3A20003F2841296D706C696666
:102D700069636174696F6E206F7574206F6620627D
:102D80006F756E64732028302E352D322E30292E2B
:102D90000A003F2854296172676574206163637576
:102DA00072616379206F7574206F6620626F756E33
:102DB00064732028302E30312D312E30292E0A0018
:102DC0003F2849297465726174696F6E206F75744C
:102DD000206F6620626F756E64732028312D33304A
:102DE000292E0A003F285929206F7574206F66200C
:102DF000626F756E64732E0A003F285829206F7524
:102E000074206F6620626F756E64732E0A003F280F
:102E100053292050726F62652D706F736974696FEA
:102E20006E20696E64657820696E76616C69642EC7
:102E30000A003F28532920697320726571756972F1
:102E400065642E0A004D34323220530044657669A1
:102E50006174696F6E0025533A2025730046696ED0
:102E60006973686564210A003A207A3A2000206F6D
:102E7000662000476F696E6720746F3A20580043E0
:102E8000570A00206469723A0020616E676C653AE7
:102E9000005374617274207261646975733A004DF5
:102EA000343820506F696E740025533A2025642F02
:102EB000256400506F736974696F6E696E67207462
:102EC00068652070726F62652E2E2E0A003F4C6579
:102ED0006773206F66206D6F76656D656E7420690F
:102EE0006D706C61757369626C652028302D3135A9
:102EF000292E0A003F2028582C5929206F7574204C
:102F00006F6620626F756E64732E0A0050726F6276
:102F100065206F7574206F6620626F756E64730034
:102F20003F53616D706C652073697A65206E6F74B4
:102F300020706C61757369626C652028342D3530A2
:102F4000292E0A004D3438205A2D50726F626520A8
:102F50005265706561746162696C69747920546549
:102F600073740A003F2856296572626F7365206C7E
:102F70006576656C20696D706C61757369626C65EE
:102F80002028302D34292E0A005374616E6461723A
:102F90006420446576696174696F6E3A200020523E
:102FA000616E67653A2000204D61783A2000204D1F
:102FB000696E3A2000205369676D613A20004D65C3
:102FC000616E3A2000205200416363656C65726156
:102FD00074696F6E3A2050005741524E494E472156
:102FE000204C6F77205A204A65726B206D617920E2
:102FF0006C65616420746F20756E77616E746564B2
:10300000207061757365732E0A0070012C019001A8
:103010002701B0012201C0011D01F00118011002B9
:10302000130130020E016002090190020401C00286
:10303000FF000003FA004003F5008003F000D00316
:10304000EB002004E6007004E100E004DC00400531
:10305000D700C005D2004006CD00D006C8008007CA
:10306000C3003008BE00F008B900C009B400B00ABF
:10307000AF00B00BAA00D00CA500000EA000500FAE
:103080009B00C01096005012910000148C00C015D7
:103090008700B0178200B0197D00D01B7800001E99
:1030A000730040206E0090226900F02464004027E5
:1030B0005F0090295A00E02B5500102E5000203060
:1030C0004B0010324600E033410090353C00103791
:1030D000370070383200A0392D00B03A2800A03BEC
:1030E0002300603C1E00103D1900903D1400103E6E
:1030F0000F00703E0A00C03E0500003F0000403F48
:10310000FBFF803FF6FFC03FF1FF50726F62696EB8
:1031100067204661696C656400205A3A2000205996
:103120003A200042656420583A20003D3D6F6E55BC
:10313000736572436F6E6669726D526571756972FF
:1031400065643D3D00220A00556E6B6E6F776E2000
:10315000636F6D6D616E643A202200204200205042
:10316000006F6B00204500205A00205900204D3987
:103170003220580020453A00205A3A0020593A009F
:10318000583A0020746F6F206C6F6E6720657874FA
:10319000727573696F6E2070726576656E746564A2
:1031A0000A0020636F6C6420657874727573696FB0
:1031B0006E2070726576656E7465640A0043616E98
:1031C0006E6F7420656E74657220737562646972C7
:1031D0003A20004D323520500A4D3234005265738A
:1031E000756D65005549205061757365004E6F20FF
:1031F0004D61746368203A00506755700050674411
:103200006F776E0049732046696C65200049732012
:103210004469722000476F557044697200486173B9
:10322000204D656469610046696C656E616D65205D
:1032300053656C6563746564004D31303030430014
:103240004D313030300046696C616D656E742053CD
:103250007461742030202D20330046696C616D65E7
:103260006E7420537461742030202D203200466922
:103270006C616D656E7420537461742030202D2054
:1032800031002046696C616D656E74205265737003
:103290006F6E7365204E6F00526573756D652059B2
:1032A000657320647572696E67207072696E740050
:1032B0000A204E6F2046696C616D656E7400496E20
:1032C00076616C6964204F7074696F6E004D3530A3
:1032D000300053746F72652053657474696E677340
:1032E00000426564205049442053746172746564DF
:1032F000004D3939390A4D3238305030533136307B
:1033000000424C546F756368205265736574004DBC
:103310003530320A4D35303000496E6974204545EC
:1033200050524F4D00486F74656E642050494420E0
:103330005374617274656400456E676C69736820CC
:10334000416C726561647920536574004368696EED
:10335000657365204E6F7420537570706F7274655D
:103360006400496E4C616E6743686F696365000A6B
:10337000202A2A2A7265636461742E646174615B19
:10338000305D203D004732380A4731204631303029
:1033900030205A313000556E737570706F727465DD
:1033A00064204F7074696F6E2053656C656374653B
:1033B000640047323652323535004D31393053359D
:1033C000350A4732380A47333449380A4732390A0E
:1033D0004D3430300A4D313034533231350A4732B2
:1033E000380A4D313039533231350A4D3432305389
:1033F000310A47315831303059313030463530306C
:10340000300A47315A300A4D3530300A4D313137A4
:1034100020536574205A204F6666736574004731E7
:10342000204631303030205A302E30004732380AB2
:103430004731204631303030205A302E30004D3563
:103440003030005A204F6666736574203A20257329
:10345000004D353030005A204F6666736574203A4F
:10346000202573004732380A473146313530305A0B
:10347000302E30004732385A0A4731463135303025
:103480005A302E30004D383400473146313030301C
:103490005A302E30004732380A473146313030300A
:1034A0005A302E30004D616E75616C5365745465F1
:1034B0006D70005A204F6666736574203A2025733C
:1034C0000053746F70205472696767657265640099
:1034D00053746F70204E6F0053746F705072696E2A
:1034E000740048616E646C652044617461204164BD
:1034F0006A75737420322053657474696E67205343
:10350000637265656E200048616E646C652044617D
:103510007461205072696E7446696C652033205363
:10352000657474696E672053637265656E20004828
:10353000616E646C652044617461205072696E74C0
:1035400046696C6520322053657474696E67205338
:10355000637265656E20004D38340048616E646C9E
:10356000652044617461205072696E7446696C65AF
:1035700020506F73740048616E646C652044617400
:1035800061205072696E7446696C652050726500E6
:10359000426567696E537769746368003D3D2043F7
:1035A0006865636B6B65793D3D007265636461744A
:1035B0002E61646472203D3D007265636461742E07
:1035C000646174615B305D203D3D007761697477B3
:1035D0006179203D3D0020202A2A2A2A2A2A2A52BF
:1035E00054535F48616E646C65446174612A2A2A91
:1035F0002A2A2A2A2A2000526573656E643A20001E
:1036000000002200250028002B002E00310034008D
:1036100002010000050108010B0100002100240047
:1036200027002A002D0030003300010100000401B2
:1036300007010A0105050505070508080808020233
:1036400002020A0A0808040404040101010101013C
:1036500001010303030303030303040707070C0C1F
:103660000C0C0C0C0C0C02020202060606060606E6
:1036700006060B0B0B0B0B0B0B0B0102102020088B
:1036800008102040102040800201020108040201BD
:10369000010204081020408080402010080402012C
:1036A0008004020180402010080402010804020185
:1036B000010204081020408001020408102040800C
:1036C000544D334420453520506C7573205265614C
:1036D00064792E005072696E74696E672E2E2E000A
:1036E0005072696E7420506175736564006E6F74FA
:1036F000696669636174696F6E20005049442054A3
:10370000756E652046696E69736865640000DE0049
:103710009C0011241FBECFEFD1E2DEBFCDBF00E081
:103720000CBF14E0A0E0B2E0ECE1FAE702E00BBF6E
:1037300002C007900D92AC31B107D9F726E1ACE198
:10374000B4E001C01D92A33CB207E1F71BE1C8E859
:10375000DBE100E006C021970109802FFE010F94F4
:103760003B39C738D10780E00807A9F70F948D26A9
:103770000D94FC3C0C9400009F92AF92BF92CF92AC
:10378000DF92EF92FF920F931F93CF93DF9300D0BE
:103790001F921F92CDB7DEB7E9E1F1E10027BB2709
:1037A000462F572FA82FAA2341F4A52F542FB85FD7
:1037B000AA2319F4A52F5527B85FA03138F45295E4
:1037C000A295452F4F70507FA42BBC5FA03428F4E6
:1037D000550FAA1F550FAA1FBE5FA03818F4550F2A
:1037E000AA1FB395550FAA1FEA0FF01F449151E08D
:1037F000AA27B85081F1C8F0B0FF02C0440F551F8E
:10380000B1FF04C0440F551F440F551FB2FF06C03F
:1038100052954295142F1F70407F512BB3FF1BC050
:10382000A52F542F44270C942B1CB195B0FF02C038
:1038300055954795B1FF04C05595479555954795C2
:10384000B2FF05C05295407F4295452B5F70B3FF94
:1038500002C0452F5527DD24CC24BB24B2E0649F51
:10386000D018C108B00AB00B749FC018B108B00BD3
:10387000849FB018B109659FC018B108B00B759F3F
:10388000B018B109859FB0196A9FB018B1097A9F25
:10389000B0194D9DA12C99243327992722275D9D8E
:1038A000A00C911C301F901F201FAD9D900C311D4E
:1038B000901F201F4C9DA00C911C301F901F201F9B
:1038C0005C9D900C311D901F201FAC9D300D911DF3
:1038D000201F4B9D900C311D901F201F5B9D300DB4
:1038E000911D201FAB9D900D211D4B9F300D911DF3
:1038F000201F5B9F900D211DAB9F200DB1E0BB24CD
:10390000CC24DD24639FD018C108B00AB00B739F8C
:10391000C018B108B00B839FB018B109699FC018D7
:10392000B108B00B799FB018B109899FB019629F97
:10393000B018B109729FB019D61AC70AB80A20F098
:10394000B1E03B0F901F201F1124792F632F90E0CF
:10395000822F0F900F900F900F900F90DF91CF91CB
:103960001F910F91FF90EF90DF90CF90BF90AF909D
:103970009F900895AF92BF92CF92DF92EF92FF9205
:103980000F931F93CF93DF93C1ECDCE004E119E0C8
:1039900081EDA82E8CE0B82EC12CD12C7601C394D9
:1039A00069917991899199910F947932288939890E
:1039B0004A895B890F94DA320F94B73AF801619320
:1039C0007193819391938F01C616D706E806F90685
:1039D00010F46B017C01AC16BD0611F76FEF7FEFA1
:1039E000CB01A70196010F94B83820932409309396
:1039F00025094093260950932709DF91CF911F9104
:103A00000F91FF90EF90DF90CF90BF90AF9008950F
:103A1000CF93DF9324E0829FC0011124EC01C95FA2
:103A2000D64FFC01E35CF74F8F5C974FDC012D9183
:103A30003D914D915C9160817181828193810F9460
:103A40004439688379838A839B83DF91CF9108957A
:103A500080910C1390910D13891B877089F48091CC
:103A6000140E81110DC08091090D90910A0D892BC2
:103A700039F481E09091D205911103C080E008955E
:103A800081E0089590E080E00895282F90912B0820
:103A9000833021F495FD0FC094FD0FC0892F90E075
:103AA000B0E0A0E004C0B695A795979587952A95B4
:103AB000D2F78170089581E0089580E00895CF9352
:103AC000C82FCB010E9492C78DE89EE00E9492C74A
:103AD0008EE79EE0CC2311F083E89EE00E9492C71F
:103AE0008AE0CF910C946AC70F931F93CF938C01F8
:103AF000C62F80EE99E00E9492C7C8010E9492C72B
:103B00008AE30E946AC780E38C0F0E946AC78AE03A
:103B1000CF911F910F910C946AC783E69BE00E949E
:103B200092C760E083E59BE00E94741D60E08EE335
:103B30009BE00E94741D61E087E39BE00E94741D7E
:103B400061E08CE29BE00E94741D61E08CE19BE0EF
:103B50000E94741D60E083E19BE00E94741D61E09F
:103B600089E09BE00E94741D61E08FEF9AE00E9463
:103B7000741D61E088EF9AE00E94741D61E080EF9F
:103B80009AE00E94741D61E082EE9AE00E94741D2A
:103B900061E084ED9AE00E94741D60E085EC9AE09B
:103BA0000E94741D60E087EB9AE00E94741D60E043
:103BB00081EA9AE00E94741D61E080E99AE00E9427
:103BC000741D61E081E89AE00E94741D61E08AE75B
:103BD0009AE00E94741D60E083E79AE00E94741DE1
:103BE00061E08AE69AE00E94741D61E085E59AE052
:103BF0000E94741D61E087E49AE00E94741D61E0F8
:103C000084E39AE00E94741D60E087E29AE00E94DB
:103C1000741D61E082E29AE00E94741D61E085E11A
:103C20009AE00E94741D60E081E09AE00E94741D99
:103C300060E08EEE99E00E94741D60E087EC94E1F4
:103C40000E94421D682F617085EE99E00C94741DEE
:103C5000CF93DF9380910C1390910D13891B809566
:103C6000877019F40E94A1DFF5CF80910C138F5F4C
:103C70008770A0910C1397E6A99FD0011124FD0134
:103C8000EF5BF64FEF0119929A95E9F798E0908370
:103C9000AA5AB64F90E1EEE1F3E101900D929A95A8
:103CA000E1F720910C1390910D13291303C094E6B2
:103CB0009093091380930C13DF91CF910C94A5C2BC
:103CC0002F923F924F925F926F927F928F929F922C
:103CD000AF92BF92CF92DF92EF92FF920F931F931A
:103CE000CF93DF93D62FC72FFC0180809180A280D5
:103CF000B380C501B40120E831E541E050E00F9404
:103D0000B838C9016DE671E00F9427396B017C0169
:103D1000C501B40120E13EE040E050E00F94B83826
:103D2000CA01B90128E130E040E050E00F94B83812
:103D3000362E272E062F172F8CE3482E512C612C60
:103D4000712CC501B401A30192010F94B838B62EAD
:103D5000A72ECA01B901A30192010F94B838CB0173
:103D6000C114D10479F1AF92BF927F936F932F92D8
:103D70003F92FF92EF92DF92CF9280E29DE09F937D
:103D80008F93CF93DF930F940B328DB79EB70E9620
:103D90000FB6F8949EBF0FBE8DBF8D2F9C2FDF9165
:103DA000CF911F910F91FF90EF90DF90CF90BF9038
:103DB000AF909F908F907F906F905F904F903F90CB
:103DC0002F900895E114F104C9F0AF92BF927F9350
:103DD0006F932F923F92FF92EF9280E19DE09F932D
:103DE0008F93CF93DF930F940B32EDB7FEB73C96D2
:103DF0000FB6F894FEBF0FBEEDBFCFCF012BB9F0C9
:103E0000AF92BF927F936F932F923F9284E09DE099
:103E10009F938F93CF93DF930F940B328DB79EB701
:103E20000A960FB6F8949EBF0FBE8DBFB6CF892BF2
:103E3000A9F0AF92BF927F936F938CEF9CE09F931A
:103E40008F93CF93DF930F940B32EDB7FEB7389675
:103E50000FB6F894FEBF0FBEEDBF9FCFAF92BF92DB
:103E600088EF9CE09F938F93CF93DF930F940B3257
:103E70000F900F900F900F900F900F908ECFCF93C9
:103E8000DF9300D01F92CDB7DEB784EF91E0A0E0C2
:103E9000B0E089839A83AB83BC83BE016F5F7F4FA1
:103EA0008CE30E942EC58BEA9EE00E9492C78CB1E3
:103EB00065EA7EE085FB882780F90E945F1D80917E
:103EC00003016FE97EE0869581700E945F1D89B1D4
:103ED00069E97EE083FB882780F90E945F1D8CB131
:103EE00060E97EE0829581700E945F1D4B9909C058
:103EF0000E9469C50F900F900F900F90DF91CF91A6
:103F000008950E944EC50F900F900F900F90DF9173
:103F1000CF91089580911206882319F0109212060D
:103F2000089540E070E060E080E79EE00E94D0DE0F
:103F3000CF93C091A304CF7739F50E94C1C38823E2
:103F400019F18091BC149091BD14A091BE14B09150
:103F5000BF140097A105B105B9F0BC01CD016D59A1
:103F60007F4F8F4F9F4F24E630E040E050E00F94AA
:103F7000B8386091C0147091C1148091C2149091AE
:103F8000C3140F94B838C22F8C2FCF910895CF93BC
:103F9000DF93EB010E945FBE882319F00E94AFBD42
:103FA000EB01CE01DF91CF9108954F925F926F9216
:103FB0007F928F929F92AF92BF92CF92DF92EF92B9
:103FC000FF921F93CF93DF9300D01F92CDB7DEB740
:103FD00019821A821B821C82CE0101964C018BEA47
:103FE000C82E87E0D82E99E6E92E92E0F92E27E038
:103FF000A22E29E0B22E10E088E5810F0E945FBE5C
:10400000F40181934F01882309F4E0C00E94E7BDC9
:104010002B013C01812F0E94451D882309F4CCC04F
:10402000F7012081318142815381C301B2010F9494
:104030004439F60160837183828393831F5FF4E0C8
:10404000CF0ED11C84E0E80EF11C94E0A90EB11C47
:10405000133091F685E40E945FBE8C83882309F4B7
:10406000C0C00E94E7BD6B017C0183E00E94451D3A
:10407000882371F020917502309176024091770289
:1040800050917802C701B6010F9444396B017C014D
:10409000C092B707D092B807E092B907F092BA077A
:1040A0008091E404882359F18091C41482FF27C0D1
:1040B0008C81882321F18981811103C08A81882321
:1040C000F1F02DEC3CEC4CE45DE360915208709112
:1040D000530880915408909155080F9444399B01DE
:1040E000AC016091710270917202809173029091A3
:1040F00074020F94A43B181614F40F94E72040E0C8
:1041000050E0BA0186E40E94CCBE20E030E0A90174
:104110000F94A43B181684F40E94E7BD20E030E021
:1041200040E752E40F943E3A6093490270934A028A
:1041300080934B0290934C028091790C83FD28C0B0
:104140008091BD05882321F120917502309176027E
:1041500040917702509178026091B7077091B8074B
:104160008091B9079091BA070F9443392091CA05FD
:104170003091CB054091CC055091CD050F94443939
:104180006093CA057093CB058093CC059093CD05C1
:104190000F900F900F900F90DF91CF911F91FF9094
:1041A000EF90DF90CF90BF90AF909F908F907F90D7
:1041B0006F905F904F900895F50120813181428189
:1041C0005381C301B2010F94433933CFF70180818A
:1041D0009181A281B381F60180839183A283B3830D
:1041E0002DCF8091750290917602A0917702B091C7
:1041F00078028093B7079093B807A093B907B0935C
:10420000BA074ECFCF9384E50E945FBEC0E08823FB
:10421000D9F00E94BFBDC82F1816B4F40E94F6DB77
:104220008DE40E946AC780919404909195040E9445
:1042300032F26C2FCC0F770B8DE495E00E9459CAB7
:104240008AE00E946AC7CFEF8C2FCF910895CF925A
:10425000DF92EF92FF920F931F93CF93DF93CDB72F
:10426000DEB7A0970FB6F894DEBF0FBECDBF0E9499
:10427000022187FDCCC085E40E9411BE882309F489
:10428000D5C00E94E7BD6B017C0120E030E0A901B0
:104290000F94A43B87FF04C0F7FAF094F7F8F0946A
:1042A000F7FAF094F7F8F094CD8EDE8EEF8EF8A248
:1042B0008CE0E3E9F2E0DE01119601900D928A951F
:1042C000E1F78AE50E945FBE882351F040E050E0AC
:1042D000BA018AE50E94CCBE69877A878B879C8762
:1042E00088E50E945FBE882351F040E050E0BA01AB
:1042F00088E50E94CCBE69837A838B839C8389E5A1
:104300000E945FBE882351F040E050E0BA0189E589
:104310000E94CCBE6D837E838F83988785E50E9443
:1043200011BE882309F489C00E94E7BD6B017C019E
:1043300020E030E0A901C701B6010F94A43B87FF3C
:1043400004C0F7FAF094F7F8F094F7FAF094F7F85D
:10435000F094C98EDA8EEB8EFC8E1D8A1E8A1F8A1F
:10436000188E8CE40E9411BE882309F46FC00E944D
:10437000E7BD6B017C0120E030E0A901C701B60177
:104380000F94A43B87FF04C0F7FAF094F7F8F09479
:10439000C98ADA8AEB8AFC8A62E070E082E40E94D1
:1043A000E3BEF82E8091A611811131C021E0AE014B
:1043B000475E5F4FBE016F5F7F4FCE014D960E94FB
:1043C00050EE882321F16F2D81E00E9422EF82E5DB
:1043D0000E945FBE882309F442C00E94E3BD40E012
:1043E00050E060EA71E44D875E876F87788B20919B
:1043F000A611222361F08C012F2DAE01435F5F4F88
:10440000BE016F5E7F4FCE0145960E940DEDA096D6
:104410000FB6F894DEBF0FBECDBFDF91CF911F91D5
:104420000F91FF90EF90DF90CF900895C12CD12C89
:1044300080E8E82E80E4F82E33CFC090DC04D090E2
:10444000DD04E090DE04F090DF0472CFC090E00461
:10445000D090E104E090E204F090E3048CCF90E08F
:1044600080E0BDCFCF92DF92EF92FF920F931F9328
:10447000CF93DF93CDB7DEB76C970FB6F894DEBF5E
:104480000FBECDBF8CE40E9411BE882309F4B0C0DA
:104490000E94E7BD6B017C0120E030E0A9010F9490
:1044A000A43B87FF04C0F7FAF094F7F8F094F7FA0A
:1044B000F094F7F8F094C98EDA8EEB8EFC8E8CE0D7
:1044C000E3E9F2E0DE01119601900D928A95E1F7A1
:1044D00088E50E945FBE8823A1F040E050E0BA0169
:1044E00088E50E94CCBE20910709309108094091CF
:1044F000090950910A090F94433969837A838B83A0
:104500009C8389E50E945FBE8823A1F040E050E0D3
:10451000BA0189E50E94CCBE2091070930910809B3
:104520004091090950910A090F9443396D837E83A4
:104530008F8398878AE50E945FBE882351F040E010
:1045400050E0BA018AE50E94CCBE69877A878B87E2
:104550009C871D861E861F86188A8091A611811150
:1045600038C020E0AE01435F5F4FBE016F5F7F4FF9
:10457000CE0149960E9450EE882359F18091E404BF
:1045800081110F94E72060E080E00E9422EF898D86
:104590009A8DAB8DBC8DB0588D8B9E8BAF8BB88FA9
:1045A000198A1A8A1B8A1C8A1D861E861F86188AEB
:1045B0008091A611882369F010E000E020E0AE01B0
:1045C0004B5E5F4FBE016F5E7F4FCE010D960E9426
:1045D0000DED6C960FB6F894DEBF0FBECDBFDF9128
:1045E000CF911F910F91FF90EF90DF90CF900895A2
:1045F000C12CD12C80E8E82E80E4F82E58CF84E638
:1046000090E09093DB048093DA0410920B051092F3
:104610000A050C94FEAE0F93AB010091090521E051
:1046200002272AE035E0BC018AED94E00E94EBC34A
:104630000F910895CF93DF9300D01F92CDB7DEB7CF
:104640008091BD058823C1F083E390E09C838B8338
:104650001A8219829E012F5F3F4F40E150E06EEBBE
:1046600075E0CE0103960E9460DE8DE592E10E9426
:1046700092C78AE00E946AC70F900F900F900F9028
:10468000DF91CF910895CF93DF9300D01F921F92B7
:10469000CDB7DEB781E08093BD0580E1EEEBF5E0BC
:1046A000DF011D928A95E9F70E941A2386E18D8326
:1046B00082E390E09C838B831A8219829E012F5F94
:1046C0003F4F41E050E0BE016B5F7F4FCE0103964C
:1046D0000E9460DE0F900F900F900F900F90DF916F
:1046E000CF910895CF92DF92EF92FF92CF93DF9315
:1046F000EC0108960E94CFB96B017C0120E030E00C
:10470000A9010F94743220E030E0A901882359F008
:10471000CE010E94B8BF9B01AC01C701B6010F9446
:10472000DA329B01AC01688579858A859B850F9477
:104730004339688779878A879B87DF91CF91FF907C
:10474000EF90DF90CF9008958C3221E0920714F023
:104750008CE291E090937112809370120C94EFF0C0
:104760000F931F93CF93DF9305ED1CE0C9EED1E1CA
:10477000F80121913191419151918F0160E070E0F8
:1047800080E89FE30F943E3A6993799389939993D4
:10479000F1E1C93FDF0761F70F94261FDF91CF9149
:1047A0001F910F910C94BA1C90910C1380910D13D2
:1047B000981306C080913F0990914009892B21F000
:1047C00080E00E94A1DFF0CF089590910C138091BA
:1047D0000D13981308C080913F0990914009892BCF
:1047E00011F40C94A7C380E00E94A1DFEECFCF921A
:1047F000DF92EF92FF92CF93DF932091BC0C2223A4
:1048000029F1EC0108960E94CFB96B017C0120E0F0
:1048100030E0A9010F94743220E030E0A901882330
:1048200059F0CE010E94B8BF9B01AC01C701B6018F
:104830000F94DA329B01AC01688579858A859B8566
:104840000F944439688779878A879B87DF91CF9156
:10485000FF90EF90DF90CF900895CF92DF92EF928C
:10486000FF9280913008882309F457C0C0902C082B
:10487000D0902D08E0902E08F0902F0820E030E036
:10488000A901C701B6010F947432882309F445C009
:1048900020E030E040E05FE3C701B6010F94DA3278
:1048A0009B01AC010F94DA322BED3FE049E450E478
:1048B0000F94DA329B01AC0160E070E080E89FE386
:1048C0000F943E3A6B017C01C092BD0CD092BE0C9D
:1048D000E092BF0CF092C00C60917D0270917E025C
:1048E000072E000C880B990B0F947B322AE037EDD2
:1048F00043E25CE30F94DA32A70196010F94DA32B7
:104900006093790270937A0280937B0290937C0289
:10491000FF90EF90DF90CF900895C12CD12C80E8CC
:10492000E82E8FE3F82ED0CF0F931F93CF93DF9312
:1049300050E0FC01E40FF51F8081440F551F440F28
:10494000551F46545B4FEA01882329F188819981DC
:10495000AA81BB81EB01088119812A813B810097E3
:10496000A105B10569F40C591F4F2F4F3F4FDA01D4
:104970000D931D932D933C9313978FEF808306C067
:10498000081B190B2A0B3B0B37FDF7CFDF91CF919B
:104990001F910F910895188219821A821B82F6CFF7
:1049A0002F923F924F925F926F927F928F929F923F
:1049B000AF92BF92CF92DF92EF92FF920F931F932D
:1049C000CF93DF93CDB7DEB76C970FB6F894DEBF09
:1049D0000FBECDBF8C015B015A834983FC01EF5AA6
:1049E000FF4F208131814281538129873A874B874C
:1049F0005C87CA01B9010F9479326B017C01D50142
:104A00002D913D914D915C910F94DA320F94223AA1
:104A10002B013C01E981FA8120813181428153815E
:104A2000C701B6010F94DA320F94223A4B015C01B0
:104A3000C301B2010F94B73A698B7A8B8B8B9C8B35
:104A4000683771058105910540F428E730E040E0C2
:104A500050E0298B3A8B4B8B5C8BC501B4010F94D2
:104A6000B73A6D877E878F87988B68377105810588
:104A7000910540F448E750E060E070E04D875E87C4
:104A80006F87788BF801E35AFF4F40805180628036
:104A90007380C301B2010F947B3269837A838B8365
:104AA0009C8369897A898B899C890F9479326D8B73
:104AB0007E8B8F8B988F20E030E0A90169817A810D
:104AC0008B819C810F947432882309F4E1C1A70182
:104AD0009601C701B6010F94DA324B015C012D89B2
:104AE0003E894F89588DCA01B9010F94DA329B0172
:104AF000AC01C501B4010F9443394B015C0129811C
:104B00003A814B815C81CA01B9010F9444399B0100
:104B1000AC01C501B4010F943E3A0F94223A0F94B0
:104B2000B73A6D837E838F83988766277727CB017B
:104B300064197509860997090F947B324B015C0152
:104B40006D857E858F8598890F9479322B013C0184
:104B500020E030E0A901C501B4010F94743288232C
:104B600009F49AC1A3019201C301B2010F94DA3290
:104B7000698F7A8F8B8F9C8FA7019601C701B60131
:104B80000F94DA329B01AC01698D7A8D8B8D9C8DEF
:104B90000F9443396B017C01A5019401C501B40157
:104BA0000F9444399B01AC01C701B6010F943E3A02
:104BB0000F94E63AD80195968D909D90AD90BC905B
:104BC0009897750164012D813E814F815885C21AE5
:104BD000D30AE40AF50A0F94B73AC61AD70AE80AC4
:104BE000F90AF7FE8EC02D893E894F89588DCA017A
:104BF000B9010F94DA326B017C0129813A814B8132
:104C00005C81CA01B9010F94443969877A878B871F
:104C10009C8720E030E0A90169817A818B819C81A9
:104C20000F947432882309F43BC1C501B4010F9479
:104C3000793229853A854B855C850F94DA32A70154
:104C400096010F9443396D837E838F839887A301E8
:104C50009201C301B2010F94DA329B01AC016D8164
:104C60007E818F8198850F9444392B013C0120E08F
:104C700030E040E850E469817A818B819C810F9417
:104C8000DA329B01AC01C301B2010F943E3A0F949A
:104C9000223A2B013C0120E030E0A9010F94A43B13
:104CA00018161CF0412C512C3201C301B2010F9493
:104CB000B73A6D837E838F83988786169706A806FA
:104CC000B90620F48D829E82AF82B8866D817E8186
:104CD0008F8198850F94793229853A854B855C853B
:104CE0000F94DA32A70196010F9444390F94F23BE6
:104CF0000F94B73A69877A878B879C87C12CD12C10
:104D0000760169857A858B859C8529893A894B89C5
:104D10005C89621B730B840B950B0F94793229818C
:104D20003A814B815C810F943E3A20E034E244EFBB
:104D300059E40F94DA320F94B73A4B015C0169855C
:104D40007A858B859C852D853E854F855889621B8C
:104D5000730B840B950B0F94793229813A814B8127
:104D60005C810F943E3A20E034E244EF59E40F9422
:104D7000DA320F94B73A2B013C013FE683169104D7
:104D8000A104B10408F090C0F401EE0FFF1FEE0F74
:104D9000FF1FE35AF04F85919591A591B4918983B6
:104DA000292E3A2EBD8B4FE644165104610471043E
:104DB00008F083C0F201EE0FFF1FEE0FFF1FE35A52
:104DC000F04F45915591659174919A01CB014D81B8
:104DD0005E816F817885D80199964D935D936D932F
:104DE0007C939C974C0D5D1D6E1D7F1DF80145A7A2
:104DF00056A767A770ABEB5AFF4F49895A896B8951
:104E00007C894083518362837383D5968D929D9272
:104E1000AD92BC92D897F80141AE52AE63AE74AE7B
:104E2000FD9649814083218232825D895383349685
:104E3000208331838283938369857A858B859C85E2
:104E4000D1966D937D938D939C93D49778962D8571
:104E50003E854F85588920833183428353836C96E6
:104E60000FB6F894DEBF0FBECDBFDF91CF911F917B
:104E70000F91FF90EF90DF90CF90BF90AF909F90F9
:104E80008F907F906F905F904F903F902F900895FC
:104E900060E070E0CB0141CE60E070E0CB0188CEF5
:104EA00060E070E0CB01F3CEC501B4010E94BC1BF1
:104EB0006983272E382E9D8B76CFC301B2010E94C5
:104EC000BC1B9B0184CF80910C1390910D13891B07
:104ED000877019F490E080E0089590910913992368
:104EE00051F0833030F48FEF890F19F0809309135C
:104EF000F1CF1092091380910D1327E6829FC00114
:104F000011248F5B964FFC01208120FDE3CF20917F
:104F10000D132F5F277020930A1330910D132091EA
:104F20000B13321304C020910A1320930B1308951E
:104F300090916F0081E091FD02C080E00895909112
:104F40006F009D7F90936F000895CF92DF92EF9254
:104F5000FF92FC01C080D180E280F3802091E10CBF
:104F60003091E20C4091E30C5091E40CC701B60182
:104F70000F94DA320F94B13B60932A1370932B1382
:104F800080932C1390932D13C0921A13D0921B135D
:104F9000E0921C13F0921D1390910C1380910D134D
:104FA000981731F0FF90EF90DF90CF900C94281E6F
:104FB0000E94D4230E94982740912A1350912B13CA
:104FC00060912C1370912D13409336055093370543
:104FD0006093380570933905882331F0FF90EF9086
:104FE000DF90CF900C94A5C2FF90EF90DF90CF9010
:104FF00008954F925F926F927F928F929F92AF929D
:10500000BF92CF92DF92EF92FF920F931F93CF93B5
:10501000DF93EC018B017A016901F90180819181B3
:10502000A281B381FA014081518162817381F801CB
:1050300080809180A280B380488059806A807B8084
:1050400040920E1350920F1360921013709211132E
:105050008092121390921313A0921413B09215130E
:1050600040931613509317136093181370931913EA
:1050700080931A1390931B13A0931C13B0931D13CA
:105080002091E10C3091E20C4091E30C5091E40C42
:10509000F60160817181828193810F94DA320F94DD
:1050A000B13B4B015C012091DD0C3091DE0C409155
:1050B000DF0C5091E00CF701608171818281938156
:1050C0000F94DA320F94B13B6B017C012091D90C23
:1050D0003091DA0C4091DB0C5091DC0CF8016081CE
:1050E0007181828193810F94DA320F94B13B2B014D
:1050F0003C012091D50C3091D60C4091D70C5091A9
:10510000D80C688179818A819B810F94DA320F945F
:10511000B13B60931E1370931F13809320139093E1
:105120002113409222135092231360922413709201
:105130002513C0922613D0922713E0922813F092E1
:10514000291380922A1390922B13A0922C13B092C1
:105150002D1390910C1380910D13981791F0DF91FE
:10516000CF911F910F91FF90EF90DF90CF90BF9064
:10517000AF909F908F907F906F905F904F900C9426
:10518000281E0E94D4230E949827409126135091F4
:105190002713609128137091291300912213109105
:1051A00023132091241330912513C0901E13D09007
:1051B0001F13E0902013F0902113C0922A05D09283
:1051C0002B05E0922C05F0922D0500932E051093EF
:1051D0002F052093300530933105409332055093CD
:1051E0003305609334057093350540912A1350912F
:1051F0002B1360912C1370912D134093360550930F
:1052000037056093380570933905882391F0DF9155
:10521000CF911F910F91FF90EF90DF90CF90BF90B3
:10522000AF909F908F907F906F905F904F900C9475
:10523000A5C2DF91CF911F910F91FF90EF90DF906A
:10524000CF90BF90AF909F908F907F906F905F9026
:105250004F900895CF92DF92EF92FF92CF93DF931A
:10526000C82F0E94982794E0C99FE0011124FE01F5
:10527000E65DFA4FC080D180E280F38081110E9408
:10528000A5C2C751DE4EC701B6010F947B322881FB
:1052900039814A815B810F94DA32DF91CF91FF909F
:1052A000EF90DF90CF9008953F924F925F926F9270
:1052B0007F928F929F92AF92BF92CF92DF92EF92A6
:1052C000FF920F931F93CF93DF93CDB7DEB768970D
:1052D0000FB6F894DEBF0FBECDBFD82E2A013B011A
:1052E000480159013E2C20E030E0A901C501B80178
:1052F0000F947432811110C081E08D1508F0B6C092
:1053000060E070E080E793E420E030E040E752E4C2
:105310000F943E3A4B015C018D8A9E8AAF8AB88E0B
:105320000D2D10E0F801E65AF04FE491BB24B39440
:105330001E160CF4B12CCC24C39420E030E0A9015B
:10534000C301B2010F94A43B18160CF0C12CBC147D
:1053500071F092E0D9120BC0332049F081E00F9434
:10536000AE2269E170E080E090E00E94C2C280E07D
:105370000E942A2969837A838B839C8381E00E941F
:105380002A296D837E838F83988782E00E942A2951
:1053900069877A878B879C8783E00E942A296D879B
:1053A0007E878F87988B000F111F000F111FE1E080
:1053B000F0E0EC0FFD1F0E0F1F1FF801108211828D
:1053C000128213829E01235F3F4FAE01475F5F4F02
:1053D000BE016B5F7F4FCE0101960E94F927F80155
:1053E0004082518262827382198A1A8A1B8A1C8ABD
:1053F00080913F0990914009892B91F4CE0141960B
:105400007C018E010B5E1F4F9E01235F3F4FAE015B
:10541000475F5F4FBE016B5F7F4F40970E944EF822
:105420000E94D423BC1451F092E0D91205C033205D
:1054300019F080E00F94AE220E948A1F68960FB682
:10544000F894DEBF0FBECDBFDF91CF911F910F91BA
:10545000FF90EF90DF90CF90BF90AF909F908F9094
:105460007F906F905F904F903F90089560E070E85C
:105470008BE395E449CFCF92DF92EF92FF92CF93E7
:10548000DF93C82F0E94982794E0C99FE001112460
:10549000FE01E25EFA4FC080D180E280F38081118C
:1054A0000E94A5C2C751DE4EC701B6010F947B32E0
:1054B000288139814A815B810F94DA32DF91CF9163
:1054C000FF90EF90DF90CF9008950E9498279091E1
:1054D0000D1390930C1390930B1390930A1394E66F
:1054E0009093091320ED33E03093400920933F0956
:1054F00081110E94A5C281E080931D05089580FF5F
:1055000004C09091BB0C90FD8E7F81FF05C09091EF
:10551000BB0C969590FD8D7F82FF06C09091BB0CD1
:105520009695969590FD8B7F08958F929F92AF925E
:10553000BF92CF92DF92EF92FF92CF93DF932091B1
:105540004D02222309F49EC0EC0180918E04C82EE6
:10555000D12CF12CE12C80FF2CC080904F02909038
:105560005002A0905102B0905202288139814A81A4
:105570005B81C501B4010F94A43B181624F4888202
:105580009982AA82BB8280905B0290905C02A0907C
:105590005D02B0905E02288139814A815B81C5013C
:1055A000B4010F94743287FF04C088829982AA8262
:1055B000BB82D701C601B695A7959795879580FFC1
:1055C0002CC08090530290905402A0905502B0904D
:1055D00056022C813D814E815F81C501B4010F943B
:1055E000A43B181624F48C829D82AE82BF828090E8
:1055F0005F0290906002A0906102B09062022C81E4
:105600003D814E815F81C501B4010F94743287FFE3
:1056100004C08C829D82AE82BF8282E0F694E794C1
:10562000D794C7948A95D1F7C0FE2CC0C09057027A
:10563000D0905802E0905902F0905A02288539859E
:105640004A855B85C701B6010F94A43B181624F464
:10565000C886D986EA86FB86C0906302D090640231
:10566000E0906502F0906602288539854A855B8561
:10567000C701B6010F94743287FF04C0C886D9866B
:10568000EA86FB86DF91CF91FF90EF90DF90CF907D
:10569000BF90AF909F908F9008952F923F924F921E
:1056A0005F926F927F928F929F92AF92BF92CF92B2
:1056B000DF92EF92FF920F931F93CF93DF93CDB7BB
:1056C000DEB7A6970FB6F894DEBF0FBECDBF8BEA4C
:1056D00097E00E94952A8091790C83FD7EC02091ED
:1056E0007502309176024091770250917802609174
:1056F000B7077091B8078091B9079091BA070F94D6
:105700007432882309F469C010913E09111161C0F7
:105710008091670290916802019720916E123091FA
:105720006F12281739073CF40E94F6DB84EE9EE0E6
:105730000E9492C711E0209175023091760240914B
:105740007702509178026091B7077091B807809105
:10575000B9079091BA070F9443396B017C0120E09F
:1057600030E0A9010F94A43B87FF04C0F7FAF0943E
:10577000F7F8F0942091790230917A0240917B02FF
:1057800050917C02C701B6010F94DA3220E030E874
:105790004BE354E40F94A43B1816ECF40E94F6DBA0
:1057A00085EC9EE00E9492C78091B7079091B80760
:1057B000A091B907B091BA078093750290937602D1
:1057C000A0937702B093780287EB97E00E94A52719
:1057D00004C010E0B0CF1111E7CF2AE037ED43E26B
:1057E0005CE36091490270914A0280914B02909172
:1057F0004C020F94DA326B017C0160917F02709150
:105800008002072E000C880B990B0F947B329B01B2
:10581000AC01C701B6010F94DA32698B7A8B8B8B9E
:105820009C8B8091BC0C882309F180900309909097
:105830000409A0900509B0900609C090B307D09064
:10584000B407E090B507F090B60720E030E0A9017A
:10585000C501B4010F9474328823D1F1A7019601D8
:10586000C501B4010F94A43B181694F1C12CD12C9E
:1058700076018E010F5E1F4F27EB37E043EB57E0B9
:105880006FEA77E08BEA97E00F94BE0780E1EBEADE
:10589000F7E0A9E6B2E001900D928A95E1F7A696AD
:1058A0000FB6F894DEBF0FBECDBFDF91CF911F9131
:1058B0000F91FF90EF90DF90CF90BF90AF909F90AF
:1058C0008F907F906F905F904F903F902F900895B2
:1058D0002091690230916A0240916B0250916C02F2
:1058E0006091AB077091AC078091AD079091AE07C6
:1058F0000F9443396D8B7E8B8F8B988F20916D0227
:1059000030916E0240916F02509170026091AF072A
:105910007091B0078091B1079091B2070F9443390D
:10592000698F7A8F8B8F9C8F2091710230917202D8
:105930004091730250917402C701B6010F9443392C
:105940006D8F7E8F8F8F98A3209175023091760294
:1059500040917702509178026091B7077091B80733
:105960008091B9079091BA070F9443396B017C017C
:1059700020E030E0A9016D897E898F89988D0F9490
:10598000743281110CC020E030E0A901698D7A8D5C
:105990008B8D9C8D0F947432882309F467CF2D89E9
:1059A0003E894F89588DCA01B9010F94DA324B01F3
:1059B0005C01298D3A8D4B8D5C8DCA01B9010F9424
:1059C000DA329B01AC01C501B4010F9444394B019B
:1059D0005C012D8D3E8D4F8D58A1CA01B9010F94E8
:1059E000DA329B01AC01C501B4010F9444394B017B
:1059F0005C01A7019601C701B6010F94DA329B0141
:105A0000AC01C501B4010F9444390F94F23B4B0132
:105A10005C012DEB37E346E855E30F94743287FFC2
:105A20000FC020E030E0A901C701B6010F94A43BEC
:105A30004601570187FF04C0B7FAB094B7F8B09495
:105A40002DEB37E346E855E3C501B4010F947432FA
:105A500087FD1CCF20E030E040EA51E4C501B401ED
:105A60000F943E3A0F94B73A1B01672B19F4222486
:105A70002394312CB10190E080E00F9479329B01A6
:105A8000AC0160E070E080E89FE30F943E3A2B01A8
:105A90003C01AC019B01C501B4010F94DA324B010A
:105AA0005C01A30192016D897E898F89988D0F9485
:105AB000DA326D8B7E8B8F8B988FA3019201698D6B
:105AC0007A8D8B8D9C8D0F94DA32698F7A8F8B8FC4
:105AD0009C8FA30192016D8D7E8D8F8D98A10F9467
:105AE000DA326D8F7E8F8F8F98A3A3019201C70149
:105AF000B6010F94DA3269A37AA38BA39CA380E149
:105B0000E9E6F2E08E010F5F1F4FD80101900D9280
:105B10008A95E1F70E942A742B013C0128EC420E81
:105B2000511C611C711C0DA31EA381E0281A3108B1
:105B300009F460C00E942A748B019C0104191509A4
:105B40002609370937FD59C02B013C0128EC420ECC
:105B5000511C611C711C80E00E94A1DF2D893E89CF
:105B60004F89588D69817A818B819C810F9444394A
:105B700069837A838B839C83298D3A8D4B8D5C8DD1
:105B80006D817E818F8198850F9444396D837E83EA
:105B90008F8398872D8D3E8D4F8D58A169857A858D
:105BA0008B859C850F94443969877A878B879C877E
:105BB00029A13AA14BA15CA16D857E858F8598892D
:105BC0000F9444396D877E878F87988B75016401A8
:105BD0008E010F5E1F4F9E01235F3F4FAE01475F57
:105BE0005F4FBE016B5F7F4F8DA19EA10F94BE07DB
:105BF00081119BCF750164013CCE0E94388FAECFDE
:105C00008091B6049091B704A091B804B091B90402
:105C10008093490290934A02A0934B02B0934C02A6
:105C20008091B4049091B5049093800280937F0298
:105C300008958091490290914A02A0914B02B0913F
:105C40004C028093B6049093B704A093B804B09329
:105C5000B90480917F02909180029093B504809363
:105C6000B40484E690E09093800280937F020895CC
:105C70008F929F92AF92BF92CF92DF92EF92FF925C
:105C8000CF93DF938090490290904A02A0904B02FC
:105C9000B0904C02FC01C080D180E280F38020E013
:105CA00030E0A901C701B6010F947432882341F096
:105CB000C0924902D0924A02E0924B02F0924C020A
:105CC000C0917F02D091800284E690E090938002A0
:105CD00080937F02C0907902D0907A02E0907B029C
:105CE000F0907C0280E090E0A0E8BFE3809379022E
:105CF00090937A02A0937B02B0937C020E944D2B7A
:105D00008092490290924A02A0924B02B0924C02B9
:105D1000D0938002C0937F02C0927902D0927A021F
:105D2000E0927B02F0927C02DF91CF91FF90EF90A6
:105D3000DF90CF90BF90AF909F908F9008950F937A
:105D40001F93CF93DF9300D01F92CDB7DEB79C0196
:105D50000BEA17E090E1E9E6F2E0D80101900D923C
:105D60009A95E1F7F9012081318142815381F8014F
:105D700060857185828593850F944439F801608729
:105D800071878287938780E090E0A0EAB0E48983FE
:105D90009A83AB83BC83CE0101960E94382E0F906C
:105DA0000F900F900F90DF91CF911F910F91089559
:105DB000AF92BF92CF92DF92EF92FF920F931F9319
:105DC000CF93DF93CDB7DEB764970FB6F894DEBFFD
:105DD0000FBECDBF0E94022187FDAFC08AE50E94A1
:105DE0005FBE882309F4BAC040E050E0BA018AE5FA
:105DF0000E94CCBE7B018C01209171023091720215
:105E0000409173025091740260E070E088EC93E47A
:105E10000F9443395B016C019701A8010F94A43BD7
:105E2000181614F07501860120E030E0A901B701D1
:105E3000C8010F94A43B181624F4E12CF12C00E0C7
:105E400010E0B701C8010F94B03A072E000C880B80
:105E5000990B0F947B32698B7A8B8B8B9C8B20E018
:105E600030E0A9010F947432882321F0CE014196CD
:105E70000E949F2E80E090E0A0EAB1E48D879E878B
:105E8000AF87B88B19861A861B861C868CE40E9405
:105E900011BE882309F467C00E94E7BD6B017C0135
:105EA00020E030E0A901C701B6010F94A43B87FFB1
:105EB00004C0F7FAF094F7F8F094CD82DE82EF8216
:105EC000F88620917012309171122430310574F0EF
:105ED00080916E1290916F12821B930B97FF03C0FB
:105EE00091958195910901E004970CF400E080E020
:105EF0000E94ACEC882359F022E0AE01435F5F4F73
:105F0000BE016B5F7F4FCE0109960E94C9EB698984
:105F10007A898B899C898B019C01305809831A836B
:105F20002B833C8320E030E0A9010F947432882356
:105F300021F0CE0101960E949F2E64960FB6F89430
:105F4000DEBF0FBECDBFDF91CF911F910F91FF90AC
:105F5000EF90DF90CF90BF90AF900895E12CF12C9F
:105F600000E211E449CFC090E004D090E104E09059
:105F7000E204F090E30494CFCF92DF92EF92FF928D
:105F80000F931F93C12CD12C76018C0125E732E0B1
:105F900041E752E06DE672E089E692E00F94BE07B9
:105FA0001F910F91FF90EF90DF90CF9008954F9247
:105FB0005F926F927F928F929F92AF92BF92CF9299
:105FC000DF92EF92FF920F931F93CF93DF93CDB7A2
:105FD000DEB72C970FB6F894DEBF0FBECDBF2B01F6
:105FE0003C0129873A874B875C8747015801F601B6
:105FF000E080F1800281138120E030E0A901B70147
:10600000C8010F947432882309F488C05E2D4F2D87
:10601000302F212F852F942FA32FB22F89839A837E
:10602000AB83BC8320E030E0A901B701C8010F9425
:106030007432811108C0E0904502F0904602009150
:10604000470210914802C701D8018D839E83AF8318
:10605000B887A501940160917102709172028091DC
:106060007302909174020F94743287FF0CC0809277
:10607000710290927202A0927302B0927402CE01E9
:1060800001960E94BC2F4092690250926A0260926F
:106090006B0270926C0289859A85AB85BC85809372
:1060A0006D0290936E02A0936F02B0937002CE01C6
:1060B00005960E94BC2FA501940160917102709118
:1060C000720280917302909174020F94A43B18168F
:1060D00064F48092710290927202A0927302B09264
:1060E0007402CE0101960E94BC2F0E94D4232C96EC
:1060F0000FB6F894DEBF0FBECDBFDF91CF911F91D9
:106100000F91FF90EF90DF90CF90BF90AF909F9056
:106110008F907F906F905F904F90089550E040E097
:1061200030E820E477CFCF92DF92EF92FF920F9387
:106130001F936A01E0907102F09072020091730265
:1061400010917402FB012081318142815381FC0155
:1061500060817181828193810E94D72F1F910F915D
:10616000FF90EF90DF90CF900895CF92DF92EF9263
:10617000FF920F931F936B01FC01E080F18002817D
:106180001381E9E6F2E024813581468157816081FF
:106190007181828193810E94D72F1F910F91FF906F
:1061A000EF90DF90CF900895AF92BF92CF92DF92A1
:1061B000EF92FF920F931F93CF93DF9300D01F9224
:1061C000CDB7DEB7FC01E080F1800281138161115F
:1061D00012C0A0907102B0907202C0907302D09071
:1061E00074029501A601B701C8010F94743287FFAC
:1061F00002C07501860120E030E048EC53E4B701AD
:10620000C8010F94743287FD04C0E12CF12C08EC16
:1062100013E4C701D80189839A83AB83BC836EEEF4
:1062200072E0CE0101960E94B5300F900F900F9052
:106230000F90DF91CF911F910F91FF90EF90DF9022
:10624000CF90BF90AF900895EF92FF920F931F935E
:10625000CF93DF937C018B010E9476C3C9E6D2E025
:106260002091790230917A0240917B0250917C0218
:10627000F70160817181828193810F943E3A2C8570
:106280003D854E855F850F9444396C877D878E8769
:106290009F87C8010E94BC2FDF91CF911F910F9162
:1062A000FF90EF900C94D4238F929F92AF92BF9265
:1062B000CF92DF92EF92FF921F93CF93DF93CDB7F0
:1062C000DEB760970FB6F894DEBF0FBECDBF182FB4
:1062D00080E00E942A294B015C018092A8049092E0
:1062E000A904A092AA04B092AB0481E00E942A29DA
:1062F0006B017C01C092AC04D092AD04E092AE047C
:10630000F092AF0482E00E942A296093B004709357
:10631000B1048093B2049093B3041D861E861F8639
:10632000188A89829A82AB82BC82CD82DE82EF8219
:10633000F88669877A878B879C8783E00E942A2961
:106340006D877E878F87988B8091BC0C882321F086
:10635000CE0101960E9472231E3FD9F480E1FE0116
:106360003196A9E6B2E001900D928A95E1F7609628
:106370000FB6F894DEBF0FBECDBFDF91CF911F9156
:10638000FF90EF90DF90CF90BF90AF909F908F9055
:10639000089584E0189FF0011124DF01A759BD4F33
:1063A00081E090E08C0F9D1FE80FF91F4081518123
:1063B000628173814D935D936D937C931397D7CFD7
:1063C0000D94261F0F931F93CF93DF93EC018B0146
:1063D00081E00F94AE2269E170E080E090E00E94DD
:1063E000C2C2B801CE010E94B530C091120680E051
:1063F0000F94AE221092120682E00E9454310E9445
:10640000E031C2FBCC27C0F981E08C27DF91CF912E
:106410001F910F910895CF93DF93CDB7DEB72C97DF
:106420000FB6F894DEBF0FBECDBF0F9404200E94BC
:1064300098279CE0EAE2F5E0DE01119601900D92CA
:106440009A95E1F781110E94A5C2CE0101960E94A2
:10645000A2972C960FB6F894DEBF0FBECDBFDF918A
:10646000CF9108952F923F924F925F926F927F92B9
:106470008F929F92AF92BF92CF92DF92EF92FF9254
:106480000F931F93CF93DF9300D0CDB7DEB78090EB
:10649000690290906A02A0906B02B0906C024090EA
:1064A0006D0250906E0260906F0270907002C0900A
:1064B0007102D0907202E0907302F09074020E9418
:1064C000BA1C0E942D240DE312E18FE492E09B831D
:1064D0008A8381E3282E82E1382E198289810E94E5
:1064E000081DC8010E9474B8EA81FB816193719311
:1064F00081939193FB83EA83C1010E9474B8EA817E
:10650000FB816087718782879387F981FF5FF983B9
:106510000C5F1F4F84E0280E311CF330F9F685E044
:1065200095E00F9469200E9448C20E94B023A50103
:1065300094016091690270916A0280916B0290915E
:106540006C020F94743281111CC0A30192016091FE
:106550006D0270916E0280916F02909170020F94A3
:10656000743281110EC020917102309172024091FB
:10657000730250917402C701B6010F9474328823DC
:10658000B9F00F900F900F90DF91CF911F910F9165
:10659000FF90EF90DF90CF90BF90AF909F908F9043
:1065A0007F906F905F904F903F902F900C940B32A4
:1065B0000F900F900F90DF91CF911F910F91FF904F
:1065C000EF90DF90CF90BF90AF909F908F907F9093
:1065D0006F905F904F903F902F9008958091A70407
:1065E000659B6EC080618093A704909103018091A8
:1065F000A70491FF67C080628093A7048091A704DD
:106600004B9B62C084608093A7048091A704909103
:10661000A604981709F45AC092E09093A5048093B9
:10662000A6048091CF05811105C08091BB07882306
:1066300009F459C080911C0580FF10C08091D005DD
:1066400080FD0CC08091A40484FF08C080911206D4
:1066500080618093120680E00E94C29780911C05A1
:10666000869580FF11C08091D005869580FD0CC075
:106670008091A40485FF08C08091120680628093F7
:10668000120681E00E94C29780911C05869586952E
:1066900080FF29C08091D0058695869580FF23C014
:1066A0008091BB078823F9F08091A40482FF1BC06E
:1066B0008091120684608093120682E00C94C29747
:1066C0008F7E91CF8F7D98CF8B7F9DCF8091A504BA
:1066D000882309F4A6CF81508093A5048111A1CF0E
:1066E0009093A4049ECF08958091CF05811104C09A
:1066F0008091BB07882331F062E070E080E090E099
:106700000C94C2C208953F924F925F926F927F9213
:106710008F929F92AF92BF92CF92DF92EF92FF92B1
:106720000F931F93CF93DF9300D01F92CDB7DEB7A7
:10673000382E80E090E0A0E2B1E489839A83AB83B5
:10674000BC83C0900313D0900413E0900513F09025
:10675000061320E030E0A901C701B6010F9474329E
:1067600087FF0CC0A701960160E070E080E291E431
:106770000F94433969837A838B839C8360E0CE01D5
:1067800001960E94D4304090690250906A02609055
:106790006B0270906C0280906D0290906E02A090DF
:1067A0006F02B0907002332089F10E9417DE1982C7
:1067B0001A821B821C82E0907102F090720200919A
:1067C000730210917402CE0101966C01A50194012F
:1067D000C301B2010E94D72F3092BB070E947433CD
:1067E0000F900F900F900F90DF91CF911F910F910D
:1067F000FF90EF90DF90CF90BF90AF909F908F90E1
:106800007F906F905F904F903F9008950E94D4DDED
:10681000CECF2F923F924F925F926F927F928F9244
:106820009F92AF92BF92CF92DF92EF92FF920F931F
:106830001F93CF93DF93CDB7DEB766970FB6F8946B
:10684000DEBF0FBECDBFF82E282E312CF101E65A47
:10685000F04FD49022E0821335C08091BB078111A4
:1068600003C081E00E9483330E9417DE811139C189
:1068700086E59FE00E9474B820E030E0A9010F9403
:1068800074328823F9F06D2DDD0C770B880B990B92
:106890000F947B322B013C0186E59FE00E9474B887
:1068A0004B015C0120E030E040EA50E40F94743288
:1068B00011E087FF1CC0812C912C90EAA92E90E456
:1068C000B92E15C06D2DDD0C770B880B990B0F942D
:1068D0007B322B013C01C101880F991F880F991F42
:1068E000825B904F0E9474B84B015C0110E0A301E1
:1068F0009201C501B4010F94DA324B015C016101D0
:10690000CC0CDD1CCC0CDD1CC6018E5B904F0E94B4
:1069100074B8EE24E394E12620E030E040EC5FE33D
:106920000F94DA32A30192010F94DA32AB01BC0169
:1069300000E010E098018F2D0E94542920E030E003
:10694000A901C501B4010F947432F601EA5CF04F5D
:10695000FA8BE98B882309F44DC0F2E000E010E0E7
:1069600020E431E4FF1619F000E010E09801B501D1
:10697000A4017058E12C8F2D0E945429A501940187
:10698000C501B4010F9444396B8B7C8B8D8B9E8B2E
:1069900022E0F216E9F0F101ED5CF04F6491611133
:1069A00007C00E94F6DB81E19FE00E9492C76AE087
:1069B00070E090E080E00F9479329B01AC0160E0E0
:1069C00070E088E492E40F943E3A8B019C0104C08D
:1069D00000E010E020EC30E4EE24E3944B895C8985
:1069E0006D897E898F2D0E94542932E0F312D0C028
:1069F0000E94D4DD81E090E0A0E0B0E00F2C04C064
:106A0000880F991FAA1FBB1F0A94D2F72091BB0CB5
:106A1000282B2093BB0C20918E04822B80938E0414
:106A200089899A890E9474B8F601E759FD4F6083FD
:106A300071838283938382E0F8121AC0209103133A
:106A40003091041340910513509106136091710227
:106A50007091720280917302909174020F94433985
:106A60006093710270937202809373029093740228
:106A7000F601EF5CF74F10821182128213828F2D84
:106A80000E94081D0E94E031F601E759FD4F808108
:106A90009181A281B381F601E555F84F80839183FE
:106AA000A283B38392E0F916A9F18CE0EFE9F2E05A
:106AB000DE01119601900D928A95E1F7E1E0F0E098
:106AC000EC0FFD1FEC0DFD1D80809180A280B38036
:106AD00020E030E0A901C501B4010F9474328111A6
:106AE0001EC066960FB6F894DEBF0FBECDBFDF9115
:106AF000CF911F910F91FF90EF90DF90CF90BF90BB
:106B0000AF909F908F907F906F905F904F903F904D
:106B10002F9008950E947AB88111E3CFC6CF20E06C
:106B200030E0A901C501B4010F94A43B87FF04C064
:106B3000B7FAB094B7F8B094F601E759FD4F6F017A
:106B4000A3019201C501B4010F94DA329B01AC019B
:106B5000F60160817181828193810F944339F6013E
:106B60006083718382839383F2E080E090E0A0E40D
:106B7000B1E4FF1621F080E090E0A8E4B2E48D8754
:106B80009E87AF87B88BCE010D960E94BC2FA9CFF0
:106B900081E090E0A0E0B0E00F2C04C0880F991FC6
:106BA000AA1FBB1F0A94D2F72091BB0C282B20935D
:106BB000BB0C20918E04822B80938E0489899A8944
:106BC0000E9474B8F601E759FD4F60837183828398
:106BD00093834ECF0F931F938091A711813019F5A6
:106BE0000E942A740091C2041091C3042091C4042D
:106BF0003091C504601B710B820B930B28EE33E0C0
:106C000040E050E00F94B8386091C6047091C7041A
:106C10008091C8049091C904620F731F841F951F4F
:106C20001F910F9108956091CA047091CB048091D7
:106C3000CC049091CD04D6CF1092A7111092C2042B
:106C40001092C3041092C4041092C5041092CA0496
:106C50001092CB041092CC041092CD041092C60472
:106C60001092C7041092C8041092C90408958F921C
:106C70009F92AF92BF92CF92DF92EF92FF920F93CB
:106C80001F93CF93DF93CDB7DEB72C970FB6F89451
:106C9000DEBF0FBECDBF8B0140E050E068E472E480
:106CA0004D835E836F83788740E050E060EA70E454
:106CB00049875A876B877C878130B9F1823009F424
:106CC00059C020E030E040E050E4609171027091E2
:106CD000720280917302909174020F9444394B01B7
:106CE0007C0120E030E048EC53E40F94A43B1816FC
:106CF00034F4812C912C88ECE82E93E4F92EF801E1
:106D0000A084B184C284D3849401A701B501C601D3
:106D10000F94A43B181614F054016701C501D60165
:106D200089839A83AB83BC8348C0BE01675F7F4F72
:106D3000C80108960E94B530B8016C5F7F4FAE0164
:106D40004B5F5F4FC8010E9493300E940B322C961C
:106D50000FB6F894DEBF0FBECDBFDF91CF911F916C
:106D60000F91FF90EF90DF90CF90BF90AF909F90EA
:106D70008F900895F8012085318542855385609173
:106D800071027091720280917302909174020F945B
:106D900044396B017C0120E030E048EC53E40F946F
:106DA000743287FD06C0C12CD12C28ECE22E23E4DE
:106DB000F22EC982DA82EB82FC82BE01675F7F4FCE
:106DC000CE010196B7CFCF92DF92EF92FF92CF9391
:106DD000DF93C62FFC01C080D180E280F38020E0E9
:106DE00030E0A901C701B6010F94743220E030E011
:106DF000A90187FD14C020E030E048EC52E4C7014F
:106E0000B6010F94A43B24E630E040E050E01816B1
:106E100034F0C701B6010F94B03A9B01AC01C23007
:106E2000A0F4D0E0C45CD64FAFEFB0E00F94F938D7
:106E300024E630E040E050E00F94DA382F3F31058F
:106E400019F010F02FEF30E02883DF91CF91FF9001
:106E5000EF90DF90CF900895ECE3F5E0108211827F
:106E60001282138214820C94EFF0EF92FF920F9330
:106E70001F93CF93DF93CDB7DEB78C01EDB6FEB68F
:106E80000F94C13101962DB73EB7281B390B0FB6B1
:106E9000F8943EBF0FBE2DBF8DB79EB70196B801C7
:106EA0000F94BA310F9461230FB6F894FEBE0FBE53
:106EB000EDBEDF91CF911F910F91FF90EF9008955C
:106EC0008091090180FD06C08091C41483FB88274E
:106ED00080F9089580E00895CF92DF92EF92FF92BB
:106EE000FC01C080D180E280F380663019F51092F9
:106EF00041051092420510924305109244051092EC
:106F000045050E94BE8B20E030E0A901C701B60113
:106F10000F94743287FF1DC0C12CD12C7601C7019C
:106F2000B6010F94B13BCB01FF90EF90DF90CF9073
:106F30000C9463BD0E942C3720E030E0A901C7010A
:106F4000B6010F94743287FF15C0C12CD12C760185
:106F500021C020E030E04CE053E4C701B6010F94BB
:106F6000A43B1816E4F6C12CD12C9CE0E92E93E446
:106F7000F92ED5CF20E030E046E953E4C701B60151
:106F80000F94A43B181634F4C12CD12C86E9E82EBA
:106F900083E4F82EC701B6010F94B13BCB01FF90FB
:106FA000EF90DF90CF900C94A4239091BB0C97703E
:106FB00081E0973009F080E0089520918D0420FF52
:106FC00014C020E83EE3629FA001639F500D729FB2
:106FD000500D1124CA01969587959695879500972F
:106FE00031F08A950000E9F708950C94C2C2089523
:106FF000CF93DF9310927A0C10920D0D10920F0D1B
:1070000010920E0D1092A2041092A104CFEFDFEFA8
:107010008091C41485FD07C00E94D777D093431395
:10702000C0934213F5CF8FEF9FEF9093431380935C
:107030004213DF91CF9108958F929F92AF92BF92AA
:10704000CF92DF92EF92FF920F931F93CF93DF9334
:107050007C0121E5E20EF11CD7014C914A3509F083
:10706000A4C06C01B2E5CB0ED11CF6013081353ADB
:1070700009F09BC0EC01C05BDF4F2881233008F48E
:1070800094C08C0100561F4FD8014C93E15BFF4F19
:10709000308331962083EF54F1093081E05BFF4F5C
:1070A00030833038B1F43196AC54B1093C9130831F
:1070B000E854F109AF5ABF4F50E040E02250330B83
:1070C00042175307CCF4808132968D934F5F5F4F08
:1070D000F7CF233031F5313809F074C0FC01EC559D
:1070E000FF4FDC01AC5ABF4F2C9120833196885A58
:1070F0009F4FDC018C9180834801B12CA12C8881A9
:1071000090E002968A159B050CF43FC0F401819132
:107110004F010E94FBC50E941CF1FFEFAF1ABF0A8E
:10712000EECF323821F5FC01EC5AFF4F308141811E
:10713000E05BFF4F408331963083DC01AA55BF4F9F
:1071400050E040E02350330B42175307ACF6FA01EE
:10715000EE7FE45AFF4FE80FF91F608171817C9345
:1071600011966C9311974E5F5F4F1296EDCF2430BE
:1071700019F6333809F6FC01EC5AFF4F20813181B2
:10718000E05BFF4F30833196B0CF80E5DE011D928A
:107190008A95E9F78AE1F80111928A95E9F78AE57B
:1071A000D7018C9385EAF6018083DF91CF911F91FF
:1071B0000F91FF90EF90DF90CF90BF90AF909F9096
:1071C0008F900895323809F097CFADCFCF93DF93EA
:1071D000D091A71189E192E10E9492C78AE00E94B2
:1071E0006AC78091260D873009F449C083E08093F7
:1071F000240D81E08093860280E190E090935B14FF
:1072000080935A1485E080934E14C2E8C0935114C1
:1072100084E190E1A0E0B0E0809352149093531485
:10722000A0935414B09355148EEF93E10E941C3830
:1072300061E070E080E090E00E94DD3781E09AE557
:1072400090935B1480935A1485E390E090935D14BF
:1072500080935C1487E080934E14C093511484E8AB
:1072600090E0A0E0B0E08093521490935314A09368
:107270005414B09355148EEF93E10E941C38809102
:10728000A711813089F1823061F50E94EA3560935F
:10729000C6047093C7048093C8049093C90481E026
:1072A0008093A7110E942A746093C2047093C30450
:1072B0008093C4049093C504D23089F08091BE05B8
:1072C0009091BF0501969093BF058093BE051092E3
:1072D0008F0410929004109291041092920481E015
:1072E00004C00E941C36DBCF80E0DF91CF9108956F
:1072F0000E942DF51092BA0C10922D020E94C1C36B
:10730000882351F08091C41482FD06C084E49EE07D
:1073100090930A0D8093090D61E08DE39EE00E9439
:10732000A1C80C94E6388091A7118130C1F589E598
:107330009EE00E9492C78AE00E946AC781E09AE5B7
:1073400090935B1480935A1487E590E090935D14BA
:1073500080935C1487E080934E1482E880935114EC
:1073600084E890E0A0E0B0E080935214909353142E
:10737000A0935414B09355148EEF93E10E941C38DF
:1073800082E08093A7110E942A746093CA047093CC
:10739000CB048093CC049093CD0481E0089580E0E9
:1073A00008950F931F930E942A740091B9051091BC
:1073B000BA052091BB053091BC05011511052105C9
:1073C000310509F067C020913013222309F45FC012
:1073D000E0912E1321502093301321E02E0F2093A3
:1073E0002E1330913113231302C010922E1324E078
:1073F000E29FF0011124EE5CFC4E0081118122819C
:1074000033810093B5051093B6052093B7053093EB
:10741000B805600F711F811D911D6093B9057093B0
:10742000BA058093BB059093BC058091B7059091F8
:10743000B805892B61F11FB7F89488E49EE00E949B
:1074400092C78AE00E946AC784E096E090935B143A
:1074500080935A1480EA90E890935D1480935C14B2
:1074600087E080934E1482E88093511480EA90E084
:10747000A0E0B0E08093521490935314A09354145E
:10748000B09355148EEF93E10E941C381FBF1F91DB
:107490000F910895601B710B820B930B97FDF7CF33
:1074A00040981092B9051092BA051092BB0510923F
:1074B000BC05EDCF0F931F93CF93DF938C01EB01AE
:1074C0009091301320913113921305C00E94D1394D
:1074D0000E94388FF5CF80912F1334E0839FF00105
:1074E0001124EE5CFC4E11830083D383C2839F5F23
:1074F000909330138F5F281739F080932F13DF910B
:10750000CF911F910F91089510922F13F8CF2F92C2
:107510003F924F925F926F927F928F929F92AF9223
:10752000BF92CF92DF92EF92FF920F931F93CF9370
:10753000DF93009709F0AAC110920F0D10920E0D63
:107540009093A2048093A104BAE0CB2EB0E2DB2E8C
:10755000E12CF12C15E002E846015701C4E1D0E02E
:107560001092A1131092A0131093941300939713E9
:107570008092981390929913A0929A13B0929B13B1
:1075800084E493E10E941C3821972FEF821A920A1B
:10759000A20AB20A209721F744E1C40ED11CE11CD3
:1075A000F11C8AE5C81680E2D806E104F104A1F6D0
:1075B000C12CA0E2DA2EE12CF12CD5E0C2E8109229
:1075C000A1131092A013D0939413C0939713C09259
:1075D0009813D0929913E0929A13F0929B1384E43B
:1075E00093E10E941C381092A1131092A013D09323
:1075F0009413C0939713D701C6018C529F4FAF4F7E
:10760000BF4F8093981390939913A0939A13B093BC
:107610009B1384E493E10E941C38EFEFCE1ADE0A3C
:10762000EE0AFE0AFAE0CF16F0E2DF06E104F1040A
:1076300031F6FEEDCF2EF0E2DF2EE12CF12CD5E07D
:10764000C2E81092A1131092A013D0939413C09388
:107650009713C0929813D0929913E0929A13F092D4
:107660009B1384E493E10E941C382FEFC21AD20AC4
:10767000E20AF20A46EEC41640E2D406E104F1043E
:1076800001F7CC24C394E2E1DE2EE12CF12C0AE0D8
:1076900010E0D5E0C2E81093A1130093A013D0939B
:1076A0009413C0939713C0929813D0929913E092B9
:1076B0009A13F0929B1384E493E10E941C38109378
:1076C000A1130093A013D0939413C0939713D701E1
:1076D000C6018096A11DB11D8093981390939913B4
:1076E000A0939A13B0939B1384E493E10E941C38F7
:1076F0008FEFC81AD80AE80AF80AE5E0CE16E2E1E8
:10770000DE06E104F10439F600910E0D10910F0D23
:107710000115110509F0D6C080910D0D882309F4DB
:10772000E1C02AE030E240E050E06DEA73E084E43A
:1077300093E10E9421F1C1E0D0E003E010E0E0908D
:107740000E0DF0900F0D35E0332E42E8242E442428
:107750004A94542C64E0662E712C7FE1C72E74E0AD
:10776000D72E80910E0D90910F0D800F911FE8166E
:10777000F90608F0D5C0C7010E9438F2882309F441
:1077800081C08091221265E172E1882311F062E2EA
:1077900072E1FB0101900020E9F7CF010197861B00
:1077A000970BF4E1FC9F9001FD9F300D1124265FA3
:1077B0003F4D50E040E0459710F0FB01128A84E411
:1077C00093E10E9421F1CE018F5F9D4EB0E0A0E0D9
:1077D00021964E0124E0880C991C2A95E1F7FDEFD3
:1077E0008F1AFFE99F0AB12CA12C2091C41424FF09
:1077F0007EC07092A1136092A013309294132092D5
:1078000097138093981390939913A0939A13B0931E
:107810009B1384E493E10E941C38D092A113C09280
:10782000A013309294132092971380929813909201
:107830009913A0929A13B0929B1384E493E10E944F
:107840001C38B70185E09EE00E94B1C980912212E8
:1078500062E272E1811102C065E172E182E09EE0C4
:107860000E94E8DB6AE77CE08EEF9DE00E94E8DBA7
:1078700065E172E18DEF9DE00E94E8DB89EF9DE01C
:107880000E9492C72FEFE21AF20A6BCF20910E0DE1
:1078900030910F0DA901415051096091A1047091DF
:1078A000A2046817790738F42C5F3F4F30930F0D0F
:1078B00020930E0D45CE4430510508F43DCE2450A2
:1078C0003109F4CF0430110569F480910D0D88233E
:1078D00031F083E090E090930F0D80930E0DD0E097
:1078E000C0E02DCFD0E0C0E004E010E028CF10923F
:1078F000A1131092A01330929413209297138093A7
:10790000981390939913A0939A13B0939B1384E4C4
:1079100093E10E941C385092A1134092A01381CF92
:10792000DF91CF911F910F91FF90EF90DF90CF905B
:10793000BF90AF909F908F907F906F905F904F908F
:107940003F902F900895AF92BF92CF92DF92EF9227
:10795000FF920F931F93CF93DF93EC0184E6C82E21
:1079600080E2D82EE12CF12C02E8A12C90E2B92E75
:1079700015E000935114C0925214D0925314E09227
:107980005414F0925514B0925B14A0925A141093B0
:107990004E148EEF93E10E941C388FEFC81AD80A5C
:1079A000E80AF80A88E7C81680E2D806E104F1047C
:1079B00001F724E630E240E050E0BE018EEF93E1B3
:1079C000DF91CF911F910F91FF90EF90DF90CF90BB
:1079D000BF90AF900C9421F10F931F93CF93DF933F
:1079E0008C016F3F19F41092E81160E02091E811CA
:1079F000862F062E000C990B2817190609F08CF516
:107A00006093E81160E087E09EE00E94A1C8C80191
:107A10000E9492C78AE00E946AC7C8010F94C131D0
:107A2000800F911FEC01C01BD10BC034D1053CF07D
:107A30000197FC012491207C2038D1F3F3CFDD277E
:107A4000AE01B80188EA91E10F94E231C855DE4EEB
:107A5000188288EA91E1DF91CF911F910F910C94E8
:107A6000A33CDF91CF911F910F910895DF92EF9288
:107A7000FF920F931F93CF93DF93CDB7DEB7CA5A10
:107A8000D1090FB6F894DEBF0FBECDBFCF55DF4F83
:107A9000188219821A821B82C15AD0408091BA037F
:107AA0009091BB03A091BC03B091BD03CB55DF4FB8
:107AB00088839983AA83BB83C55AD04084E690E02B
:107AC0009093DB048093DA0410920B0510920A0560
:107AD00010920C052AE035E044E050E0BE016B5501
:107AE0007F4F8AED94E00E9460DE8091DA049091ED
:107AF000DB0402969093DB048093DA0410920B056A
:107B000010920A0581E0C655DF4F8883CA5AD040DB
:107B1000CE0186559F4F0E9423A52AE035E048E418
:107B200050E061EC7CE08AED94E00E9460DE2AE0A7
:107B300035E040E150E068E279E08AED94E00E94AF
:107B400060DE8AE097EDA3EABCE3CF55DF4F888380
:107B50009983AA83BB83C15AD040CE018F559F4FD2
:107B60000E941AA58DE398E00E9435A58FE092E06F
:107B70000E942CA58BE092E00E941AA58091030937
:107B800090910409A0910509B091060989839A830F
:107B9000AB83BC838E010F5F1F4FC8010E941AA5E3
:107BA000CF55DF4F188219821A821B82C15AD040EA
:107BB0007E018DE6E80EF11C83E0D7018C9389836A
:107BC000CE018F559F4F0E941AA5C7010E9423A581
:107BD000C8010E9423A54AE0D42EDA94DD2031F0BA
:107BE000CE018F559F4F0E941AA5F7CF8BEF92E1E0
:107BF0000E9435A5CF55DF4F188219821A821B8249
:107C0000C15AD0403AE0D32EDA94DD2031F0CE01D3
:107C10008F559F4F0E941AA5F7CF85E0D82ED982A5
:107C2000F701D082C8010E9423A5C7010E9423A5A5
:107C30002AE035E048E050E06DEF74E08AED94E032
:107C40000E9460DE2AE035E048E050E065EF74E035
:107C50008AED94E00E9460DE2AE035E044E650E0E0
:107C600067EC77E08AED94E00E9460DE19828FEF86
:107C7000D7018C93C8010E942CA5C7010E9423A59F
:107C80002AE035E044E050E062EF72E08AED94E0F3
:107C90000E9460DE8091D1058983C8010E942CA5D5
:107CA0002AE035E040E150E065EE74E08AED94E0D2
:107CB0000E9460DE198A1A8A1B8A1C8A80E090E082
:107CC000A0E8BFE38D879E87AF87B88B8091731242
:107CD00090917412A0917512B091761289839A8353
:107CE000AB83BC832CEA35EC47E25EE3609177120C
:107CF000709178128091791290917A120F943E3A95
:107D00006D837E838F8398872CEA35EC47E25EE3B0
:107D100060917B1270917C1280917D1290917E1205
:107D20000F94DA3269877A878B879C872AE035E05F
:107D300044E150E0B8018AED94E00E9460DE84E105
:107D400090E09A838983C8010E9408A58091081257
:107D500090910912A0910A12B0910B1289839A8313
:107D6000AB83BC832CEA35EC47E25EE360910C12F6
:107D700070910D1280910E1290910F120F943E3A55
:107D80006D837E838F8398872CEA35EC47E25EE330
:107D90006091101270911112809112129091131231
:107DA0000F94DA3269877A878B879C87C8010E9493
:107DB00011A58CE0EBEAF2E0D80101900D928A95D2
:107DC000E1F7C8010E9411A51982C8010E9423A5EC
:107DD0008FE790E09A838983C8010E9408A5E7EBAA
:107DE000F2E0D80101900D92DA94E1F72AE035E053
:107DF00045E050E0B8018AED94E00E9460DE809199
:107E0000E4048983C8010E942CA580E2ECEBF2E037
:107E1000D80101900D928A95E1F72AE035E040E221
:107E200050E0B8018AED94E00E9460DEF701108214
:107E3000C7010E942CA580E398E00E942CA58CE24B
:107E400098E00E941AA5CF55DF4F188219821A8236
:107E50001B82C15AD040CE018F559F4F0E941AA558
:107E600080E2D8011D928A95E9F72AE035E040E2E8
:107E700050E0B8018AED94E00E9460DEFE01F996C0
:107E800088E0DF011D928A95E9F744E650E060E062
:107E900070E049835A836B837C834D835E836F8359
:107EA000788783E090E0A0E0B0E089879A87AB878D
:107EB000BC874D875E876F87788B498B5A8B6B8B1E
:107EC0007C8B8D8B9E8BAF8BB88F898F9A8FAB8F6E
:107ED000BC8F8D8F9E8FAF8FB8A38EE190E0A0E016
:107EE000B0E089A39AA3ABA3BCA38DA39EA3AFA329
:107EF000B8A789A79AA7ABA7BCA78DA79EA7AFA72E
:107F0000B8AB89AB9AABABABBCAB8DAB9EABAFABFD
:107F1000B8AF2AE035E040E450E0B8018AED94E0E3
:107F20000E9460DE90E1D92EF8018D2D11928A9584
:107F3000E9F72AE035E040E150E0B8018AED94E04D
:107F40000E9460DED8011D92DA94E9F72AE035E05C
:107F500040E150E0B8018AED94E00E9460DE88E3E1
:107F600099E00E941AA52CE0D22EF8018D2D1192D5
:107F70008A95E9F72AE035E04CE050E0B8018AED57
:107F800094E00E9460DE8CE6D8011D928A95E9F7A4
:107F90002AE035E04CE650E0B8018AED94E00E941A
:107FA00060DE8EEC94E00E9411A52AE035E048E006
:107FB00050E06CED74E08AED94E00E9460DEF70121
:107FC0001192DA94E9F7C755DF4F1882C95AD040A9
:107FD00080E090E0A0E4B0E4C356DF4F888399834B
:107FE000AA83BB83CD59D040C7010E9435A5CE01DD
:107FF00087559F4F0E9423A5CE0183569F4F0E9415
:108000001AA580E3D7011D928A95E9F789E492E1E8
:108010000E9492C78AE00E946AC72AE035E040E3E6
:1080200050E0B7018AED94E00E9460DE80910C057B
:10803000811128C00091DA041091DB0480910A05B7
:1080400090910B05F7019183808384E690E09093F3
:10805000DB048093DA042AE035E044E050E066EF88
:1080600072E08AED94E00E9460DEC7010E9408A5DC
:1080700091E00537134009F490E080910C05892BBD
:1080800080930C0580910C05811105C060E08DE79F
:1080900092E10E94EC3C8DE592E10E9492C78AE059
:1080A0000E946AC790910C0581E08927C655DF4F71
:1080B0000FB6F894DEBF0FBECDBFDF91CF911F91F9
:1080C0000F91FF90EF90DF9008951092BA0C1092EC
:1080D0002D028091C41480648093C41461E085E112
:1080E0009EE00E94A1C84AE25EE062E37EE085E095
:1080F0000E943BF360E08CE19EE00C94EC3CCF925C
:10810000DF92EF92FF920F931F93CF93DF93CDB740
:10811000DEB77C01CDB6DEB60F94C13101962DB726
:108120003EB7281B390B0FB6F8943EBF0FBE2DBFCC
:108130000DB71EB70F5F1F4FB701C8010F94BA31BB
:10814000F80101900020E9F73197E01BF10B7597DA
:1081500020F08CED92E0F801848BC8010E94A33CD2
:108160000FB6F894DEBE0FBECDBEDF91CF911F914A
:108170000F91FF90EF90DF90CF900895CF93DF9312
:1081800000D01F92CDB7DEB78EEC9DE00E9492C763
:108190008AE00E946AC78091260D8330D9F1198246
:1081A0001A821B821C8260E0CE0101960E94E33697
:1081B00019821A821B821C8261E0CE0101960E9404
:1081C000E33681E0809385021092230D809386022E
:1081D00081E09AE590935B1480935A1483E390E0D6
:1081E00090935D1480935C1487E080934E1482E832
:1081F0008093511484E890E0A0E0B0E080935214A2
:1082000090935314A0935414B09355148EEF93E1AC
:108210000E941C380F900F900F900F90DF91CF911C
:108220000895CF92DF92EF92FF92CF93C82F809163
:10823000A7118150823008F069C00E94BE401092A0
:10824000A7110E942A746093CA047093CB04809390
:10825000CC049093CD04C0908F04D0909004E09013
:108260009104F09092040E94EA35AB01BC01409366
:108270008F045093900460939104709392048091C2
:10828000C2059091C305A091C405B091C5058C1994
:108290009D09AE09BF09840F951FA61FB71F8093C4
:1082A000C2059093C305A093C405B093C505C11141
:1082B0000AC0C1E00E941A238C2FCF91FF90EF904B
:1082C000DF90CF9008958091C0059091C1050196EF
:1082D0009093C1058093C0050E94EA35C090C60501
:1082E000D090C705E090C805F090C905C616D7061E
:1082F000E806F906F0F60E94EA356093C605709329
:10830000C7058093C8059093C905D3CFC0E0D2CFED
:108310008F929F92AF92BF92CF92DF92EF92FF9295
:108320000F931F93CF93DF930E94F8373AE0C32E49
:1083300030E2D32EE12CF12C15E002E84601570182
:10834000CAE0D0E010925B1410925A1410934E14AD
:10835000009351148092521490925314A09254148A
:10836000B09255148EEF93E10E941C3821978FEF45
:10837000881A980AA80AB80A209721F78AE0C80E36
:10838000D11CE11CF11C82EDC81680E2D806E10484
:10839000F104A1F6C12C20E2D22EE12CF12CD5E083
:1083A000C2E810925B1410925A14D0934E14C093EA
:1083B0005114C0925214D0925314E0925414F0927B
:1083C00055148EEF93E10E941C3810925B141092AA
:1083D0005A14D0934E14C0935114D701C6018C5235
:1083E0009F4FAF4FBF4F8093521490935314A0935D
:1083F0005414B09355148EEF93E10E941C388FEF04
:10840000C81AD80AE80AF80A8AE0C81680E2D8062C
:10841000E104F10431F69EEDC92E90E2D92EE12C53
:10842000F12CD5E0C2E810925B1410925A14D0934C
:108430004E14C0935114C0925214D0925314E0922F
:108440005414F09255148EEF93E10E941C388FEF74
:10845000C81AD80AE80AF80A86EEC81680E2D806D2
:10846000E104F10401F7CC24C39482E1D82EE12C7D
:10847000F12C0AE010E0D5E0C2E810935B14009301
:108480005A14D0934E14C0935114C0925214D092E7
:108490005314E0925414F09255148EEF93E10E941D
:1084A0001C3810935B1400935A14D0934E14C0934D
:1084B0005114D701C6018096A11DB11D809352149D
:1084C00090935314A0935414B09355148EEF93E1EA
:1084D0000E941C388FEFC81AD80AE80AF80A85E10A
:1084E000C81682E1D806E104F10439F682E190E091
:1084F00090935B1480935A14D0934E14C0935114EC
:1085000084E190E1A0E0B0E0809352149093531482
:10851000A0935414B09355148EEF93E1DF91CF9153
:108520001F910F91FF90EF90DF90CF90BF90AF9091
:108530009F908F900C941C384F925F926F927F9215
:108540008F929F92AF92BF92CF92DF92EF92FF9263
:108550000F931F93CF93DF9300D000D01F921F92F1
:10856000CDB7DEB780919F0481110AC480919D042C
:1085700090919E049C012F5F3F4F30939E04209367
:108580009D048E3E924008F4FBC380916E12909140
:108590006F1290935B1480935A1405E000934E146D
:1085A00012E81093511486E390E1A0E0B0E08093CC
:1085B000521490935314A0935414B09355148EEF07
:1085C00093E10E941C3880910312909104129093C1
:1085D0005B1480935A1400934E14109351148CE33F
:1085E00090E1A0E0B0E08093521490935314A093D4
:1085F0005414B09355148EEF93E10E941C3880916F
:1086000070129091711290935B1480935A1400939E
:108610004E141093511484E390E1A0E0B0E08093F5
:10862000521490935314A0935414B09355148EEF96
:1086300093E10E941C38809105129091061290934C
:108640005B1480935A1400934E14109351148AE3D0
:1086500090E1A0E0B0E08093521490935314A09363
:108660005414B09355148EEF93E10E941C3881E0AE
:1086700080939F0410929E0410929D048091260D79
:10868000882339F10E94281D811123C080919C0408
:108690008F5F80939C0480919C04853620F010921B
:1086A0009C041092260DE091260DE150E73008F071
:1086B0006AC00E2E000CFF0B8827EE59FC4B8F4F23
:1086C0000D943B396C43BB438745B345F4452C4679
:1086D000BF4310929C04DFCF0E94D537882309F452
:1086E00052C081E08093860280EC9DE00E9492C798
:1086F0008AE00E946AC780E190E090935B148093C7
:108700005A1485E080934E1412E81093511484E1BA
:1087100090E1A0E0B0E08093521490935314A093A2
:108720005414B09355148EEF93E10E941C3881E0ED
:108730009AE590935B1480935A1486E390E09093AB
:108740005D1480935C1487E080934E141093511451
:1087500084E890E0A0E0B0E080935214909353142A
:10876000A0935414B09355148EEF93E10E941C38DB
:108770001092260D08C00E94D537882321F00E9450
:10878000281D8823A9F380918602882309F433C722
:108790008091A0048111C0C284E096E090935B14A4
:1087A00080935A1480EA90E890935D1480935C144F
:1087B00017E010934E1402E80093511480EA90E001
:1087C000A0E0B0E08093521490935314A0935414FB
:1087D000B09355148EEF93E10E941C388091810272
:1087E00090918202A0918302B09184020097A1052A
:1087F000B10509F03FC210925B1410925A1415E0B3
:1088000010934E14009351148AE890E1A0E0B0E078
:108810008093521490935314A0935414B09355140E
:108820008EEF93E10E941C3889E090E090935B14F6
:1088300080935A1410934E14009351148CE890E1D5
:10884000A0E0B0E08093521490935314A09354147A
:10885000B09355148EEF93E10E941C3880918102F1
:1088600090918202A0918302B09184020097F1E07E
:10887000AF07B10508F441C2B0935B14A0935A143A
:1088800090935D1480935C1487E080934E1482E88B
:108890008093511488E890E1A0E0B0E080935214F6
:1088A00090935314A0935414B09355148EEF93E106
:1088B0000E941C388091810290918202A0918302D3
:1088C000B0918402BA2FA92F982F8827009721E012
:1088D000A207B10508F417C2B0935B14A0935A1411
:1088E00090935D1480935C1487E080934E1412E89B
:1088F0001093511481EA90E0A0E0B0E0809352140C
:1089000090935314A0935414B09355148EEF93E1A5
:108910000E941C388091BC0C882309F4FAC183E0C2
:1089200090E090935B1480935A1485E080934E14EA
:108930001093511485E490E1A0E0B0E080935214CC
:1089400090935314A0935414B09355148EEF93E165
:108950000E941C388091A004875E8093A00420911F
:10896000A004822F90E0253608F021C290935B147A
:1089700080935A1485E080934E1482E880935114BA
:1089800080E090E1A0E0B0E0809352149093531403
:10899000A0935414B09355148EEF93E10E941C38A9
:1089A0000E94281D811114C20E94C1C3811105C0FB
:1089B00090918D0491FD0E94281D90918D0480FB63
:1089C00091F990938D0491FD03C28091C41482FDAE
:1089D000FFC18091A7118150823008F4F9C16091E4
:1089E000051270910612072E000C880B990B0F943C
:1089F0007B326B017C0120E030E0A9010F947432DE
:108A0000882309F4BBC66091031270910412072EEB
:108A1000000C880B990B0F947B322B013C0120E05A
:108A200030E040E050E4C701B6010F944339A301A0
:108A300092010F94A43B18160CF4C2C660916E12FA
:108A400070916F12072E000C880B990B0F947B32DC
:108A50006D837E838F8398876091701270917112FD
:108A6000072E000C880B990B0F947B324B015C0195
:108A700020E030E040E251E40F9443392D813E8103
:108A80004F8158850F94A43B18160CF499C620E02A
:108A900030E040E050E4C701B6010F944439A3012F
:108AA00092010F94743287FD10C020E030E040E264
:108AB00051E4C501B4010F9444392D813E814F81A9
:108AC00058850F94743287FF6AC684E190E09093D2
:108AD0005B1480935A1485E080934E1482E880934F
:108AE000511484E190E1A0E0B0E08093521490939F
:108AF0005314A0935414B09355148EEF93E10E9435
:108B00001C388091240D81117CC682E07AC682EBEC
:108B10009DE00E9492C78AE00E946AC781E09AE5C0
:108B200090935B1480935A1480E490E090935D14CA
:108B300080935C1417E010934E1482E880935114D4
:108B400084E890E0A0E0B0E0809352149093531436
:108B5000A0935414B09355148EEF93E10E941C38E7
:108B60001093260D10CE8091130D882309F40BCE9F
:108B70000E94D537882309F406CE0E94281D811152
:108B800002CE84EA9DE00E9492C78AE00E946AC7F2
:108B90008091140D90E0B0E0A0E0895B9F4FAE4F54
:108BA000B54A21E03AE530935B1420935A14909330
:108BB0005D1480935C1487E080934E1482E8809368
:108BC000511484E890E0A0E0B0E0809352149093B8
:108BD0005314A0935414B09355148EEF93E10E9454
:108BE0001C381092130DC4CD0E94D537882309F488
:108BF000CACD0E94281D8111C6CD81E080938602D6
:108C00001092260D86E99DE00E9492C78AE00E949C
:108C10006AC781E09AE590935B1480935A148EE4BE
:108C200090E090935D1480935C1487E080934E14E1
:108C300082E88093511484E890E0A0E0B0E0809353
:108C4000521490935314A0935414B09355148EEF70
:108C500093E10E941C3897CD0E94281D811193CD6D
:108C600019821A821B821C8262E0CE0101960F9447
:108C700020087ECD0196A11DB11D35E0B695A795C2
:108C8000979587953A95D1F70197A109B109009772
:108C9000E1E0AE07B10548F1B0935B14A0935A141C
:108CA00090935D1480935C1410934E1412E810930B
:108CB00051148AE890E1A0E0B0E0809352149093C0
:108CC0005314A0935414B09355148EEF93E10E9463
:108CD0001C3888E090E090935B1480935A1485E0F0
:108CE00080934E1410935114A9CD90935B148093EC
:108CF0005A1485E080934E14D9CF90935B148093DF
:108D00005A1485E0C2CD90935B1480935A1485E089
:108D1000ECCD82E090E005CE8A3F08F020CE8EEFC9
:108D20008093A00485E89DE00E9492C78AE00E949B
:108D30006AC781E08093860281E09AE590935B1494
:108D400080935A148DE290E090935D1480935C14AC
:108D500087E080934E1482E88093511484E890E079
:108D6000A0E0B0E08093521490935314A093541455
:108D7000B09355148EEF93E10E941C3810929F041B
:108D800028960FB6F894DEBF0FBECDBFDF91CF910E
:108D90001F910F91FF90EF90DF90CF90BF90AF9019
:108DA0009F908F907F906F905F904F900895845622
:108DB000910990935B1480935A1485E080934E142C
:108DC00082E88093511481E090E1A0E0B0E0DCCD36
:108DD0008CE090E090935B1480935A1415E010930C
:108DE0004E1482E88093511484E190E1A0E0B0E059
:108DF0008093521490935314A0935414B093551429
:108E00008EEF93E10E941C380E94EA3520E13EE09B
:108E100040E050E00F94B8382115310581E0480753
:108E2000510508F470C050935B1440935A1430936A
:108E30005D1420935C1487E080934E1412E8109325
:108E4000511480E190E1A0E0B0E08093521490933F
:108E50005314A0935414B09355148EEF93E10E94D1
:108E60001C380E94EA3520E13EE040E050E00F94DB
:108E7000B8382CE330E040E050E00F94B83830933D
:108E80005B1420935A1405E000934E141093511470
:108E900082E190E1A0E0B0E08093521490935314EB
:108EA000A0935414B09355148EEF93E10E941C3894
:108EB0000E94981F882309F45CC48F5F80939B04F1
:108EC000E82EF12C833330F5EE0CFF1CF0925B148E
:108ED000E0925A1400934E14109351148EE090E1D6
:108EE000A0E0B0E08093521490935314A0935414D4
:108EF000B09355148EEF93E10E941C3810925B14CE
:108F000010925A142BC030935B1420935A14109370
:108F10004E1494CF84E690E090935B1480935A149F
:108F200000934E14109351148EE090E1A0E0B0E055
:108F30008093521490935314A0935414B0935514E7
:108F40008EEF93E10E941C38A2E3EA1AA0E8FA0A25
:108F5000EE0CFF1CF0925B14E0925A1400934E1436
:108F6000109351148FE090E1A0E0B0E08093521490
:108F700090935314A0935414B09355148EEF93E12F
:108F80000E941C380E94981F90E090935B1480937D
:108F90005A1485E080934E1482E88093511486E140
:108FA00090E1A0E0B0E08093521490935314A0930A
:108FB0005414B09355148EEF93E10E941C3820E0B6
:108FC00030E0A9016091031370910413809105139F
:108FD000909106130F94443920E030E048EC52E4BD
:108FE0000F94DA320F94B03A70935B1460935A1472
:108FF00005E000934E1412E81093511486E290E1BC
:10900000A0E0B0E08093521490935314A0935414B2
:10901000B09355148EEF93E10E941C3880917D022D
:1090200090917E0290935B1480935A1400934E1497
:109030001093511480E093E1A0E0B0E080935214CB
:1090400090935314A0935414B09355148EEF93E15E
:109050000E941C3820E030E040E251E46091D50CE1
:109060007091D60C8091D70C9091D80C0F94DA3275
:109070000F94B73A70935B1460935A1400934E1494
:109080001093511482E492E1A0E0B0E08093521476
:1090900090935314A0935414B09355148EEF93E10E
:1090A0000E941C3820E030E040E251E46091D90C8D
:1090B0007091DA0C8091DB0C9091DC0C0F94DA3219
:1090C0000F94B73A70935B1460935A1400934E1444
:1090D0001093511486E492E1A0E0B0E08093521422
:1090E00090935314A0935414B09355148EEF93E1BE
:1090F0000E941C3820E030E040E251E46091DD0C39
:109100007091DE0C8091DF0C9091E00C0F94DA32BC
:109110000F94B73A70935B1460935A1400934E14F3
:10912000109351148AE492E1A0E0B0E080935214CD
:1091300090935314A0935414B09355148EEF93E16D
:109140000E941C3820E030E040E251E46091E10CE4
:109150007091E20C8091E30C9091E40C0F94DA3260
:109160000F94B73A70935B1460935A1400934E14A3
:10917000109351148EE492E1A0E0B0E08093521479
:1091800090935314A0935414B09355148EEF93E11D
:109190000E941C3820E030E048EC52E46091FB1261
:1091A0007091FC128091FD129091FE120F94DA32B0
:1091B0000F94B03A70935B1460935A1400934E145A
:1091C0001093511486E392E1A0E0B0E08093521432
:1091D00090935314A0935414B09355148EEF93E1CD
:1091E0000E941C3820E030E048EC52E46091FF120D
:1091F0007091001380910113909102130F94DA3251
:109200000F94B03A70935B1460935A1400934E1409
:10921000109351148AE392E1A0E0B0E080935214DD
:1092200090935314A0935414B09355148EEF93E17C
:109230000E941C3880918D0290918E0290935B1455
:1092400080935A1400934E141093511482E592E1C6
:10925000A0E0B0E08093521490935314A093541460
:10926000B09355148EEF93E10E941C3880918B02CD
:1092700090918C0290935B1480935A1400934E1437
:109280001093511484E592E1A0E0B0E08093521471
:1092900090935314A0935414B09355148EEF93E10C
:1092A0000E941C3820E030E040E251E460917312EB
:1092B0007091741280917512909176120F94DA3237
:1092C0000F94B73A70935B1460935A1400934E1442
:1092D0001093511486E592E1A0E0B0E0809352141F
:1092E00090935314A0935414B09355148EEF93E1BC
:1092F0000E941C382CEA35EC47E25EE3609177125D
:10930000709178128091791290917A120F943E3A6E
:1093100020E030E040E251E40F94DA320F94B73AA3
:1093200070935B1460935A1400934E14109351146D
:109330008AE592E1A0E0B0E0809352149093531438
:10934000A0935414B09355148EEF93E10E941C38EF
:109350002CEA35EC47E25EE360917B1270917C125F
:1093600080917D1290917E120F94DA3220E030E0ED
:1093700040E251E40F94DA320F94B73A70935B14E1
:1093800060935A1400934E14109351148EE592E199
:10939000A0E0B0E08093521490935314A09354141F
:1093A000B09355148EEF93E10E941C3820E030E01A
:1093B00040E251E4609108127091091280910A1202
:1093C00090910B120F94DA320F94B73A70935B14AA
:1093D00060935A1400934E141093511482E692E154
:1093E000A0E0B0E08093521490935314A0935414CF
:1093F000B09355148EEF93E10E941C382CEA35ECA3
:1094000047E25EE360910C1270910D1280910E1292
:1094100090910F120F943E3A20E030E040E251E488
:109420000F94DA320F94B73A70935B1460935A1426
:1094300000934E141093511486E692E1A0E0B0E040
:109440008093521490935314A0935414B0935514D2
:109450008EEF93E10E941C382CEA35EC47E25EE384
:10946000609110127091111280911212909113124A
:109470000F94DA3220E030E040E251E40F94DA3227
:109480000F94B73A70935B1460935A1400934E1480
:10949000109351148AE692E1A0E0B0E08093521458
:1094A00090935314A0935414B09355148EEF93E1FA
:1094B0000E941C3880911D0D811105C080911F0DE7
:1094C000882309F46DC060916E1270916F12072E9F
:1094D000000C880B990B0F947B3220E030E048ECB5
:1094E00052E40F94DA326B017C016091701270913A
:1094F0007112072E000C880B990B0F947B329B0185
:10950000AC01C701B6010F943E3A0F94B73A6536E5
:10951000710510F064E670E070935B1460935A1468
:1095200005E000934E1412E81093511484E290E188
:10953000A0E0B0E08093521490935314A09354147D
:10954000B09355148EEF93E10E941C3860916E1217
:1095500070916F12072E000C880B990B0F947B32C1
:109560006B017C0120E030E04AE253E40F94A43B1D
:10957000181624F480911D0D811146C1609170125E
:1095800070917112072E000C880B990B0F947B328F
:109590009B01AC01C701B6010F94A43B87FFAFC18B
:1095A0008091130D882339F18091120D91E0980F6D
:1095B0009093120D90E090935B1480935A1485E081
:1095C00080934E1482E88093511482E490E1A0E0ED
:1095D000B0E08093521490935314A0935414B0931A
:1095E00055148EEF93E10E941C388091120D8A3041
:1095F00010F01092120D0E946037882309F4B5C153
:1096000060910B0D70910C0DEE24E394F12C61151B
:109610007105A9F090E080E00F94793220E030E00D
:1096200040E85EE30F94DA320F94223A20E030E013
:1096300040E85FE30F9444390F94B73A7B0101E0AF
:1096400010E080910D0D811102C010E000E08091CA
:109650004213909143138F3F980711F40E94CD80DD
:109660009093431380934213080F191FB80190E0A1
:1096700080E00F94793220E030E040E85EE30F9420
:10968000DA320F94223A4B015C01F0925B14E092C3
:109690005A1405E000934E1412E81093511480E11F
:1096A00093E1A0E0B0E08093521490935314A09300
:1096B0005414B09355148EEF93E10E941C38C501E9
:1096C000B4010F94B73A70935B1460935A140093EB
:1096D0004E141093511482E193E1A0E0B0E0809326
:1096E000521490935314A0935414B09355148EEFC6
:1096F00093E10E941C380EE914E1AAE1FA2E809150
:109700004B0490914C042091990430919A04891B48
:109710008F7309F449C12A3131050CF0DBC19091F6
:109720004B0480914C044FEF5FEF981749F0E82FFE
:10973000F0E0E55BFB4F42818F5F8F7380934C04B9
:10974000F901E256FB4E408380919E148A3509F060
:10975000B3C162E070E080E090E00E94DD3780916C
:10976000990490919A04019690939A048093990495
:10977000C6CF10925B1410925A14ACCB6091701249
:1097800070917112072E000C880B990B0F947B328D
:1097900020E030E0A9010F947432811134C98CE0CB
:1097A00090E090935B1480935A1485E080934E145C
:1097B00082E88093511484E190E1A0E0B0E0F3CB23
:1097C0008DE090E090935B1480935A1485E0809331
:1097D0004E1482E88093511484E190E1A0E0B0E05F
:1097E0008093521490935314A0935414B09355142F
:1097F0008EEF93E10E941C388091240D811101C0ED
:1098000081E08093240DDBCB10921D0D20E030E031
:1098100040E251E46091150D7091160D8091170D85
:109820009091180D0F94DA320F94B03A70935B1444
:1098300060935A1400934E141093511484E590E1F0
:10984000A0E0B0E08093521490935314A09354146A
:10985000B09355148EEF93E10E941C3820E030E065
:1098600040E251E46091190D70911A0D80911B0D29
:1098700090911C0D0F94DA320F94B03A70935B14F0
:1098800060935A1400934E141093511488E590E19C
:10989000A0E0B0E08093521490935314A09354141A
:1098A000B09355148EEF93E10E941C3884E69DE03E
:1098B0000E9492C78AE00E946AC781E09AE590936D
:1098C0005B1480935A1481E490E090935D1480932C
:1098D0005C1487E080934E141093511484E890E058
:1098E000A0E0B0E08093521490935314A0935414CA
:1098F000B09355148EEF93E10E941C3851CE6091C5
:109900001F0D662309F44CCE062E000C770B8BE45A
:109910009DE00E9459CA8AE00E946AC710921F0DFA
:1099200084E090E090935B1480935A1485E08093D8
:109930004E1412E8109351148EE890E1A0E0B0E0CC
:109940008093521490935314A0935414B0935514CD
:109950008EEF93E10E941C3881E09AE590935B14AE
:1099600080935A1483E590E0B0CF10925B1410926C
:109970005A1405E000934E1412E81093511480E13C
:1099800093E1A0E0B0E08093521490935314A0931D
:109990005414B09355148EEF93E10E941C3810922A
:1099A0005B1410925A1493CE121613060CF492C044
:1099B0008091021490910314A0910414B0910514A5
:1099C0008C34E0E19E07A105B10509F4D7C98A34BA
:1099D0009041A105B10509F4D1C920E030E040E291
:1099E00051E46091690270916A0280916B029091DA
:1099F0006C020F94DA320F94B03A70935B14609358
:109A00005A1405E000934E1412E81093511488E4A0
:109A100090E1A0E0B0E08093521490935314A0938F
:109A20005414B09355148EEF93E10E941C3820E03B
:109A300030E040E251E460916D0270916E028091DD
:109A40006F02909170020F94DA320F94B03A7093D3
:109A50005B1460935A1400934E14109351148AE4CB
:109A600090E1A0E0B0E08093521490935314A0933F
:109A70005414B09355148EEF93E10E941C3820E0EB
:109A800030E040E251E46091710270917202809185
:109A90007302909174020F94DA320F94B03A70937B
:109AA0005B1460935A1400934E14109351148CE479
:109AB00090E1A0E0B0E056C9121613060CF01FCEDC
:109AC000F8012F2D11922A95E9F710929A0410921D
:109AD000990415CE9091FF1380919E14981321C084
:109AE0009091001480919F1498131BC0233031056E
:109AF000C4F09091A0149093FE138091A1148093D0
:109B000001149330D1F4982F9D7F9038B1F4909147
:109B1000A2149F3409F059C09091A3149B3409F00A
:109B200054C0EEE9F4E18AE1DF011D928A95E9F77C
:109B300010929A04109299043BCF833809F045C0E3
:109B40008091A2149091A314982789279827B0E0B8
:109B5000A0E08093021490930314A0930414B09394
:109B60000514C090A414D12CF12CE12CC092061441
:109B7000D0920714E0920814F092091425EA34E117
:109B800040E050E0BA014C155D056E057F0508F018
:109B90004AC0DB01CA01B695A795979587950696A9
:109BA000880F991FFC01E250FC4ED9018C9111964F
:109BB0009C91892798278927918380834E5F5F4FE7
:109BC0006F4F7F4F2E5F3F4FDECF813861F5809121
:109BD000A21490E0B0E0A0E08093021490930314EC
:109BE000A0930414B09305148091A314482F50E05F
:109BF00070E060E0409306145093071460930814DB
:109C000070930914A4EAB4E1EAE0F4E190E030E0F2
:109C100020E08217930739F04D9150E04193519322
:109C20002F5F3F4FF6CFEEE9F4E18AE1DF011D92AD
:109C30008A95E9F710929A04109299040F94C20839
:109C4000B7CE6F927F928F929F92AF92BF92CF9238
:109C5000DF92EF92FF920F931F93CF93DF93CDB7D5
:109C6000DEB764970FB6F894DEBF0FBECDBF10927B
:109C7000D0008091D00082608093D0001092D500F7
:109C800080E18093D4008091D10080618093D100E5
:109C90008091D10088608093D1008091D10080684C
:109CA0008093D1008091D1008F7D8093D1008AE58F
:109CB00080934F148093FF1385EA80935014809310
:109CC0000014EEE9F4E18AE1DF011D928A95E9F7DB
:109CD0008091220D882309F474C283E090E0909370
:109CE0005B1480935A1485E080934E1482E880932D
:109CF00051148FE190E1A0E0B0E080935214909372
:109D00005314A0935414B09355148EEF93E10E9412
:109D10001C3884E690E090935B1480935A1405E01D
:109D200000934E1412E81093511486E090E1A0E0E5
:109D3000B0E08093521490935314A0935414B093B2
:109D400055148EEF93E10E941C388BE090E09093C5
:109D50005B1480935A1400934E141093511480E0B6
:109D600092E1A0E0B0E08093521490935314A0933A
:109D70005414B09355148EEF93E10E941C38109246
:109D80005B1410925A1400934E141093511484E3F0
:109D900090E1A0E0B0E08093521490935314A0930C
:109DA0005414B09355148EEF93E10E941C38109216
:109DB0005B1410925A1400934E14109351148AE3BA
:109DC00090E1A0E0B0E08093521490935314A093DC
:109DD0005414B09355148EEF93E10E941C38809177
:109DE0006E1290916F1290935B1480935A140093AB
:109DF0004E141093511486E390E1A0E0B0E08093FC
:109E0000521490935314A0935414B09355148EEF9E
:109E100093E10E941C388091031290910412909358
:109E20005B1480935A1400934E14109351148CE3D6
:109E300090E1A0E0B0E08093521490935314A0936B
:109E40005414B09355148EEF93E10E941C3882E0B5
:109E500090E090935B1480935A1400934E141093E7
:109E600051148EE190E1A0E0B0E080935214909301
:109E70005314A0935414B09355148EEF93E10E94A1
:109E80001C3881E08093850270E6C72E70E1D72EE2
:109E9000E12CF12C10925B1410925A1400934E1482
:109EA00010935114C0925214D0925314E09254144F
:109EB000F09255148EEF93E10E941C38BFEFCB1A3D
:109EC000DB0AEB0AFB0AE4E7CE16E0E1DE06E1047A
:109ED000F10401F7CE0101967C0184E1D7011D92C6
:109EE0008A95E9F781E08F9390E99F938F9390E6AD
:109EF0009F938F9388E68F938EEB93E09F938F933E
:109F0000FF92EF920F94CC3C20E630E140E050E02D
:109F10006BEC73E08EEF93E10E9421F12AE630E1D1
:109F200040E050E068ED73E08EEF93E10E9421F194
:109F300024E730E140E050E0B7018EEF93E10E946A
:109F400021F12EE730E140E050E064EE73E08EEF67
:109F500093E10E9421F110925B1410925A14009325
:109F60004E14109351148EE090E1A0E0B0E0809385
:109F7000521490935314A0935414B09355148EEF2D
:109F800093E10E941C3810925B1410925A140093B3
:109F90004E14109351148FE090E1A0E0B0E0809354
:109FA000521490935314A0935414B09355148EEFFD
:109FB00093E10E941C380FB6F894DEBF0FBECDBFF0
:109FC0004AE0C42E40E2D42EE12CF12C55E0752E4F
:109FD00062E8662E460157010AE010E010925B1419
:109FE00010925A1470924E1460925114809252142E
:109FF00090925314A0925414B09255148EEF93E1A2
:10A000000E941C3801501109FFEF8F1A9F0AAF0AF6
:10A01000BF0A0115110511F78AE0C80ED11CE11C19
:10A02000F11C92EDC91690E2D906E104F10491F613
:10A03000C12C30E2D32EE12CF12C05E012E8109275
:10A040005B1410925A1400934E1410935114C09242
:10A050005214D0925314E0925414F09255148EEF8F
:10A0600093E10E941C3810925B1410925A140093D2
:10A070004E1410935114D701C6018C529F4FAF4F0D
:10A08000BF4F8093521490935314A0935414B093E1
:10A0900055148EEF93E10E941C38AFEFCA1ADA0A0A
:10A0A000EA0AFA0ABAE0CB16B0E2DB06E104F104F0
:10A0B00031F62EEDC22E20E2D22EE12CF12C05E05D
:10A0C00012E810925B1410925A1400934E141093DD
:10A0D0005114C0925214D0925314E0925414F0923E
:10A0E00055148EEF93E10E941C38EFEFCE1ADE0A72
:10A0F000EE0AFE0AF6EECF16F0E2DF06E104F10406
:10A1000001F7CC24C39482E1D82EE12CF12C9AE003
:10A11000A92EB12C05E012E8B0925B14A0925A145B
:10A1200000934E1410935114C0925214D0925314B1
:10A13000E0925414F09255148EEF93E10E941C3873
:10A14000B0925B14A0925A1400934E1410935114C1
:10A15000D701C6018096A11DB11D80935214909322
:10A160005314A0935414B09355148EEF93E10E94AE
:10A170001C388FEFC81AD80AE80AF80A95E1C91600
:10A1800092E1D906E104F10439F684E39DE00E94EE
:10A1900092C78AE00E946AC764960FB6F894DEBF41
:10A1A0000FBECDBFDF91CF911F910F91FF90EF9028
:10A1B000DF90CF90BF90AF909F908F907F906F90E7
:10A1C000089582E090E08BCD0E94214E1092A00471
:10A1D00081E08093860286EE9DE00E9492C78AE02D
:10A1E0000C946AC7AB01BC014093C0145093C114D6
:10A1F0006093C2147093C31488E296E10C94767C49
:10A20000CF93DF93DB01F9019C919130C1F0943041
:10A2100080F094509C938830D1F480819181009794
:10A2200071F0019791838083480F591FEA011882CA
:10A2300006C08C3539F49C5F9C93943041F4DF91D7
:10A24000CF9108958B3339F781E08C93F8CF20813B
:10A250003181B9016F5F7F4F71836083420F531F5C
:10A26000EA018883808191818F3591056CF7E7CF72
:10A270000F931F9381E00091C0141091C11420919D
:10A28000C2143091C3144091BC145091BD1460911C
:10A29000BE147091BF14041715072607370708F47A
:10A2A00080E01F910F9108954F925F926F927F927D
:10A2B0008F929F92AF92BF92CF92DF92EF92FF92D6
:10A2C0000F931F93CF9310929804109297042FE34B
:10A2D0002093960410929504109294041092930483
:10A2E00010924604109247041092480410924904B8
:10A2F0009C01F90190812F5F3F4F9032D1F39E3442
:10A30000C9F4818190ED980F9A3020F08D3211F0D0
:10A310008B3281F432969F012F5F3F4F80818053B3
:10A320008A3008F47EC09F012F5F3F4F80818032CA
:10A3300009F479C0F093BE07E093BD078F010F5F6A
:10A340001F4FC0816AE270E0C8010F94923C0097F1
:10A3500031F0FC01319780818032E1F31182CD34FC
:10A3600029F0C43519F0C73409F04BC0F8018081D9
:10A370000F5F1F4F8032D1F380538A3008F041C005
:10A38000C093960490E080E04AE0DF011196489F78
:10A390009001499F300D1124C901C0972081820F7F
:10A3A000911D27FD9A95218130ED320F3A30E8F169
:10A3B00090939504809394042E3261F4329630E0A9
:10A3C0004AE0DF0131962C9150ED520F5A3078F16E
:10A3D000309393049D01D9012F5F3F4F4C91403240
:10A3E000D1F3CD34A1F58E31910539F030F58731B7
:10A3F000910519F08C31910551F5B0939804A09313
:10A400009704CF911F910F91FF90EF90DF90CF9025
:10A41000BF90AF909F908F907F906F905F904F9084
:10A420000895F90178CFF9017ECFFD01AECF349FB9
:10A43000200D112430ED320FC4CF8537910538F04F
:10A4400087379105D0F2803A23E09207B1F250911C
:10A45000BD0770E060E0C12CD12C7601C394FD01F2
:10A4600031964C91442309F492C04132A1F4CD3489
:10A4700091F48032910579F4F0939804E093970475
:10A4800063E270E0CF010F94923C009709F4B9CFDA
:10A49000FC011082B6CF41544A3108F073C0DF018D
:10A4A0002D91203209F459C030ED320F3A3008F4C2
:10A4B00065C02E3209F053C0218120532A3008F4A0
:10A4C0005DC030E020E06115710519F4BF016150F5
:10A4D0007109A42FB0E02601370104C0440C551CBB
:10A4E000661C771C4A95D2F78090460490904704EA
:10A4F000A0904804B090490484289528A628B7283D
:10A500008092460490924704A0924804B092490475
:10A5100021153105A9F1251BA45DBB4F2C9320818A
:10A520002154DF012A3108F49ACFDF01219122233F
:10A5300009F495CF30ED320F3A30B8F333ED320FE6
:10A54000323098F32B3289F39D012F5F3F4F4C91AE
:10A55000403209F084CFD901F7CFFD01A0CF2D32D1
:10A5600019F02B3209F0ADCF218130ED320F3A30A6
:10A5700028F02E3209F0A5CF22819FCF9F01A9CFCD
:10A5800020E0CACF6115710551F6BD01C8CF7093A7
:10A5900098046093970435CFCF93DF93EC018991B2
:10A5A000882319F00E946AC7FACF8DE00E946AC71B
:10A5B0008AE0DF91CF910C946AC7EF92FF920F93DC
:10A5C0001F93CF93DF93CDB7DEB762970FB6F894A2
:10A5D000DEBF0FBECDBF0E947F2A882309F43FC093
:10A5E00042E054E082FF02C047EF53E022E034E053
:10A5F00081FF02C029EF33E080FD2EC082E094E0AD
:10A600005F934F933F932F939F938F938FEF9EE092
:10A610009F938F938E010F5F1F4F1F930F930F9484
:10A620000B320E94F6DBC8010E94CC52C8010E9486
:10A63000F5F40FB6F894DEBF0FBECDBF81E0629691
:10A640000FB6F894DEBF0FBECDBFDF91CF911F9143
:10A650000F91FF90EF9008958BEF93E0D1CF80E0C2
:10A66000EECFAF92BF92CF92DF92EF92FF920F9315
:10A670001F93CF93DF93CDB7DEB7E6970FB6F8946D
:10A68000DEBF0FBECDBF0091970410919804F80172
:10A6900001900020E9F731976F01C01AD10AF80143
:10A6A000CF01801B910B8C159D053CF481918F325D
:10A6B000B9F7DF0111971C92F3CF8BE1E4EEF4E1DF
:10A6C000DE015C9601900D928A95E1F7F12CE12C68
:10A6D000EC14FD040CF05DC0F801EE0DFF1D80814F
:10A6E000811103C08FEFE81AF80A5801AE0CBF1CA5
:10A6F000F5018081882309F44CC0FFEFEF1AFF0AAF
:10A70000F801EE0DFF1D7F01E01AF10A8191811120
:10A71000FACFCE014C960E94C8808BE1FE017C9658
:10A72000DE01119601900D928A95E1F7B501CE01F7
:10A7300001960E94D678CE0101960E94B2BF8FE2A8
:10A740000E946AC78091221281113BC08DEF93E075
:10A750000E94357C8091C41484FF1BC019821C8226
:10A7600021E0A501BE01645E7F4FCE0101960E94EB
:10A770000A83811129C08AE00E946AC70E94F6DB21
:10A78000B50184EE9CE00E94E8DBCE0101960E94B8
:10A79000B2BF8AE00E946AC7CE014C960E94B2BF47
:10A7A000E6960FB6F894DEBF0FBECDBFDF91CF9116
:10A7B0001F910F91FF90EF90DF90CF90BF90AF90DF
:10A7C000089582E292E1C4CFCE014C960E94378078
:10A7D0008BE1FE013196DE015C9601900D928A9527
:10A7E000E1F7CE0101960E94B2BF72CF3F924F9225
:10A7F0005F926F927F928F929F92AF92BF92CF9211
:10A80000DF92EF92FF920F931F93CF93DF9380918C
:10A81000480487FD38C0809149048370A1F5C09138
:10A820000713D0910813488159816A817B8185ED96
:10A830009CE00E94C3C94C815D816E817F818AE664
:10A8400091E30E94C3C94091031350910413609196
:10A8500005137091061387E691E30E94C3C98AE04D
:10A86000DF91CF911F910F91FF90EF90DF90CF90EC
:10A87000BF90AF909F908F907F906F905F904F9020
:10A880003F900C946AC76090FB127090FC1280900D
:10A89000FD129090FE12A090FF12B0900013009154
:10A8A000011310910213C0900313D0900413E09091
:10A8B0000513F090061388E50E945FBEC82F882319
:10A8C00009F49AC00E94E7BD362E472E582ED92F84
:10A8D00020E030E040EB53EC0F94A43B87FD0DC02B
:10A8E00020E030E040EB53E4632D742D852D9D2F47
:10A8F0000F94743218160CF081C060E671E082EC9F
:10A900009CE00E9459CA60E671E08DEB9CE00E94D9
:10A9100059CA8AEB9CE00E9492C7C0E089E50E9478
:10A920005FBE882361F10E94E7BD362E472E582E68
:10A93000D92F20E030E044EB53EC0F94A43B87FD8B
:10A940000DC020E030E044EB53E4632D742D852DE1
:10A950009D2F0F94743218160CF055C068E671E004
:10A9600087EA9CE00E9459CA68E671E082EA9CE0AE
:10A970000E9459CA8FE99CE00E9492C7C0E08AE514
:10A980000E945FBE882309F443C00E94E7BD6B01AB
:10A990007C0120E030E040E151EC0F94A43B87FDC6
:10A9A0000AC020E030E040E151E4C701B6010F9455
:10A9B000743218166CF567EF7FEF8DE89CE00E940B
:10A9C00059CA69E070E088E89CE00E9459CA85E8AD
:10A9D0009CE0DF91CF911F910F91FF90EF90DF905E
:10A9E000CF90BF90AF909F908F907F906F905F902F
:10A9F0004F903F900C9492C7C1E090CF632C742C81
:10AA0000852C9D2E8BCFA32CB42C052D1D2FB7CFBD
:10AA1000CC23E1F0C301D4018093FB129093FC128C
:10AA2000A093FD12B093FE12C501D8018093FF12CE
:10AA300090930013A0930113B0930213C0920313D9
:10AA4000D0920413E0920513F0920613DF91CF9198
:10AA50001F910F91FF90EF90DF90CF90BF90AF903C
:10AA60009F908F907F906F905F904F903F90089550
:10AA7000CF92DF92EF92FF928AE50E945FBE882319
:10AA800009F45AC00E94E7BD20E030E040E050ECFD
:10AA90000F947432C12CD12CE12C90ECF92E87FD4F
:10AAA0000FC00E94E7BD20E030E040E050E40F948A
:10AAB000A43B18160CF462C00E94E7BD6B017C0138
:10AAC0002091DD0C3091DE0C4091DF0C5091E00CB8
:10AAD000C701B6010F94DA320F94B03ACB010E944D
:10AAE0007EF480E50E9411BE81114EC0A70196013F
:10AAF00060910313709104138091051390910613D4
:10AB00000F944439609303137093041380930513D7
:10AB1000909306130E94F6DB4091031350910413A7
:10AB2000609105137091061386E79CE00E94C3C9EB
:10AB30008AE00E946AC705C083E50E945FBE81115A
:10AB4000A1CF8091480487FD24C08091490483707F
:10AB500001F50E94F6DB40910313509104136091BC
:10AB600005137091061387E69CE00E94C3C98AE032
:10AB7000FF90EF90DF90CF900C946AC7C12CD12C3E
:10AB8000E12C80E4F82E9CCF0E94D3BD8111AECF82
:10AB9000D8CF82E50E9411BE8111DBCFFF90EF90EC
:10ABA000DF90CF9008954F925F926F927F928F9235
:10ABB0009F92AF92BF92CF92DF92EF92FF92CF938C
:10ABC000DF93CDB7DEB72C970FB6F894DEBF0FBE7C
:10ABD000CDBF409007095090080960900909709016
:10ABE0000A0920914F023091500240915102509138
:10ABF0005202C301B2010F94443969837A838B8373
:10AC00009C8380900B0990900C09A0900D09B09046
:10AC10000E092091530230915402409155025091F7
:10AC20005602C501B4010F9444396D837E838F832E
:10AC30009887C0900F09D0901009E0901109F0900A
:10AC400012092091570230915802409159025091B7
:10AC50005A02C701B6010F94443969877A878B87F6
:10AC60009C8720915B0230915C0240915D02509183
:10AC70005E02C301B2010F9444392B013C012091C3
:10AC80005F02309160024091610250916202C50101
:10AC9000B4010F9444394B015C012091630230915F
:10ACA00064024091650250916602C701B6010F949B
:10ACB00044396B017C010E94F6DB88E894E00E9435
:10ACC00092C783E50E9411BE882321F00E94D3BD64
:10ACD00080934D0280914D02811151C08FE694E026
:10ACE0000E9492C780E894E00E9492C749815A81ED
:10ACF0006B817C8186EE93E10E94C3C94D815E81A8
:10AD00006F8178858AE691E30E94C3C949855A8597
:10AD10006B857C8587E691E30E94C3C98EE794E04A
:10AD20000E9492C786E794E00E9492C7B301A201F5
:10AD300086EE93E10E94C3C9B501A4018AE691E3BE
:10AD40000E94C3C9B701A60187E691E30E94C3C967
:10AD50008AE02C960FB6F894DEBF0FBECDBFDF9110
:10AD6000CF91FF90EF90DF90CF90BF90AF909F90EA
:10AD70008F907F906F905F904F900C946AC783E79D
:10AD800094E0AECF2F923F924F925F926F927F925C
:10AD90008F929F92AF92BF92CF92DF92EF92FF92EB
:10ADA0000F931F93CF93DF93CDB7DEB7E5970FB621
:10ADB000F894DEBF0FBECDBF8DAB20912B042CAB22
:10ADC00081E080932B04809196048D3409F40EC6A3
:10ADD000843511F40C942E6C873409F091C1809164
:10ADE0009404909195048B31910509F430C208F0D8
:10ADF00079C18430910508F030C12091130682306A
:10AE0000910508F4E1C1213009F0E4C111E0029795
:10AE100009F010E00E94D51F19821A821B821C8241
:10AE20001D821E821F82188682E50E945FBE8823D3
:10AE300009F4E3C10E94E7BD6B017C0120E030E032
:10AE4000A9010F947432882309F4EAC04090690282
:10AE500050906A0260906B0270906C0280916D025B
:10AE600090916E02A0916F02B09170028CA79DA785
:10AE7000AEA7BFA78090AB079090AC07A090AD079E
:10AE8000B090AE078091AF079091B007A091B10745
:10AE9000B091B20788AB99ABAAABBBABA50194014B
:10AEA000C301B2010F94743281110DC028A939A9D0
:10AEB0004AA95BA96CA57DA58EA59FA50F947432A8
:10AEC000882309F4ADC0A3019201C501B4010F9418
:10AED000433920E030E040E05FE30F94DA3268A7C6
:10AEE00079A78AA79BA72CA53DA54EA55FA568A914
:10AEF00079A98AA99BA90F94433920E030E040E06A
:10AF00005FE30F94DA322B013C0120E030E0A9012D
:10AF1000C701B6010F947432881F8827881F18173D
:10AF200009F462C180E090E0A0E8BFEB8CA79DA788
:10AF3000AEA7BFA728A539A54AA55BA5CA01B90137
:10AF40000F94DA324B015C01A3019201C301B201FB
:10AF50000F94DA329B01AC01C501B4010F9444395E
:10AF60000F94F23B4B015C01AC019B01C701B601A0
:10AF70000F94433968AB79AB8AAB9BABA5019401C5
:10AF8000C701B6010F9444399B01AC0168A979A9A6
:10AF90008AA99BA90F94DA326B017C0120E030E092
:10AFA000A9010F94A43B87FD24C1C701B6010F94EA
:10AFB000F23B6B017C01C301B2019058A5019401E1
:10AFC0000F943E3A2CA53DA54EA55FA50F94DA320D
:10AFD000A70196010F94DA3228A539A54AA55BA5E9
:10AFE0000F94443969837A838B839C83A5019401F0
:10AFF00068A579A58AA59BA50F943E3A2CA53DA5E9
:10B000004EA55FA50F94DA32A70196010F94DA32AC
:10B01000A30192010F9444396D837E838F839887B7
:10B0200020E030E0A90169817A818B819C810F94B5
:10B0300074328111F6C020E030E0A9016D817E817B
:10B040008F8198850F9474328111EBC00E94F2DBDE
:10B0500080E695E00E9492C7BDC08531910509F454
:10B06000B9C08A31910509F4EFC0049709F048C0CE
:10B0700080E50E945FBEC12CD12C7601882321F08F
:10B080000E9464B86B017C0183E50E945FBE882347
:10B0900061F00E94E7BD20E030E04AE754E40F94FD
:10B0A000DA320F94B73A6B017C010E94D42380916D
:10B0B000A811811105C060E086E795E00E94EC3C94
:10B0C0000E942A74C60ED71EE81EF91E0E942A741A
:10B0D0006C197D098E099F0997FF7CC080E00E9452
:10B0E000A1DFF4CF8232910509F444C360F48D31BD
:10B0F000910509F46CC208F4C3C04E9709F4BFC2AD
:10B100000F94532367C08A35910509F4F8C308F5F5
:10B110008A97B1F780911306813009F05BC089E40A
:10B120000E945FBE082FF12C882319F00E94E3BD16
:10B13000F82E8AE40E945FBEE82E882309F41DC31E
:10B140000E94E3BD182F01111BC3153008F422C360
:10B150001AC38B35910509F4D5C38C35910581F659
:10B1600080919304882309F4D1C3893099F56AEE5C
:10B17000A62E62E0B62E79E6C72E72E0D72EE12C1D
:10B1800000E010E0D5018D915D010E945FBEF82EB8
:10B19000882361F0133011F4082FFE2C0E94E7BDC4
:10B1A000F6016083718382839383EF2C1F5FF4E049
:10B1B000CF0ED11C143031F7EE2009F4F9C30E94F0
:10B1C000E0310E940B3206C0213021F40E94D51FCD
:10B1D0000E944D2B3DA9311102C00F9400238CA970
:10B1E00080932B040C948F6480E090E0A0E8BFE390
:10B1F0009DCEC12CD12C7601DECE89E40E945FBEAB
:10B20000882331F00E94E7BD69837A838B839C8316
:10B210008AE40E945FBE882309F402CF0E94E7BD42
:10B22000FBCE412FBE016F5F7F4F8BEA97E00E94FC
:10B2300078930E942A746093F9117093FA118093A5
:10B24000FB119093FC11C6CF0E94B9D3C3CF87E006
:10B250000E94DD528111BECF8CE0EEEDF2E0DE0106
:10B26000119601900D928A95E1F770E060E080E51B
:10B270000E94C71FBE016F5F7F4F0E943736AACF63
:10B2800087E00E947F2A811106C060E08FE40E945F
:10B29000FEBE81119FCF0E94D42310924E02609176
:10B2A000BC0C8CE40E94FEBEE82E80E00E94A5C18A
:10B2B0000E942A746093F9117093FA118093FB1124
:10B2C0009093FC110E94192E81E08093CF050E947B
:10B2D00074338AE50E9411BEF82E882369F081E05C
:10B2E0000E947F2A182F82E00E947F2A11110C945D
:10B2F000516C11E0811101C010E088E50E9411BE7F
:10B3000081110C94436C111149C189E50E9411BE51
:10B31000082F811307C0012FF11204C011E001E0D2
:10B32000FF24F39482E50E945FBE882309F439C1AB
:10B330000E94E7BD6CA37DA38EA39FA320E030E015
:10B34000A9010F947432882381F0111105C00111F5
:10B3500003C0FF2009F414C160E0CE0184960E946E
:10B36000D4300E9484C50E944EC5112309F47DC0CB
:10B37000002309F477C01092690210926A021092B9
:10B380006B0210926C0210926D0210926E0210927B
:10B390006F02109270020E94E03182E49FE00E94EE
:10B3A00074B84B015C0186E49FE00E9474B82B01E5
:10B3B0003C01AC019B01C501B4010F94A43B1816DC
:10B3C0000CF0F4C0A5019401C301B2010F943E3A00
:10B3D0009B01AC010F94DA3220E030E040E85FE3FB
:10B3E0000F9444390F94F23B20E030E048E452E4FB
:10B3F0000F94DA3268A379A38AA39BA320E030E0FC
:10B4000040EC5FE3C301B2010F94DA3269837A83BF
:10B410008B839C8320E030E040EC5FE3C501B40106
:10B420000F94DA326C8F7D8F8E8F9F8FAE01405ECE
:10B430005F4FBE016F5F7F4FCE014C960E949330ED
:10B440000E948A1F1092690210926A0210926B0287
:10B4500010926C0210926D0210926E0210926F02A6
:10B460001092700280E00E940934002319F081E0FC
:10B470000E940934FF2009F483C010921205109233
:10B4800011051092130583E00E94DD52811178C0EE
:10B490000E94E03120913D0830913E0840913F08E4
:10B4A0005091400860E070E080E393E40F944339EA
:10B4B0002B013C0120914108309142084091430802
:10B4C0005091440860E070E084E393E40F944339C2
:10B4D0004B015C018091710290917202A091730204
:10B4E000B09174028093B3079093B407A093B5070B
:10B4F000B093B6070091071310910813D8012D914E
:10B500003D914D915C91C301B2010F944339609319
:10B51000AB077093AC078093AD079093AE07F8012B
:10B520002481358146815781C501B4010F94433987
:10B530006093AF077093B0078093B1079093B20701
:10B540008BEA97E00E946EBD8823A9F11C8E1D8EA8
:10B550001E8E1F8E88E0EBEAF7E0DE011196019067
:10B560000D928A95E1F7AE01445E5F4FBE016B5FBD
:10B570007F4FCE0101960E94933082E00E940934F1
:10B580000E94E0318091CE058093CF058E2D0E94E0
:10B59000A5C10E94002E0E940B321CCE012F10E08C
:10B5A000C1CE60E070E080E890E4C4CEA3019201D7
:10B5B000C501B4010BCF60E081E995E00E94EC3C4D
:10B5C0000E94F6DB8FE795E00E9492C7D9CF14E086
:10B5D0000E942A746093F9117093FA118093FB1101
:10B5E0009093FC118091BC0C811127C08EE40E94C5
:10B5F00011BE882321F082EA95E00E94836C87E0E7
:10B600000E94DD5281111FC00E94CDE68823D9F02F
:10B61000115001F130E020E04AE25EE06DEC75E0AF
:10B6200085E00E94FAC861E080EC95E00E94A1C824
:10B6300088EA95E00E94836CCBCF60E08FE40E94A3
:10B64000FEBE882399F20E94D2C88BE696E00E9443
:10B65000836CC0CD61E08EE596E00E94A1C889EEC2
:10B6600095E00E94836C61E085E19EE00E94A1C8A4
:10B6700040E070E060E08AED95E00E94D0DE00914D
:10B68000071310910813D8012D913D914D915C91B4
:10B690006091690270916A0280916B0290916C02D4
:10B6A0000F944439AB01BC0188E50E94CCBE69838C
:10B6B0007A838B839C83F80124813581468157816D
:10B6C00060916D0270916E0280916F029091700294
:10B6D0000F944439AB01BC0189E50E94CCBE6D8357
:10B6E0007E838F839887BE016B5F7F4FCE0101966B
:10B6F0000E949DB8882309F46DCD80E00E94A5C109
:10B700000E94192E61E085E40E94FEBE182F01E020
:10B7100021E0482FBE016B5F7F4FCE0101960F9451
:10B7200090236B017C01AC019B010F94363C81118D
:10B7300019C049815A816B817C818DE896E00E9415
:10B74000C3C94D815E816F81788588E896E00E944B
:10B75000C3C9B701A60183E896E00E94C3C98AE085
:10B760000E946AC70E94002E11110E9483B80E9495
:10B770000B3230CD0E9420CF2DCD10E0002351F0B0
:10B78000F4E0FF1528F485E996E00E9492C722CDE7
:10B79000E110DBCC80E1E9E6F2E0ABEAB7E0019052
:10B7A0000D928A95E1F7002319F16F2DFF0C770BAD
:10B7B000880B990B0F947B322091FD043091FE048D
:10B7C0004091FF04509100050F94DA322091F50466
:10B7D0003091F6044091F7045091F8040F944439E5
:10B7E0006093AB077093AC078093AD079093AE075F
:10B7F000EE2019F1612F110F770B880B990B0F9425
:10B800007B32209101053091020540910305509152
:10B8100004050F94DA322091F9043091FA04409132
:10B82000FB045091FC040F9444396093AF0770936C
:10B83000B0078093B1079093B20760E080E50E9463
:10B84000FEBE8823C1F10023D1F0E0910713F091EF
:10B85000081320813181428153816091AB0770913F
:10B86000AC078091AD079091AE070F944339609378
:10B87000AB077093AC078093AD079093AE07EE20B3
:10B88000D1F0E0910713F0910813248135814681AE
:10B8900057816091AF077091B0078091B107909187
:10B8A000B2070F9443396093AF077093B00780934A
:10B8B000B1079093B20740E050E0BA0186E40E94DD
:10B8C000CCBE6B017C0120E030E0A9010F94A43BC9
:10B8D00018168CF420E030E040E752E4C701B601CE
:10B8E0000F943E3A69837A838B839C83CE010196C1
:10B8F0000E94382E6FCC60E070E0CB01F3CF109245
:10B900002B0868CC8FE080932B0864CC5AEEC52EB0
:10B9100052E0D52EF12CE12C00E010E0D6018D9103
:10B920006D010E945FBE382E8823D9F10E94E7BDC9
:10B930004B015C01133059F0F701E95FF64F2081AC
:10B940003181428153810F9443394B015C01F701EE
:10B95000E759FD4F2081318142815381C501B401F6
:10B960000F9443392B013C012DEB37E346E855EBAF
:10B970000F94A43B87FD0AC02DEB37E346E855E35F
:10B98000C301B2010F94743218165CF41330C1F481
:10B990008092750290927602A0927702B09278021D
:10B9A000032D1F5FB4E0EB0EF11C143009F0B6CF8D
:10B9B000002309F406CC85E792E00E94A52701CC7C
:10B9C000F701EF5CF74F5F01A30192016081718184
:10B9D000828193810F944439D5016D937D938D932A
:10B9E0009C931397812F0E94081DDBCF80919404B4
:10B9F000909195048937910511F40C94A26608F092
:10BA0000B2C18D34910509F497C608F0CEC08A31D1
:10BA1000910509F4CCC508F071C08431910509F491
:10BA200012C508F04EC08131910509F4D1C408F067
:10BA300042C0029708F064CB80E50E945FBEC12C33
:10BA4000D12C7601882321F00E9464B86B017C011F
:10BA500083E50E945FBE882361F00E94E7BD20E07D
:10BA600030E04AE754E40F94DA320F94B73A6B01AE
:10BA70007C010E94D4238091970490919804892B93
:10BA800009F4A1C40F9461238091940490919504CA
:10BA900066EB76E0892B11F46EEA76E030E020E088
:10BAA0004EEB56E082E00E94FAC840E0C701B601C2
:10BAB0000E94E6EE8FCB429709F022CB0E946CBE2B
:10BAC00089CB8731910509F4F3C470F48531910570
:10BAD00009F4EAC4469709F013CB8091C41482FD9F
:10BAE00079CB0E94518076CB8831910509F4F5C459
:10BAF000499709F005CB0E9432226CCB8032910528
:10BB000009F4D9C5C0F58D31910509F4BDC570F4AE
:10BB10008B31910509F45EC54C9709F0F1CA80910B
:10BB20009704909198040E94438554CB8E319105DF
:10BB300009F4B1C54F9709F0E3CA0E94EA356C8F4A
:10BB40007D8F8E8F9F8FBE016F5F7F4FCE014C9692
:10BB50000E94601ECE0101960E94F5F40E94F6DB61
:10BB6000BE016F5F7F4F82E397E00E94E8DB8AE0CF
:10BB70000E946AC72FCB8934910509F4C9C550F4D6
:10BB80008132910509F4C0C5C09709F0B9CA0E9475
:10BB900063CA20CB8B34910509F4CAC58C34910556
:10BBA00009F0AECA0E94933915CB8C36910509F481
:10BBB00011CB08F071C08535910509F4B0C790F537
:10BBC0008235910509F49BC720F58E34910509F45F
:10BBD000B7C58135910509F093CA0E94EB8B0E948D
:10BBE000E5230E94CFC30E94D2C31092C6071092D1
:10BBF000C5071092C40768EE73E080E090E00E94F1
:10BC0000C2C20E94D7C360E08DEF97E00E94EC3C77
:10BC1000E1CA8335910509F47AC78435910509F4A1
:10BC20004DCF6ECA8936910509F467C600F58C358B
:10BC3000910509F499C78836910509F061CA809188
:10BC4000790C83FDC7CA0E94022187FDC3CA83E520
:10BC50000E945FBE882341F00E94E3BD0E94A4239E
:10BC600061E080E00F9474260F94D325B3CA8A361E
:10BC7000910509F46DC68B36910509F041CA60E063
:10BC800080E50E94F2BE823008F0A4CAE82FF0E0FE
:10BC9000E45CF64F10829ECA8237910511F40C9431
:10BCA0005566A0F58F36910509F47BC6C8F48D362C
:10BCB000910509F4D7C58E36910509F021CA8EE4A5
:10BCC0000E945FBE882309F485CA0E94AFBD6093BD
:10BCD000A90D7093AA0D8093AB0D9093AC0D7ACA09
:10BCE0008037910509F476CA8137910509F008CAB1
:10BCF00083E50E945FBE882309F49AC60E94BFBDF7
:10BD00008D3308F090C68093000264CA863791058F
:10BD100009F4DBC7B8F48337910509F4CEC785373A
:10BD2000910509F0EDC980919704909198040097CE
:10BD300009F4C7C7DC012C91222309F4C2C70E9471
:10BD4000F5F448CA8737910511F40C949E6688373C
:10BD5000910509F0D5C981E08093CF058093CE0588
:10BD60000E94743337CA8A39E1E09E0709F432CA67
:10BD700008F0D0C18C3D910511F40C944D6708F08A
:10BD800076C0893C910509F4E7C708F055C08B39A6
:10BD9000910509F48DC6D8F48D37910509F4ABCE21
:10BDA0008C38910509F0ACC98091790C83FD12CAD9
:10BDB00083E50E945FBE882309F40CCA0E94E3BD9C
:10BDC0000E9463BD61E080E00F94742603CA8E3B3D
:10BDD000910509F43AC6883C910509F091C90E9481
:10BDE0000221182F87FDF6C90091300884E40E94D3
:10BDF0005FBEF82E8823B9F00E94E7BD4B015C01BD
:10BE000020E030E0A9010F947432882309F4A2C71E
:10BE100024E01202F0011124E45DF74F8082918248
:10BE2000A282B3820F2D602F83E50E94FEBE809315
:10BE300030080E942D24CEC98D3C910509F4D9C744
:10BE400058F48B3C910509F4B1C78C3C910509F07D
:10BE500057C90E94D4C9BEC98E3C910509F4CDC70B
:10BE6000833D910509F04CC90E94D355B3C98E3268
:10BE700021E0920711F40C94886808F0B4C0823273
:10BE8000A1E09A0711F40C94666848F58D3D910580
:10BE900011F40C9490678831914009F031C980E524
:10BEA0000E9411BE882309F495C90E94E3BD8C014C
:10BEB000892B11F00C94596883E50E9411BE8823E8
:10BEC00011F40C94EE670E94E3BD8F3F980711F0C8
:10BED0000C94E76788EF92E10E94DCC37BC98C3247
:10BEE000F1E09F0711F40C946A688D32914009F0DB
:10BEF00007C960E085E40E94F2BE81110C9480685D
:10BF000080E50E9411BE882351F00E94E7BD609336
:10BF1000731270937412809375129093761289E461
:10BF20000E9411BE882381F00E94E7BD2CEA35EC07
:10BF300047E25EE30F94DA326093771270937812DF
:10BF40008093791290937A1284E40E9411BE882320
:10BF500081F00E94E7BD2CEA35EC47E25EE30F94E6
:10BF60003E3A60937B1270937C1280937D12909383
:10BF70007E120E94F6DB4091731250917412609110
:10BF80007512709176128EE498E00E94C3C92CEA73
:10BF900035EC47E25EE36091771270917812809100
:10BFA000791290917A120F943E3AAB01BC018AE467
:10BFB00098E00E94C3C92CEA35EC47E25EE3609149
:10BFC0007B1270917C1280917D1290917E120F9461
:10BFD000DA32AB01BC0186E498E00E94C3C98AE072
:10BFE0000E946AC7F7C8803931E0930711F40C94B6
:10BFF000136908F07DC08F32B1E09B0711F40C94F7
:10C00000CE688033914009F07BC880E50E9411BE64
:10C01000882351F00E94E7BD6093081270930912C3
:10C0200080930A1290930B1289E40E9411BE882318
:10C0300081F00E94E7BD2CEA35EC47E25EE30F9405
:10C04000DA3260930C1270930D1280930E1290935B
:10C050000F1284E40E9411BE882381F00E94E7BD84
:10C060002CEA35EC47E25EE30F943E3A60931012FF
:10C070007093111280931212909313120E94F6DBA8
:10C08000409108125091091260910A1270910B129E
:10C090008CE698E00E94C3C92CEA35EC47E25EE3E7
:10C0A00060910C1270910D1280910E1290910F12EE
:10C0B0000F943E3AAB01BC0188E698E00E94C3C9E8
:10C0C0002CEA35EC47E25EE3609110127091111298
:10C0D00080911212909113120F94DA32AB01BC01CD
:10C0E00084E698E00E94C3C98AE00E946AC772C8C9
:10C0F0008139F1E09F0711F40C941769823991405E
:10C1000011F00C9480580E947AB80E9483B80E9463
:10C110000B3260C88C3032E0930711F40C94B26A91
:10C1200008F068C08C3AB1E09B0711F40C94F169F7
:10C1300070F5843AF1E09F0711F40C947469C8F427
:10C140008C3931E0930711F40C9421698D399140B9
:10C1500011F00C94805883E50E9411BE882311F4DD
:10C160000C94176C0E94D3BD8093E4040E9492BF8C
:10C1700031C8853AB1E09B0711F40C947869863A8E
:10C18000914011F00C9480580E943BCE23C8863F0A
:10C19000F1E09F0711F40C94A46A70F4843F31E03D
:10C1A000930711F40C94A06A853F914011F00C9410
:10C1B00080580E94FEB20EC8873FB1E09B0711F481
:10C1C0000C94A86A883F914011F00C94805881E04B
:10C1D000809309050E94FF2210920905882311F41B
:10C1E0000C94EA580E94F6DB86E799E00E9492C719
:10C1F0000C94EA588C36F3E09F0711F40C94EA583B
:10C2000008F091C08D3B32E0930711F40C94DD6A85
:10C2100008F07AC08835B2E09B0711F40C94C36A29
:10C220008B35924011F00C9480580E940221082F07
:10C2300087FF02C00C94EA5885E50E9411BE88234E
:10C2400069F10E94E7BD4B015C01E02E002E000C5D
:10C25000FF0820E030E0A9010F94A43B87FF04C051
:10C26000B7FAB094B7F8B09420E030E84BE354E468
:10C27000C501B4010F94A43B970153E0220F331F73
:10C280005A95E1F724523B4F181614F40C94C76AE0
:10C29000D9018D929D92AD92BC9213978CE40E942D
:10C2A00011BE882311F40C94EA580E94E7BD6B017B
:10C2B0007C01002E000C110B20E030E0A9010F944E
:10C2C000A43B87FF04C0F7FAF094F7F8F09420E05D
:10C2D00030E84BE354E4C701B6010F94A43B980146
:10C2E00043E0220F331F4A95E1F724523B4F1816C3
:10C2F00014F40C94D26AD9011496CD92DD92ED9289
:10C30000FC9217970C94EA588E3BF2E09F0711F4C9
:10C310000C94E16A8335934011F00C9480580E948C
:10C32000F6530C94EA58873E33E0930711F40C94CB
:10C33000076CC8F48438B3E09B0711F40C949C6B31
:10C34000803A934011F00C948058209197043091DA
:10C3500098049091C41492609093C414C9010E94EF
:10C3600043850C94EA58883EF3E09F0711F40C943F
:10C37000236C893E934011F00C9480588091BA143C
:10C3800081110C94276C0E948ABF0E9438850E94FC
:10C39000EA356D3371058105910520F08CED99E04A
:10C3A0000E94836C88ED99E00E94836C84EE8093F8
:10C3B000A30484EC99E00E9492C780EC99E00E946B
:10C3C000836C0C94EA5887EC96E00E9435375CCB7E
:10C3D0008091460484FD18C08091480487FD14C0F4
:10C3E00080914904837081F460E08AED96E00E94B8
:10C3F000EC3C5F988A9880910801817080930601D7
:10C40000479812980C94EA5888E50E9411BE811151
:10C410005F9889E50E9411BE81118A988AE50E9481
:10C4200011BE882331F0809108018170809306014C
:10C43000479885E40E9411BE882311F40C94EA58B1
:10C4400012980C94EA588091C41483FF25C082EF9F
:10C4500096E00E9492C78091C41483FF17C084EEB7
:10C4600094E10E94C8808BE1E4EEF4E1DE011196D4
:10C4700001900D928A95E1F770E060E0CE0101969F
:10C480000E947F86CE0101960E94B2BF83EE96E0A5
:10C490000E9492C70C94EA580E94F6DB83E097E072
:10C4A0000E9492C70C94EA580E9462800C94EA5849
:10C4B0008091970490919804FC012191222331F0FE
:10C4C0002032D9F7DF0111971C92F7CF60E00E946C
:10C4D0008C851092A3040C94EA5883E50E945FBEF9
:10C4E000882321F00E94AFBD0E94F25084E50E9493
:10C4F0005FBE8823A9F00E94AFBD6B017C010E9442
:10C500001C36C092C604D092C704E092C804F092D0
:10C51000C904CD28CE28CF2819F081E08093A71137
:10C520008091A6118823F9F080E090E0A0EAB1E4C0
:10C5300089839A83AB83BC831C8E1D8E1E8E1F8EB7
:10C5400018A219A21AA21BA210E000E020E0AE017E
:10C550004F5F5F4FBE01645E7F4FCE0180960E94A9
:10C560000DED0C94EA580E94C1C3882381F00E940B
:10C570003F780E94E63887E898E00E94F07F1092AA
:10C58000100E1092110E1092120E1092130E61E006
:10C590008DE39EE00E94A1C84AE25EE06DE077E094
:10C5A00085E00E943BF30E942DF50C94EA5880919F
:10C5B000C41483FD02C00C94EA5883E50E945FBE58
:10C5C000882311F40C94EA580E94AFBD0E94F250E7
:10C5D0000C94EA5883E40E9411BE882361F183E23F
:10C5E00097E00E9492C780912B168823F9F0BE0134
:10C5F0006F5F7F4F88E296E10E94837FCE010196B4
:10C600000E94357CCE0101960E940E8180912212FB
:10C61000882339F080E20E946AC782E292E10E9498
:10C62000357C8AE00E946AC70C94EA5889E197E059
:10C630000E9492C7F6CF83E50E945FBE882301F176
:10C640000E94BFBD182F8C3308F08CE38093200428
:10C650000E942A746B017C01212F30E0A8EEB3E028
:10C660000F940C39C60ED71EE81EF91EC0921C048A
:10C67000D0921D04E0921E04F0921F040C94EA581C
:10C680000E94FD770C94EA588091C4148E7F8093A9
:10C69000C4140C94EA588091C41483FD02C00C9415
:10C6A000EA580F94E62280919704909198040E9492
:10C6B000D0840C94EA588091C41482FD0E94D42343
:10C6C0008091C41483FD02C00C94EA5860E080E5B8
:10C6D0000E94FEBE182F682F8091970490919804B5
:10C6E0000E948C8583E50E945FBE882321F00E9412
:10C6F000AFBD0E94F2500E943F7811110C94EA588D
:10C700000E94E6380C94EA580E9431530C94EA587F
:10C7100080E50E9411BE882311F40C94EA580E940F
:10C72000BFBD853608F084E68093A3040C94EA58D4
:10C730000E94E6380C94EA580E94CFC30C94EA5841
:10C7400070E060E083E50E94E3BE8E34910531F431
:10C750000E9443230E942DF50C94EA588DE997E03E
:10C760000E9492C76091BE057091BF0584E997E071
:10C770000E94B1C96091C0057091C10587E897E03A
:10C780000E94B1C96091BE057091BF058091C0053E
:10C790009091C105681B790B8091A711815021E010
:10C7A00030E0823010F030E020E0621B730B8CE749
:10C7B00097E00E94B1C98AE00E946AC784E797E0C7
:10C7C0000E9492C78091C2059091C305A091C405B3
:10C7D000B091C5058C8F9D8FAE8FBF8FBE016F5FEF
:10C7E0007F4FCE014C960E94601EBE016F5F7F4F4F
:10C7F00087E697E00E94E8DB8091C6059091C70527
:10C80000A091C805B091C9058C8F9D8FAE8FBF8F49
:10C81000BE016F5F7F4FCE014C960E94601EBE012D
:10C820006F5F7F4F87E597E00E94E8DB20E030E014
:10C830004AE754E46091CA057091CB058091CC051C
:10C840009091CD050F943E3AAB01BC018FE397E088
:10C850000E94C3C98DE60E946AC78AE00E946AC727
:10C860000C94EA588091790C83FF02C00C94EA582A
:10C870000E940221082F87FF02C00C94EA5883E52A
:10C880000E945FBE182F882359F10E94E3BD0E94C9
:10C89000A42361E081E00F947426209170123091FE
:10C8A000711280916E1290916F1282179307F4F4B7
:10C8B00080EB97E09F938F938BEB97E09F938F9301
:10C8C0001F920F94CC220F94D3250F900F900F90AE
:10C8D0000F900F90612F802F0E94068A0C94EA58C7
:10C8E00082E50E945FBE8111D0CFBEC985EA97E084
:10C8F000112301F30F94D325EDCF0E940221182FAD
:10C9000087FD0AC080EC97E00E9492C7812F0E94A9
:10C910001C888AE00E946AC73CA930932B04E596E4
:10C920000FB6F894DEBF0FBECDBFDF91CF911F9140
:10C930000F91FF90EF90DF90CF90BF90AF909F90BE
:10C940008F907F906F905F904F903F902F900895C1
:10C9500060E080E50E94F2BEF82E81E08F1510F4B1
:10C960000C94EA5881E40E9411BE60913C09062FA4
:10C97000811102C00FEF10E083E50E945FBE8823A3
:10C9800049F00E94AFBD8B016F3F710519F010F0A7
:10C990000FEF10E0EF2DF0E0E45CF64F00830C9415
:10C9A000EA5883E50E9411BE882331F060E083E5F8
:10C9B0000E94F2BE8093790C0E94F6DB81ED97E035
:10C9C0000E9492C78091790C882351F110E000E019
:10C9D00020E08091790C90E0B0E0A0E0002E04C04F
:10C9E000B695A795979587950A94D2F780FF12C0C0
:10C9F000FF24F394F20E222319F08CE20E946AC7FE
:10CA0000F801EE0FFF1FE953F84F859194910E94B2
:10CA100092C72F2D0F5F1F4F05301105D1F601CEA4
:10CA200083EC97E005CE8CE3809300020C94EA58E7
:10CA30000E94F6DB6091000288ED97E00E94BBC97E
:10CA40008AE00E946AC70C94EA588091790C83FFAF
:10CA500002C00C94EA5883E50E945FBE182F882319
:10CA6000E9F00E94E3BD0E9463BD60E081E00F94A5
:10CA70007426209105123091061280910312909134
:10CA80000412821793078CF08FED97E060E00E940C
:10CA9000EC3C812F0E948F880C94EA5882E50E941A
:10CAA0005FBE8111DECF0C94EA588EEE97E0EECF98
:10CAB00083E50E945FBE882311F40C94EA580E941B
:10CAC000BFBD182F8C3308F08CE3809325040E949F
:10CAD0002A746B017C01212F30E0A8EEB3E00F94A3
:10CAE0000C39C60ED71EE81EF91EC0922104D09242
:10CAF0002204E0922304F09224040C94EA588091DA
:10CB00002B088F7D806180932B080C94EA588091CC
:10CB10002B088F7E806280932B080C94EA5883E563
:10CB20000E9411BE882311F40C94EA580E942A74C2
:10CB30006093F9117093FA118093FB119093FC119B
:10CB40000E94E7BD20E030E04AE754E40F94DA3277
:10CB50000F94B73A609326047093270480932804B7
:10CB6000909329040C94EA580E94022187FF02C086
:10CB70000C94EA588091460484FD09C080914804D1
:10CB800087FD05C080914904837009F489C02AEEAD
:10CB9000C22E22E0D22E31ECE32E3CE0F32E10E048
:10CBA000D6018D916D010E945FBE882309F465C096
:10CBB000133009F06DC00E94E7BD4B015C0120E01D
:10CBC00030E040EA51E40F94743287FF4EC0A50173
:10CBD00094016091E10C7091E20C8091E30C9091D2
:10CBE000E40C0F943E3A2B013C01AC019B01609197
:10CBF00034097091350980913609909137090F9465
:10CC0000DA32609334097093350980933609909332
:10CC10003709A30192016091F10C7091F20C80919F
:10CC2000F30C9091F40C0F94DA326093F10C709342
:10CC3000F20C8093F30C9093F40C609120097091A6
:10CC4000210980912209909123090F947932A3013F
:10CC500092010F94DA320F94B73A609320097093DF
:10CC6000210980932209909323098092E10C9092EC
:10CC7000E20CA092E30CB092E40C1F5FF4E0EF0E24
:10CC8000F11C143009F08CCF0E94B0230C94EA58A8
:10CC90000E94E7BDF701648B758B868B978BEDCF78
:10CCA00081E00F9473220C94EA580F9404208EE1D3
:10CCB00093E10E94A2970C94EA580E948D1D0C9457
:10CCC000EA580E942DF50C94EA58009197041091AF
:10CCD000980494E0F12C40E09150F9F0F801808143
:10CCE000282F2B7F213499F421812133B1F4813411
:10CCF00011F1853409F441E098012E5F3F4F89011D
:10CD00002F5F3F4FF80180818032C9F3E5CF803536
:10CD100021F4818180538A3078F341110E94F6DB3F
:10CD2000FF2021F08FE098E00E9492C7C8010E9486
:10CD3000CC520C94EA58FF24F394DECF0E943F1F9C
:10CD40000C94EA581092CF051092CE050E947433CD
:10CD50000C94EA5880E06BC80E94022187FF02C051
:10CD60000C94EA580AEE12E081ECE82E8CE0F82EE2
:10CD70009EEEC92E92E0D92ED8018D918D010E9490
:10CD800011BE882359F00E94E7BD0F94B73AF7010E
:10CD900060837183828393830E94BA1CF4E0EF0E58
:10CDA000F11CC016D10641F70C94EA580E940221EA
:10CDB00087FF02C00C94EA581AEEE12E12E0F12E21
:10CDC00010E000E0D7018D917D010E9411BE882303
:10CDD00049F00E94E7BDF801EF53F34F64A375A338
:10CDE00086A397A30C5F1F4F0031110559F70C94D0
:10CDF000EA580E94A0C70C94EA58BDE3EB2EB8E0B5
:10CE0000FB2E10E088E5810F0E9411BE882351F0AF
:10CE10000E94E7BDF7016083718382839383812F32
:10CE20000E94081D1F5FF4E0EF0EF11C133051F754
:10CE30008091480487FF02C00C94E1588091490416
:10CE4000837011F00C94E15840913D0850913E08D8
:10CE500060913F087091400882E198E00E94C3C948
:10CE600040914108509142086091430870914408F4
:10CE70008AE691E30E94C3C9409145085091460853
:10CE8000609147087091480887E691E30E94C3C902
:10CE90008AE00E946AC70C94EA5882E40E9411BE9C
:10CEA000882341F080917F0290918002909302024A
:10CEB0008093010282E50E9411BE882341F0809197
:10CEC0000102909102029093800280937F0283E599
:10CED0000E945FBE882331F00E94E3BD90938002E0
:10CEE00080937F028091460490914704A09148046A
:10CEF000B0914904892B8A2B8B2B11F00C94EA58A2
:10CF000060917F027091800289E198E00E9459CA85
:10CF100085E20E946AC78AE00E946AC70C94EA58B8
:10CF20000E940221082F87FF02C00C94EA5883E573
:10CF30000E945FBE002E000C110B7801EE0CFF1C4E
:10CF4000882359F10E94E3BDF701E358FD4F918317
:10CF50008083000F111F000F111F980127583D4FAC
:10CF60007901BC01990F880B990B0F947B322AE051
:10CF700037ED43E25CE30F94DA320354134FD801E8
:10CF80002D913D914D915C910F94DA32F7016083C0
:10CF90007183828393830C94EA580E94F6DB85E4C4
:10CFA0000E946AC780E3800F0E946AC7F701E358B6
:10CFB000FD4F608171818DE198E00E9459CA85E240
:10CFC0000E946AC78AE00E946AC70C94EA58BC01B2
:10CFD00088EF92E10E944AC40C94EA580E94F6DB62
:10CFE00070E060E088E298E00E9459CA8091FA12ED
:10CFF00058E5C52E52E0D52EC81AD10887FDD39426
:10D00000CC0CDD1CCC0CDD1C0D2C000CEE08FF083C
:10D010008091F91278E8872E912C881A910887FD63
:10D020009394880C991C880C991C092C000CAA0854
:10D03000BB088091F81290E08F3FC9F1FC01EE0F20
:10D04000FF1FE80FF91FE155FD4E8181928133E00A
:10D05000880F991F3A95E1F7B0E0A0E044E0B5955C
:10D06000A795979587954A95D1F702969C012F5FD2
:10D070003F4F032E000C440B550B281939094A0960
:10D080005B09A4EBB0E00F94F938A70196012819C9
:10D0900039094A095B090F94DA38B90185E298E049
:10D0A0000E9459CA8AE00E946AC70C94EA5880E03C
:10D0B000DDCF0E94F2DBB8018FE398E00E9459CAED
:10D0C00080E398E00E9492C70C94EA580E94385579
:10D0D0000C94EA5864E071E083E50E94C71F8C015C
:10D0E00068EE73E080E50E94C71F893823E192074C
:10D0F00010F088E893E1B8010E945A3A0C94EA587B
:10D100000E94F2DB82E598E00E9492C70C94EA58F4
:10D1100083E50E9411BE182F882369F00E94E3BDA9
:10D120009C01909368028093670291E0232B09F0A1
:10D1300090E090933E0980E50E9411BE882361F043
:10D140002091670230916802232B11F00E94D3BD19
:10D1500080933E090C94EA5811110C94EA580E94ED
:10D16000F6DB8CE898E00E9492C780913E09882304
:10D1700091F084E798E00E9492C7609167027091F5
:10D1800068028BE798E00E9459CA87E798E00E94FE
:10D1900092C70C94EA5880E798E0EDCF70E060E029
:10D1A00085E40E94E3BEF82E3FEF8317C9F1882380
:10D1B00041F08CEA98E00E9492C70E9444F30C94DC
:10D1C000EA5804EB10E083E50E945FBE882319F063
:10D1D0000E94E3BD8C0165E070E083E40E94E3BE41
:10D1E000E82E60E085E50E94FEBED82E60E08FE963
:10D1F00098E00E94EC3CB801110F880B990B0F943A
:10D200007B3269837A838B839C832D2D4E2D6F2DEA
:10D21000CE0101960E94B4A60E942DF50C94EA5806
:10D2200006E410E0D0CF0E94D4230C94EA588091F9
:10D23000BB0781110C94E15881E00E9483330C9468
:10D24000E158809146048878F9F48091480486700A
:10D25000D9F40E94F6DB80EF98E00E9492C780919B
:10D260000F020E94A5C940910B0250910C026091DF
:10D270000D0270910E0280ED98E00E94C3C98AE011
:10D280000E946AC70C94EA5888E40E9411BE882361
:10D2900021F00E94D3BD80932A0482E50E9411BE32
:10D2A000082F83E50E9411BE182F011102C08823A8
:10D2B00041F00E9476C3112321F00E94D3BD8093D8
:10D2C0000F0284E40E9411BE882311F40C94EA58E2
:10D2D0000E94E7BD60930B0270930C0280930D02D5
:10D2E00090930E020C94EA580E94FADB0C94EA58D0
:10D2F0006FEF7FEF89E40E94E3BE082F6FEF7FEFAF
:10D300008AE40E94E3BE182F8AE50E945FBED12CFA
:10D31000811107C081E50E945FBED82E882309F4E1
:10D32000B8C2C02E81E0800F863008F052C0912E26
:10D3300081E0810F863008F04CC00E94E7BD2B01D0
:10D340003C01F02E07FDF12C07FF02C004E0C02EC7
:10D35000812E17FD812C17FF02C014E0912EB5E03D
:10D360003B2ECF1410F40C94EA58E82C3F9C50014B
:10D3700011249E1460F10E2D10E020E030E0A90190
:10D38000DD2069F0F501E00FF11FEE0FFF1FEE0F3A
:10D39000FF1FE953F84F20813181428153810A0DEB
:10D3A0001B1D000F111F000F111F0953184FC30140
:10D3B000B2010F944439D8016D937D938D939C9362
:10D3C00013976E2D8F2D0F94A121E394D2CFF39458
:10D3D000C8CF0E94F2DB81E299E00E9492C70C94D0
:10D3E000EA5887E00E94DD5281110C94EA5876E3F6
:10D3F000C72E7FE0D72EE9E6F2E0F9A7E8A79E0165
:10D400002F5F3F4F1901790110E000E0C6010E9433
:10D4100074B8A8A5B9A58D909D90AD90BD90B9A701
:10D42000A8A7A50194010F9443392B013C01F701F2
:10D43000408251826282738220E030E040EA51EC07
:10D440000F94A43B87FD0AC020E030E040EA51E49D
:10D45000C301B2010F947432181684F4F801E65A2D
:10D46000F04FE4911E1654F4B7FAB094B7F8B094A4
:10D47000D7018D929D92AD92BC921397F701819046
:10D480009190A190B1907F0120E030E040EA51EC12
:10D49000C501B4010F94A43B87FD3FC020E030E0FC
:10D4A00040EA51E4C501B4010F9474321816ACF18E
:10D4B0000F5F1F4FF4E0CF0ED11C0330110509F0B0
:10D4C000A5CF6DE3E62E68E0F62E10E0F101819124
:10D4D0009191A191B1911F01F70181939193A19332
:10D4E000B1937F01812F0E94081D1F5F133071F7D8
:10D4F0000E940B3260E08AE399E00E94EC3C63E911
:10D5000072E084E690E00E945A3A6AEB72E084E6A8
:10D5100090E00E945A3A0C94EA580E94F2DB88E5A7
:10D5200099E00E9492C761E08AE499E00E94EC3C95
:10D5300068E270E088EC90E00E945A3A0C94EA5855
:10D540000E94363D0C94EA580E943EA50C94EA587D
:10D5500061E083E50E94FEBE91E089270E94C8AB8E
:10D560000C94EA588091C41482FF05C080648093B3
:10D57000C4140C94EA5883FD02C00C94EA580F942A
:10D58000E6220C94EA580E9427210C94EA5880E085
:10D5900090E8ABE3B4E4F90180839183A283B38381
:10D5A0000C944E6180E090E8ABE3B4E4F90184832D
:10D5B0009583A683B7830C94EA580E94D82E0C94C6
:10D5C000EA580E940221182F87FF02C00C94EA58E3
:10D5D0008AE50E945FBE812C912C90E2A92E91E4F5
:10D5E000B92E882379F040E050E0BA018AE50E9424
:10D5F000CCBE4B015C0120E030E0A9010F94A43BBC
:10D6000018167CF580E090E0A0EAB0E489839A8364
:10D61000AB83BC83209171023091720240917302FE
:10D6200050917402C501B4010F9444396B017C011F
:10D6300020E030E048EC53E40F94743287FD06C0DC
:10D64000C12CD12C88ECE82E83E4F82ECC8EDD8E14
:10D65000EE8EFF8EBE016F5F7F4FCE014C960E9413
:10D66000B53085E50E9411BE882309F45AC00E9496
:10D67000E7BD6B017C0120E030E0A901C701B601E4
:10D680000F94A43B87FF04C0F7FAF094F7F8F094E6
:10D69000F7FAF094F7F8F094C982DA82EB82FC8210
:10D6A00080E00E94ACEC882321F0CE0101960E941C
:10D6B000E6C220E030E0A901C501B4010F94A43B0B
:10D6C000181614F00C94EA5880E090E0A0EAB0E458
:10D6D00089839A83AB83BC83A50194016091710215
:10D6E0007091720280917302909174020F94433989
:10D6F0006B017C0120E030E0A9010F94A43B1816D7
:10D700001CF0C12CD12C7601CC8EDD8EEE8EFF8EDE
:10D71000BE016F5F7F4FCE014C960E94B5300C94D6
:10D72000EA5828E01202F0011124E452FB4FC080B5
:10D73000D180E280F3809FCFA0903809B090390962
:10D74000C0903A09D0903B098BE40E945FBE8823C9
:10D7500039F10E94E7BD7B018C0120E030E0A90196
:10D760000F94A43B87FD0AC020E030E040E251E482
:10D77000B701C8010F9474321816A4F48FE30E9405
:10D780006AC78BE40E946AC78CE899E00E9492C73E
:10D7900084E899E00E9492C781E899E00E9492C7CC
:10D7A000750186019701A801B501C6010F94743275
:10D7B000882361F00E94D423C701D80180933809DF
:10D7C00090933909A0933A09B0933B09809146049C
:10D7D00090914704A0914804B0914904892B8A2B69
:10D7E0008B2B11F00C94EA580E94F6DB409138091B
:10D7F0005091390960913A0970913B0980EA99E0AA
:10D800000E94C3C98AE00E946AC70C94EA5881E06A
:10D81000809313061092E81160E083E50E94FEBE3B
:10D8200081110C94EA580E940DF80C94EA580E9459
:10D83000F6DB8BEA99E00E9492C78091E4040E9493
:10D84000A5C90C94EA580E94F56C0C94EA580E9401
:10D85000398481110C94EA580C94C361109194049A
:10D860000E942A746093F9117093FA118093FB114E
:10D870009093FC11112311F40C94EA58812F0E940B
:10D8800066870C94EA5811110C948B5911E00C9492
:10D8900085590E94F2DB81E099E00E9492C70C94C6
:10D8A000EA58882399F30C948E59DF92EF92FF92F5
:10D8B0000F931F93CF93DF93EC01E090BD07F0909F
:10D8C000BE078AE0D82E6AE070E0CE010F94923C49
:10D8D0008C01009711F0FC011082CE010E9454517E
:10D8E00081E00E94C2560115110519F0E801D99294
:10D8F000EACFC701DF91CF911F910F91FF90EF9079
:10D90000DF900C9454514F925F926F927F928F925E
:10D910009F92AF92BF92CF92DF92EF92FF920F93BE
:10D920001F93CF93DF93CDB7DEB77C014DB65EB6C4
:10D930006090BD077090BE078DB69EB66AE070E03D
:10D94000C7010F94AF316C018C010E191F09892B8F
:10D9500021F4C7010F94C1318C01C80101962DB784
:10D960003EB7281B390B0FB6F8943EBF0FBE2DBF34
:10D970008DB79EB701965C01A801B7010F94E23103
:10D98000F501E00FF11F1082C5010E94545181E0A2
:10D990000E94C256C114D10451F076019FEFE91ADA
:10D9A000F90A0FB6F8949EBE0FBE8DBEC5CF0FB656
:10D9B000F8949EBE0FBE8DBEC3010E9454510FB697
:10D9C000F8945EBE0FBE4DBEDF91CF911F910F91B7
:10D9D000FF90EF90DF90CF90BF90AF909F908F908F
:10D9E0007F906F905F904F9008954F925F926F92EB
:10D9F0007F928F929F92AF92BF92CF92DF92EF92DF
:10DA0000FF920F931F93CF93DF93CDB7DEB7C0592B
:10DA1000D1090FB6F894DEBF0FBECDBF0E94A0BFE4
:10DA20008823B9F183E50E9411BE882309F449C017
:10DA300088E994E00E9492C78AE00E946AC78EEF4C
:10DA40008093A00481E08093860210929F0481E07D
:10DA50009AE590935B1480935A148CE490E0909331
:10DA60005D1480935C1487E080934E1482E8809369
:10DA7000511484E890E0A0E0B0E0809352149093B9
:10DA80005314A0935414B09355148EEF93E10E9455
:10DA90001C38C057DF4F0FB6F894DEBF0FBECDBFA6
:10DAA000DF91CF911F910F91FF90EF90DF90CF907A
:10DAB000BF90AF909F908F907F906F905F904F90AE
:10DAC000089583E40E9411BE882349F00E948ABF12
:10DAD0000E9438850E948D840E94BE40DACF8090DB
:10DAE000F0089090F108A090F208B090F3088091AF
:10DAF000F90880FF05C09091790C98609093790C9B
:10DB00008695817080933E0982E495E00E94836C43
:10DB100080917F08909180089E012F5F3F4F79018F
:10DB2000009799F09F938F9389E395E09F938F934C
:10DB30003F932F930F940B32C7010E94556C0F90A7
:10DB40000F900F900F900F900F9080917D08909103
:10DB50007E08009799F09F938F9380E395E09F93C1
:10DB60008F93FF92EF920F940B32C7010E94556C76
:10DB70000F900F900F900F900F900F906E0131E863
:10DB8000C30ED11C60915C0870915D0880915E08A5
:10DB900090915F08860123E041E00F94412D9F930F
:10DBA0008F938EE195E09F938F93FF92EF920F9466
:10DBB0000B32C7010E94556C86E195E00E94836C90
:10DBC00087E08093BB0C80938E040F900F900F9092
:10DBD0000F900F900F90809178088823F9F0609152
:10DBE000790870917A0880917B0890917C0823E0F5
:10DBF00041E00F94412D9F938F938DE095E09F938B
:10DC00008F93FF92EF920F940B32C7010E94556CD5
:10DC10000F900F900F900F900F900F9080918108B0
:10DC20008823A1F01F928F931F921F9280E095E0AE
:10DC30009F938F93FF92EF920F940B32C7010E9434
:10DC4000556C0FB6F894DEBF0FBECDBF8091820831
:10DC50008823A9F01F928F931F9281E08F9380E019
:10DC600095E09F938F93FF92EF920F940B32C70131
:10DC70000E94556C0FB6F894DEBF0FBECDBF40902A
:10DC8000830850908408609085087090860820E092
:10DC900030E0A901C301B2010F947432811104C0B4
:10DCA0008091F90882FF20C0860121E041E0C30194
:10DCB000B2010F94412D9F938F938091F90882FBBD
:10DCC000882780F91F928F9383EF94E09F938F931F
:10DCD000FF92EF920F940B32C7010E94556C0FB662
:10DCE000F894DEBF0FBECDBF60914E0870914F0813
:10DCF00080915008909151088E010F581F4F23E0DA
:10DD000041E00F94412D782E692E60914A08709160
:10DD10004B0880914C0890914D08860123E041E02A
:10DD20000F94412D6F927F929F938F9382EE94E098
:10DD30009F938F93FF92EF920F940B32C7010E9433
:10DD4000556C6091520870915308809154089091DD
:10DD5000550823E041E00F94412D87ED94E00E94A7
:10DD6000836CDF92CF928DEC94E09F938F93FF9220
:10DD7000EF920F940B32C7010E94556C80915B08A3
:10DD80008F9380915A088F9386EC94E09F938F93A2
:10DD9000FF92EF920F940B32C7010E94556C609175
:10DDA000560870915708809158089091590823E0BF
:10DDB00041E00F94412D9F938F938CEB94E09F93C0
:10DDC0008F93FF92EF920F940B32C7010E94556C14
:10DDD0008CE0E0E6F8E0ADE3B8E001900D928A95C2
:10DDE000E1F78CE0ECE6F8E0A1E3B8E001900D92F9
:10DDF0008A95E1F780E00E94081D81E00E94081DDD
:10DE000082E00E94081D8091F80880932B0881E031
:10DE10008093E4040E9492BF87E898E09F938F93D9
:10DE20008BE091E29F938F93FF92EF920F940B32CE
:10DE30000FB6F894DEBF0FBECDBFC7010E94556C70
:10DE40008091F7088F938091F6088F938091F50861
:10DE50008F938091F4088F93BF92AF929F928F928D
:10DE60008EEA94E09F938F93FF92EF920F940B3280
:10DE7000C7010E94556C0FB6F894DEBF0FBECDBF30
:10DE800008CECF93DF93C091150EC093130981E69E
:10DE9000C89FE0011124C95ED14F8091790C80FFA9
:10DEA00005C00E94F6DBCE010E94CC52CE010E943A
:10DEB000545180E0DF91CF910C94C2563FB7F89453
:10DEC0008091A2069091A306A091A406B091A50608
:10DED00026B5A89B05C02F3F19F00196A11DB11DC5
:10DEE0003FBFBA2FA92F982F8827BC01CD01620F01
:10DEF000711D811D911D42E0660F771F881F991FBC
:10DF00004A95D1F708958BE1E4EEF4E1AFEFB4E187
:10DF100001900D928A95E1F78091C41480628093FC
:10DF2000C4140895CF938091A311C1E08823C9F050
:10DF30008091A4119091A51140919B1150919C1139
:10DF400060919D1170919E11DC01ED91FC91028810
:10DF5000F389E02D2BE93FE01995C82F811104C00A
:10DF6000C0E08C2FCF91089540919F115091A01146
:10DF70006091A1117091A2114115510561057105C2
:10DF8000B9F08091A4119091A511DC01ED91FC9163
:10DF90000288F389E02D2BE93FE01995882301F3EE
:10DFA00010929F111092A0111092A1111092A21123
:10DFB0001092A311D6CF0F931F93CF93DF93CDB7BA
:10DFC000DEB760970FB6F894DEBF0FBECDBF8C01F1
:10DFD000DC01ED91FC910280F381E02DBE016F5FC9
:10DFE0007F4F1995882309F464C08981807CC9F525
:10DFF0006F81637070E0762F6627770F770F8885C3
:10E00000B4E08B9FC0011124682B792B8985829500
:10E01000869586958370682B6F5F7F4F90E080E0D8
:10E020002A852370220F3B8537FB332730F9232BBA
:10E030003E813F70230F3327331F2750310904C01F
:10E04000660F771F881F991F2A95D2F760960FB623
:10E05000F894DEBF0FBECDBFDF91CF911F910F911E
:10E060000895803419F568856695669570E090E0AE
:10E0700080E0CB01772766272A85622B098510E08F
:10E08000102F0027012E000C220B330B602B712B5D
:10E09000822B932B6F5F7F4F8F4F9F4F4AE0660F0E
:10E0A000771F881F991F4A95D1F7D0CF8BE0F801D1
:10E0B000848360E070E0CB01C9CF0895FC018281C8
:10E0C00008954F925F926F927F928F929F92AF923C
:10E0D000BF92EF92FF920F931F93CF93DF93B0E223
:10E0E000A0E06A2F70E0AB014B0F511D559547958D
:10E0F000411117C0E6E9FFE185919491282F822F05
:10E10000DF91CF911F910F91FF90EF90BF90AF9053
:10E110009F908F907F906F905F904F900895B42F55
:10E12000E2CFA41711F0B41303C0E2E1F0E2E4CFB0
:10E130009A0121503109220F331F220F331FF90199
:10E14000EC56F04EE590F490F901E856F04E05914A
:10E1500014918E159F051CF3A42F081719070CF4B2
:10E16000C0CFBC01F901EA56F04EC591D491F90136
:10E17000E656F04EA590B4906E197F09072E000C5C
:10E18000880B990B0F947B322B013C01B5016C1B62
:10E190007D0B072E000C880B990B0F947B329B0193
:10E1A000AC01C301B2010F94DA324B015C01B8013A
:10E1B0006E197F09072E000C880B990B0F947B3288
:10E1C0009B01AC01C501B4010F943E3A4B015C01C7
:10E1D000BE01DD0F880B990B0F947B329B01AC01C4
:10E1E000C501B4010F9444390F94B03A262F972FEC
:10E1F00086CFEF92FF920F931F93E0920D05F0925E
:10E200000E0500930F051093100560931805709389
:10E21000190580931A059FEFFF27621B730B840B70
:10E2200030F4809570956195790B890B99279093BF
:10E23000B206A6E06A9F0092A606512DEE277A9FAD
:10E24000500DE11D8A9FE00D5093A706E093A806AC
:10E25000AFE06A9F0092AA06512DEE277A9F500DDB
:10E26000E11D8A9FE00D5093AB06E093AC06AAE057
:10E270006A9F0092AE06512DEE277A9F500DE11D48
:10E280008A9FE00D5093AF06E093B0061F910F9167
:10E29000FF90EF90089500000000000000008091C2
:10E2A000D00580FF21C089988FEF8093140680915C
:10E2B000D005869580FF1BC08F988FEF8093150641
:10E2C0008091D0058695869580FF14C080910B01C2
:10E2D00082708093090143988FEF809316060000A7
:10E2E0000000000000000895899A81E0DECF8F9A37
:10E2F00081E0E4CF80910B018095827080930901C9
:10E30000439A81E0EACF0F931F93CF93811113C0FB
:10E31000C42F8B010E94F6DB87ED92E10E9492C729
:10E32000C8010E9492C7CC2331F08AE0CF911F919F
:10E330000F910C946AC7CF911F910F9108950F937D
:10E340000091090521E002272AE035E04CE050E089
:10E35000BC018AED94E00E94EBC30F9108950F93E6
:10E360000091090521E002272AE035E044E050E071
:10E37000BC018AED94E00E94EBC30F9108950F93C6
:10E380000091090521E002272AE035E041E050E054
:10E39000BC018AED94E00E94EBC30F9108950F93A6
:10E3A0000091090521E002272AE035E042E050E033
:10E3B000BC018AED94E00E94EBC30F9108950F9386
:10E3C0000091090521E002272AE035E041E050E014
:10E3D000BC018AED94E00E94EBC30F9108950F9366
:10E3E0000091090521E002272AE035E048E050E0ED
:10E3F000BC018AED94E00E94EBC30F9108950F9346
:10E400000091090521E002272AE035E04CE050E0C8
:10E41000BC018AED94E00E94EBC30F9108950F9325
:10E4200001E02AE035E041E050E0BC018AED94E0F3
:10E430000E94EBC30F910895CF93DF93CAE6D2E118
:10E440008A819B810F946C1F9D838C83CFEFD1E1D8
:10E450008A819B810E9461709D838C83A895109214
:10E460009406DF91CF9108951F93CF93DF93182FD8
:10E47000EB010E94F6DB8AE292E20E9492C786E1FB
:10E4800092E2113011F48CE192E20E9492C7BE0137
:10E4900082E292E20E94E8DB8AE0DF91CF911F9155
:10E4A0000C946AC7282F30E0F901E058FC4D949194
:10E4B000F901E658F94C44912C5C394CF90124914E
:10E4C000222309F435C0992311F191509231F8F4C7
:10E4D000E92FF0E08827E059FD488F4F0D943B3934
:10E4E000A172A572827299729D728772A872AE72C1
:10E4F000B272B872BC72C072C672CA728772CE72C1
:10E50000D472D872809180008F7780938000E22F40
:10E51000F0E0EE0FFF1FE050FA4CA591B4918FB7D9
:10E52000F894EC91611148C040954E234C938FBFF5
:10E530000895809180008F7DE8CF80918000877F53
:10E54000E4CF84B58F7784BDE2CF84B58F7DFBCFD8
:10E550008091B0008F778093B000D9CF8091B000C8
:10E560008F7DF9CF809190008F7780939000CFCFEF
:10E57000809190008F7DF9CF80919000877FF5CFBB
:10E580008091A0008F778093A000C1CF8091A000E0
:10E590008F7DF9CF8091A000877FF5CF80912001FA
:10E5A0008F7780932001B3CF809120018F7DF9CFA9
:10E5B00080912001877FF5CF4E2BB8CFCF93DF938B
:10E5C000EC018D810E94C8F060E08B81DF91CF91DA
:10E5D0000C94527261E0FC0183810E9452728FEFB1
:10E5E0000C94BCF0CF93DF93EC016EBDFA01CA012D
:10E5F0009E5F0DB407FEFDCF20812EBD0DB407FE3A
:10E60000FDCF21812EBD3296E817F90791F70DB4A1
:10E6100007FEFDCF8FEF0E94BCF08FEF0E94BCF091
:10E620000E94C1F08E838F71853049F083E18C8325
:10E63000CE010E94EA7280E0DF91CF91089581E0DF
:10E64000FBCF1F93CF93DF93182FEB010E94C5F7E9
:10E65000209739F460E0812FDF91CF911F910C94C6
:10E660005272CF3FD10511F461E0F5CFE12FF0E018
:10E67000E058FC4DE491E150E23108F0B3C0F0E025
:10E680008827EA5BFC488F4F0D943B3958736073C1
:10E6900065736F737973F27383738B7393739D7365
:10E6A000A773B173C073CA73F273D473DE73E87364
:10E6B00084B5806884BDC7BDDF91CF911F91089557
:10E6C00084B5806284BDC8BDF7CF8091800080682A
:10E6D00080938000D0938900C0938800EDCF809113
:10E6E0008000806280938000D0938B00C0938A006A
:10E6F000E3CF80918000886080938000D0938D006C
:10E70000C0938C00D9CF8091B00080688093B00016
:10E71000C093B300D1CF8091B00080628093B000ED
:10E72000C093B400C9CF809190008068809390001E
:10E73000D0939900C0939800BFCF809190008062E1
:10E7400080939000D0939B00C0939A00B5CF8091A6
:10E750009000886080939000D0939D00C0939C00AF
:10E76000ABCF8091A00080688093A0008091A00032
:10E770008F7B8093A000D093A900C093A8009CCF6A
:10E780008091A00080628093A000D093AB00C093E2
:10E79000AA0092CF8091A00088608093A000D093BF
:10E7A000AD00C093AC0088CF809120018068809339
:10E7B0002001D0932901C09328017ECF80912001B0
:10E7C000806280932001D0932B01C0932A0174CFE3
:10E7D00080912001886080932001D0932D01C09307
:10E7E0002C016ACFC038D1050CF03ECF33CF8F92C9
:10E7F0009F92AF92BF92CF92DF92EF92FF926B0106
:10E800007C010E945E6F4B015C01C114D104E104E4
:10E81000F104B9F00E945E6F681979098A099B09B1
:10E82000683E73408105910580F321E0C21AD1084A
:10E83000E108F10888EE880E83E0981EA11CB11C47
:10E84000E4CFFF90EF90DF90CF90BF90AF909F907C
:10E850008F9008952FB7F89460919E0670919F064F
:10E860008091A0069091A1062FBF0895CF92DF92CC
:10E87000EF92FF920E942A746B017C0128E5C20E80
:10E8800022E0D21EE11CF11C0E94C1F08F3F71F00A
:10E890000E942A746C197D098E099F0997FDF4CF97
:10E8A00080E0FF90EF90DF90CF90089581E0F9CF66
:10E8B0000F931F93CF938C010E94DE720E943674D7
:10E8C000C82F882371F08DEF0E94BCF00E9436742F
:10E8D000C82FC8010E94EA728C2FCF911F910F910F
:10E8E000089582E1F8018483F4CF0F931F93CF93AF
:10E8F000DF93EC018B010E94DE720E94367481115D
:10E900000CC085E18C8310E0CE010E94EA72812F59
:10E91000DF91CF911F910F910895A8016CEFCE0167
:10E920000E94F272182F882361F3EECFDF92EF92EC
:10E93000FF920F931F93CF93DF938C01C62FD22F9B
:10E94000F32EE42ED52E0E94DE720E9436748C2F98
:10E9500080640E94BCF08D2D0E94BCF08E2D0E9420
:10E96000BCF08F2D0E94BCF08D2F0E94BCF087E878
:10E97000C11101C085E90E94BCF0CC3011F40E94A5
:10E98000C1F0C0E00E94C1F0F801868387FF04C097
:10E99000CF3F11F0CF5FF6CFDF91CF911F910F9155
:10E9A000FF90EF90DF9008958F929F92AF92BF9269
:10E9B000CF92DF92EF92FF920F931F93CF93DF934B
:10E9C000EC016A017B01590120E030E0A90167E315
:10E9D0000E949674A501980167E1CE010E94967489
:10E9E000811127C08F81833039F089E0CC0CDD1C88
:10E9F000EE1CFF1C8A95D1F7A701960169E1CE01B3
:10EA00000E94967411E0882319F010E087E08C834F
:10EA1000CE010E94EA72812FDF91CF911F910F9159
:10EA2000FF90EF90DF90CF90BF90AF909F908F902E
:10EA3000089589E08C8310E0EBCF0F931F93CF9361
:10EA4000DF93EC0189018F81833039F089E0440F35
:10EA5000551F661F771F8A95D1F79A01AB0168E1B0
:10EA6000CE010E94967481112AC0A8016EEFCE01DA
:10EA70000E94F272182F8823B1F00E943674182F6A
:10EA80008823D1F020E030E0A9016DE0CE010E94A2
:10EA90009674882321F086E18C8310E004C00E94E4
:10EAA000C1F08111F8CFCE010E94EA72812FDF916F
:10EAB000CF911F910F91089587E18C83F4CF86E069
:10EAC000EBCF1F93CF93DF93EC010E94DE7220E027
:10EAD00030E0A9016CE0CE010E94967411E0882319
:10EAE00019F010E083E08C83CE010E94EA72812F3E
:10EAF000DF91CF911F9108951F93CF93DF93EC0186
:10EB00008F81833039F089E0440F551F661F771FCE
:10EB10008A95D1F79A01AB0162E1CE010E94967409
:10EB200011E0882319F010E085E08C83CE010E946B
:10EB3000EA72812FDF91CF911F9108958F929F925A
:10EB4000AF92BF92EF92FF920F931F93CF93DF93F9
:10EB50008C01EB017A010E942A744B015C012CE2CA
:10EB6000820E21E0921EA11CB11C0E94C1F0F8018E
:10EB700086838F3F69F40E942A74681979098A098B
:10EB80009B0997FDF2CF81E1F8018483C0E021C0A9
:10EB90008E3F71F5F1E0EF1AF1088FEF8EBDFE01A7
:10EBA0002FEF0DB407FEFDCF8EB581932EBDCF01A3
:10EBB0008C1B9D0B8E159F05A0F30DB407FEFDCF9A
:10EBC0008EB5CE0DDF1D88830E94C1F00E94C1F07A
:10EBD000C1E0C8010E94EA728C2FDF91CF911F9192
:10EBE0000F91FF90EF90BF90AF909F908F900895FE
:10EBF0008FE0CACF0F931F93CF93DF93EC018B016C
:10EC00000E94DE7240E052E0B801CE01DF91CF9168
:10EC10001F910F910C949E750F931F93CF93DF93C9
:10EC2000EC0189018F81833039F089E0440F551F51
:10EC3000661F771F8A95D1F79A01AB0161E1CE017A
:10EC40000E94967481110AC040E052E0B801CE01E2
:10EC5000DF91CF911F910F910C949E7584E08C836E
:10EC6000CE010E94EA7280E0DF91CF911F910F9157
:10EC700008950F931F93CF93DF93EC018B0120E056
:10EC800030E0A90169E00E94967481110AC040E158
:10EC900050E0B801CE01DF91CF911F910F910C94FC
:10ECA0009E7580E18C83CE010E94EA7280E0DF9144
:10ECB000CF911F910F9108958F929F92AF92BF9223
:10ECC000CF92DF92EF92FF920F931F93CF93DF9338
:10ECD000EC01162F1F821C824B830E942A746B0149
:10ECE0007C0120EDC20E27E0D21EE11CF11CA8958C
:10ECF00061E08B810E9452728B810E94C5F7209A3D
:10ED0000289A219A2398229A81E00E94C8F085E0EF
:10ED10008D830E94C8F00AE08FEF0E94BCF0015082
:10ED2000D9F7A89520E030E0A90160E0CE010E946B
:10ED300096748E83813081F00E942A746C197D094B
:10ED40008E099F0997FDEECF81E08C83CE010E9452
:10ED5000EA721A8280E06AC0A8952AEA31E040E0AF
:10ED600050E068E0CE010E949674853041F581E064
:10ED70008F83A8958F81812C912C5401823029F4A6
:10ED8000812C912CA12C80E4B82E20E030E0A90148
:10ED900067E3CE010E949674A501940169E2CE0159
:10EDA0000E9496748E838823F1F00E942A746C1955
:10EDB0007D098E099F0997FDE8CF8AE0C6CF04E060
:10EDC0000E94C1F08E830150D9F78A3A11F482E093
:10EDD000CFCF0E942A746C197D098E099F0997FD77
:10EDE000BCCF82E0B2CF8F818230C1F420E030E02E
:10EDF000A9016AE3CE010E949674882311F088E08D
:10EE0000A4CF0E94C1F0807C803C11F483E08F830A
:10EE10000E94C1F00E94C1F00E94C1F0CE010E9488
:10EE2000EA7281E08A83173070F41D83DF91CF91FD
:10EE30001F910F91FF90EF90DF90CF90BF90AF9018
:10EE40009F908F90089588E18C8384CF1F920F92BA
:10EE50000FB60F9211242F933F938F939F93AF93ED
:10EE6000BF9380919E0690919F06A091A006B091BD
:10EE7000A10630919D0623E0230F2D3758F501960A
:10EE8000A11DB11D20939D0680939E0690939F0621
:10EE9000A093A006B093A1068091A2069091A3062C
:10EEA000A091A406B091A5060196A11DB11D809365
:10EEB000A2069093A306A093A406B093A506BF91C3
:10EEC000AF919F918F913F912F910F900FBE0F9017
:10EED0001F90189526E8230F0296A11DB11DD2CFD1
:10EEE000CF92DF92EF92FF920F931F93CF93DF9316
:10EEF000CDB7DEB7A0970FB6F894DEBF0FBECDBF7B
:10EF0000442309F445C0611571058105910579F126
:10EF100000E0C42ED12CF12CE12CA70196010F9416
:10EF2000B83811E0100FE1E0F0E0EC0FFD1FE00F4A
:10EF3000F11D07FDFA956083B901CA01012F611522
:10EF400071058105910549F7115010F1E1E0F0E0FC
:10EF5000EC0FFD1FE10FF11D17FDFA95908187E37E
:10EF60009A3008F480E3890F0E946AC7EDCF80E3EE
:10EF7000A0960FB6F894DEBF0FBECDBFDF91CF9144
:10EF80001F910F91FF90EF90DF90CF900C946AC784
:10EF9000A0960FB6F894DEBF0FBECDBFDF91CF9124
:10EFA0001F910F91FF90EF90DF90CF900895809187
:10EFB000B9148823C1F081508093B914E4EEF4E1D0
:10EFC000882351F08150990B2BE1289FF001299F54
:10EFD000F00D1124E65EFA4E8BE1AFEFB4E1019043
:10EFE0000D928A95E1F78091B914811105C0909135
:10EFF000C41490629093C4140895CF92DF92EF925C
:10F00000FF928091C41482FF29C0C090C014D09098
:10F01000C114E090C214F090C31481EE91E20E94FA
:10F0200092C74AE0C701B6010E9470778FE20E9442
:10F030006AC76091BC147091BD148091BE14909108
:10F04000BF144AE00E9470778DE00E946AC78AE090
:10F05000FF90EF90DF90CF900C946AC783EF91E21E
:10F06000FF90EF90DF90CF900C9492C7BC0185E1A8
:10F0700091E20E94E8DB82E191E20C9492C78091D8
:10F08000C41483FF03C084608093C4140895CF9296
:10F09000DF92EF92FF920F931F93CF93DF93CDB741
:10F0A000DEB7EDB6FEB6DC010D900020E9F79D015C
:10F0B000281B390B285F3F4FEDB7FEB7E21BF30B60
:10F0C0000FB6F894FEBF0FBEEDBF0DB71EB70F5FB2
:10F0D0001F4F9F938F938BE091E29F938F931F938A
:10F0E0000F930F940B326801F4E0CF0ED11C0F90F8
:10F0F0000F900F900F900F900F90D6018D916D0192
:10F10000882349F0082E000C990B0F94563CF60109
:10F1100031978083F2CF66E071E2C8010F94A43189
:10F120004FE350E0B80182ED95E00F94B23C0FB68A
:10F13000F894FEBE0FBEEDBEDF91CF911F910F91EF
:10F14000FF90EF90DF90CF900895FC01938591FDA3
:10F1500013C0987121E0903109F020E08091C4142F
:10F1600020FB84F98093C414903141F0808587346A
:10F1700019F481858E3711F480E0089581E00895B7
:10F18000FC0120E03EE2DB014D91BD01403249F03F
:10F19000283011F430833196DB0111974C91408374
:10F1A00031962F5F2B3079F710820895EF92FF92FE
:10F1B0000F931F93CF93DF93CDB7DEB7A0970FB612
:10F1C000F894DEBF0FBECDBF7C018B01BE016F5F27
:10F1D0007F4FC7010E9482F11816A4F4CE01019658
:10F1E0000E94A578882391F3BE016F5F7F4F85E170
:10F1F00092E10E94C07865E172E1C8010F94743C0D
:10F20000892B21F7A0960FB6F894DEBF0FBECDBFB5
:10F21000DF91CF911F910F91FF90EF900895CF92C2
:10F22000DF92EF92FF92CF936B017C01C42F80910C
:10F230009B1190919C11A0919D11B0919E118C15E4
:10F240009D05AE05BF0529F10E94926F811108C08E
:10F25000C0E08C2FCF91FF90EF90DF90CF9008957A
:10F260008091A4119091A511DC01ED91FC91008891
:10F27000F189E02D2BE93FE0B701A601199588231C
:10F2800039F3C0929B11D0929C11E0929D11F092A3
:10F290009E11CC2321F081E08093A311DACFC1E04D
:10F2A000D8CF4F925F926F927F928F929F92AF9240
:10F2B000BF92CF92DF92EF92FF920F931F93CF9363
:10F2C000DF93EC01423051056105710590F480E057
:10F2D000DF91CF911F910F91FF90EF90DF90CF9032
:10F2E000BF90AF909F908F907F906F905F904F9066
:10F2F000089589859A85AB85BC850196A11DB11DB0
:10F3000084179507A607B70710F38F898031C9F5D1
:10F31000852E962EA72EBB248B899C89AD89BE890C
:10F32000880E991EAA1EBB1E280139016A017B01A5
:10F3300041E0C501B4010E940F79882341F29F8901
:10F34000903181F5DD24EE24FF24F601EE0FFF1F3E
:10F35000E556F04F118300839A89923008F4B8CFB4
:10F360004D815E816F817885840E951EA61EB71E25
:10F3700080929F119092A011A092A111B092A2111F
:10F38000A7CF803209F0A3CF8B899C89AD89BE8934
:10F390004A015B01E7E0B694A79497948794EA95B5
:10F3A000D1F7BECFE894C7F8DD24EE24FF24F601A0
:10F3B000EE0FFF1FEE0FFF1FE556F04F4082518208
:10F3C00062827382C9CFCF92DF92EF92FF920F9346
:10F3D0001F93CF93DF93FC0181859285A385B4852C
:10F3E0000196A11DB11D84179507A607B70750F414
:10F3F00080E0DF91CF911F910F91FF90EF90DF9010
:10F40000CF90089587898031A9F5BB27A72F962F24
:10F41000852FC388D488E588F6888C0D9D1DAE1D88
:10F42000BF1DE9016A017B018F0140919B11509141
:10F430009C1160919D1170919E1184179507A607EC
:10F44000B70749F5F8018789803169F5B701A60149
:10F45000552766277727440F551F4556504FFA0109
:10F4600080819181B0E0A0E088839983AA83BB83E7
:10F4700081E0BFCF803209F0BBCFC388D488E58854
:10F48000F688DB01CA01C7E0B695A79597958795E1
:10F49000CA95D1F7C2CF40E0BC01CD010E940F79DF
:10F4A0008111D0CFA5CFB701A6014F775527662789
:10F4B0007727440F551F440F551F4556504FFA01EB
:10F4C00080819181A281B381BF70CECF4F925F9234
:10F4D0006F927F92AF92BF92CF92DF92EF92FF92A4
:10F4E0000F931F93CF93DF9300D01F92CDB7DEB75A
:10F4F0008C0149835A836B837C835901C12CD12CA5
:10F500007601412C82E0582E612C712C49815A8160
:10F510006B817C819E012F5F3F4FC8010E94E37980
:10F52000882319F1F8018585A301920104C0220FF7
:10F53000331F441F551F8A95D2F7DA01C901C80E3F
:10F54000D91EEA1EFB1E49815A816B817C81878905
:10F550008031F1F481E0483F5F4F61057105B0F201
:10F56000F501C082D182E282F3820F900F900F905A
:10F570000F90DF91CF911F910F91FF90EF90DF904F
:10F58000CF90BF90AF907F906F905F904F90089515
:10F5900081E0483F5F4F6F4F7F4008F4B7CFE0CF27
:10F5A0000F931F93CF93DF93FC012381222331F02C
:10F5B00080E0DF91CF911F910F9108958B01EC01B5
:10F5C000FB018789803139F582E08B831D8A1E8A91
:10F5D0001F8A188E808D918DB0E0A0E025E0880F05
:10F5E000991FAA1FBB1F2A95D1F7898B9A8BAB8BCA
:10F5F000BC8B1A8F098F81E08983188619861A8639
:10F600001B861C821D821E821F82188A1C861D86F4
:10F610001E861F86CECF803259F683E08B83428DC3
:10F62000538D648D758D4D8B5E8B6F8B788F9E01A6
:10F630002F5E3F4FC8010E94667A8111DACFB8CFA2
:10F640003F924F925F926F927F928F929F92AF9272
:10F65000BF92CF92DF92EF92FF920F931F93CF93BF
:10F66000DF93CDB7DEB72C970FB6F894DEBF0FBE91
:10F67000CDBF5C01DC0159968D909C90F401818591
:10F680009285A385B4859C01AD012F5F3F4F4F4FFD
:10F690005F4F29873A874B875C87D50114964D9039
:10F6A0005D906D907C901797411451046104710432
:10F6B00009F459C0BFEF4B1A5B0A6B0A7B0A312C65
:10F6C000730162011D821E821F821886F4018185EA
:10F6D0009285A385B4852D813E814F815885281759
:10F6E00039074A075B0708F056C089859A85AB85BC
:10F6F000BC858C159D05AE05BF0550F482E0C82E73
:10F70000D12CE12CF12C92E0492E512C612C712C42
:10F710009E012F5F3F4FB701A601C4010E94E3790C
:10F720008823C9F189819A81AB81BC81892B8A2B7D
:10F730008B2B01F1260137019FEF491A590A690AFB
:10F74000790A2D813E814F8158852F5F3F4F4F4F62
:10F750005F4F2D833E834F8358873FEFC31AD30AF1
:10F76000E30AF30AB3CF4080518062807380332470
:10F770003394A6CFC414D504E604F70411F70FEFB1
:10F780001FEF2FEF3FE0B701A601C4010E9451799E
:10F79000782E81111AC0712C872D2C960FB6F894F3
:10F7A000DEBF0FBECDBFDF91CF911F910F91FF90B4
:10F7B000EF90DF90CF90BF90AF909F908F907F9011
:10F7C0006F905F904F903F900895F501448155816F
:10F7D00066817781411551056105710539F0970101
:10F7E0008601C4010E9451798823A9F2D50114969B
:10F7F000CD92DD92ED92FC921797332051F0D70114
:10F80000C6010196A11DB11DF40180839183A283DD
:10F81000B383F50185899689A789B08D892B8A2BB9
:10F820008B2B09F0B9CFC58AD68AE78AF08E818101
:10F8300080688183B1CFCF93DF93EC01462F417075
:10F840006C857D858E859F850E940F79882351F078
:10F85000888920E2829FC00111248556904FDF9154
:10F86000CF91089590E080E0FACFCF93DF93EC0141
:10F870008991882319F00E946AC7FACFDF91CF914E
:10F880000895CF93DF93EC018B81882349F189811F
:10F8900087FF22C061E0CE010E941B7CFC01892B06
:10F8A000F9F08081853EE1F08B81823040F48989D6
:10F8B0009A89AB89BC89848F958FA68FB78F8D89E4
:10F8C0009E89938F828F8D899E89AF89B88DB58BE4
:10F8D000A48B89818F778983DF91CF910C94926F6C
:10F8E00081E0888380E0DF91CF9108958F929F928D
:10F8F000AF92BF92CF92DF92EF92FF920F931F933E
:10F90000CF93DF93EC018B8181110EC080E0DF91FA
:10F91000CF911F910F91FF90EF90DF90CF90BF900C
:10F92000AF909F908F90089509891A892B893C89FF
:10F93000041715072607370748F34A015B01823091
:10F9400031F488869986AA86BB8681E0E0CF81144F
:10F950009104A104B10449F4188619861A861B86FD
:10F960001C821D821E821F82F0CF088519852A8580
:10F970003B85E98DFA8D858590E00996B901A8014E
:10F980004150510961097109082E04C076956795A7
:10F99000579547950A94D2F775016401E1E0CE1AB4
:10F9A000D108E108F10804C0F694E794D794C7940D
:10F9B0008A95D2F7C416D506E606F70620F0012B85
:10F9C000022B032B11F58D899E89AF89B88D8C830D
:10F9D0009D83AE83BF838E010C5F1F4FC114D10482
:10F9E000E104F10409F4ADCF4C815D816E817F812A
:10F9F0009801898D9A8D0E94E37991E0C91AD10806
:10FA0000E108F1088111EACF81CFC41AD50AE60ACC
:10FA1000F70AE1CF2F923F924F925F926F927F92BF
:10FA20008F929F92AF92BF92CF92DF92EF92FF920E
:10FA30000F931F93CF93DF9300D01F92CDB7DEB704
:10FA40008C014B011A01DC0113968C9113978130C4
:10FA500009F0CFC011968C9181FFCBC082FDB5C05B
:10FA60006101D80118964D915D916D917C911B9724
:10FA7000C114D10409F41BC159968D919C915A97D8
:10FA8000FC0174802FEF270D2A013B0139E07694A9
:10FA90006794579447943A95D1F7722E74207A015F
:10FAA000F1E0FF22711020C0E114F104E9F4149692
:10FAB0004D915D916D917C911797411551056105AF
:10FAC000710509F09CC055968D919D910D90BC914A
:10FAD000A02D0097A105B10509F0AAC0C8010E9498
:10FAE000207B882309F485C0A12C82E0B82EAE18B3
:10FAF000BF08CA14DB0408F45601D80159964D9189
:10FB00005C915A9714968D919D910D90BC91A02D6A
:10FB10000297A109B109FA01258504C0880F991F30
:10FB2000AA1FBB1F2A95D2F7468557856089718920
:10FB3000840F951FA61FB71F9C01AD01270D311D16
:10FB4000411D511D29013A01A11432E0B30609F00B
:10FB50007DC080919B1190919C11A0919D11B091BD
:10FB60009E11481659066A067B0669F41092A31185
:10FB70008FEF9FEFDC0180939B1190939C11A093DA
:10FB80009D11B0939E118091A4119091A511DC015B
:10FB9000ED91FC910288F389E02D9401B301A2015B
:10FBA0001995882331F1F80180859185A285B38567
:10FBB0008A0D9B1DA11DB11D80879187A287B387E8
:10FBC0008A0C9B1CCA18DB084CCFF801418952896A
:10FBD0006389748980859185A285B3854817590703
:10FBE0006A077B0709F43CCFC8010E94767C81112B
:10FBF00037CF81E0D8018C938FEF9FEF6EC09E01CD
:10FC00002F5F3F4F0E94E379882399F389819A817E
:10FC1000AB81BC81F801218D328DF901278920311A
:10FC200069F4883FFFEF9F07A105B10508F056CFA3
:10FC3000F80184839583A683B78356CF883F2FEF3F
:10FC40009207A2072FE0B20798F348CFE114F1041E
:10FC500031F5F801408551856285738581899289E6
:10FC6000A389B489481759076A077B07C0F00E9427
:10FC7000926F882309F4BDCF81E08093A311409255
:10FC80009B1150929C1160929D1170929E11A50142
:10FC9000B401C7018556904F0F946B3C84CF41E06F
:10FCA000C301B2010E940F798111F1CFA2CFF801F7
:10FCB00081899289A389B48984179507A607B70714
:10FCC00038F48181418B528B638B748B8068818384
:10FCD000F801818183FD18C0C1010F900F900F9032
:10FCE0000F90DF91CF911F910F91FF90EF90DF90D8
:10FCF000CF90BF90AF909F908F907F906F905F90CC
:10FD00004F903F902F900895C8010E94417C81112F
:10FD1000E3CF6FCF2F923F924F925F926F927F927D
:10FD20008F929F92AF92BF92CF92DF92EF92FF920B
:10FD30000F931F93CF93DF93EC014B017A018B81DB
:10FD4000811115C08FEF9FEFDF91CF911F910F9120
:10FD5000FF90EF90DF90CF90BF90AF909F908F90EB
:10FD60007F906F905F904F903F902F900895898182
:10FD700080FFE8CF89899A89AB89BC8948855985F4
:10FD80006A857B85841B950BA60BB70BA70170E0DA
:10FD900060E084179507A607B70708F47C016701A0
:10FDA0001E0124E0220E311CC114D10409F4A9C0A3
:10FDB000488559856A857B855A0181E0B822898DFD
:10FDC0009A8D2A013B0129E07694679457944794D1
:10FDD0002A95D1F72B81FC01223081F5628D738D3C
:10FDE000848D958D640D751D861D971D00E012E0B4
:10FDF0000A191B09C016D10608F486010115E2E0B4
:10FE00001E0771F440909B1150909C1160909D11C1
:10FE100070909E11641575058605970509F04EC012
:10FE200040E00E940F79882309F48CCFB501655614
:10FE3000704FA801C4010F946B3C52C01481115043
:10FE40001421A114B10471F411110CC0452B462BDF
:10FE5000472B51F58D899E89AF89B88D8C839D8301
:10FE6000AE83BF83E98DFA8D4C805D806E807F808C
:10FE700022E0421A510861087108858504C0440CCB
:10FE8000551C661C771C8A95D2F786859785A089B4
:10FE9000B189480E591E6A1E7B1EC301B201610F53
:10FEA000711D811D911DA2CF4C815D816E817F816D
:10FEB00091010E94E3798111D5CF44CFA091A41183
:10FEC000B091A511ED91FC9111970088F189E02D79
:10FED0009401AB01BC01CD011995882309F432CFFF
:10FEE000800E911E88859985AA85BB85800F911FFC
:10FEF000A11DB11D88879987AA87BB87C01AD10A1F
:10FF000053CFC70121CFCF93DF93EB01FC012381B6
:10FF1000211104C080E0DF91CF910895225022305A
:10FF200028F48FE28883198281E0F5CF60E00E9497
:10FF30001B7C009779F3DC0160E080E09EE22D916C
:10FF4000203299F0883031F49E01260F311DF901DD
:10FF500090836F5F9E01260F311DAD014150510905
:10FF6000FA014081F90140836F5F8F5F8B3039F771
:10FF7000FE01E60FF11D1082D7CFCF93DF93EC0186
:10FF8000CB01E881F981608171810E94837F2881A2
:10FF90003981D901ED91FC91AA81BB818C9190812D
:10FFA000992359F08936C8F4CF010196F90191835C
:10FFB00080838C918F5F8C93EACF893670F48FE2C7
:10FFC0008083E881F981808191810196918380838A
:10FFD000EA81FB8180818F5F8083DF91CF910895DB
:10FFE0000F931F93CF93DF9300D000D01F92CDB714
:10FFF000DEB79C012F5F3F4F3F832E832FE2FC0132
:020000021000EC
:10000000208381E08D83CE0106969A8389830197B0
:100010009C838B8310E00BE18091B914181758F47E
:10002000109FB0011124665E7A4ECE0101960E94A7
:10003000BD7F1F5FF1CF8D818B3558F468E276E18B
:10004000CE0101960E94BD7F8E819F8101979F8383
:100050008E83EE81FF81108227960FB6F894DEBF63
:100060000FBECDBFDF91CF911F910F910895CF9318
:10007000DF93EC010E94417C1B82DF91CF910895B8
:100080001092A6118091C4148F7B8B7F8093C4142F
:100090000E94C1C3882321F088E296E10C94378046
:1000A00008958091C41482FF0AC080648093C414B0
:1000B0008091C414877F80628093C41408950E9445
:1000C0004080F6CFCF93DF938091C414877F8093D5
:1000D000C4148091E714882321F084EE94E10E94F7
:1000E00037808091C5149091C614DC01ED91FC918C
:1000F0000190F081E02D45E360E0199581110EC07B
:100100000E94F6DB8AEF90E20E9492C78091C414AD
:1001100083FF30C0DF91CF910C94836FC091C514E1
:10012000D091C61461E0CE010E945FF681110BC030
:1001300060E0CE010E945FF6811105C00E94F2DBF3
:1001400086EE90E2E1CF6FE772E184EE94E10E94E7
:10015000D07A811105C00E94F2DB85ED90E2D4CF08
:100160008091C41488608093C4140E94F6DB89ECEB
:1001700090E2CACF80911306882339F06FEF8CEBA1
:1001800090E2DF91CF910C94EC3CDF91CF910895F8
:1001900040E050E0BA010C94767C0F931F93CF930C
:1001A000DF93CDB7DEB7EB970FB6F894DEBF0FBE87
:1001B000CDBF8091C41400E010E083FF23C08FEF17
:1001C00094E10E94C8808BE1EFEFF4E1DE019196AB
:1001D00001900D928A95E1F710E000E0BE016F5F9B
:1001E0007F4FCE0181960E9482F118163CF4CE0119
:1001F00001960E94A578080F111DF0CFCE018196BF
:100200000E94B2BFC801EB960FB6F894DEBF0FBED6
:10021000CDBFDF91CF911F910F9108950F931F9341
:10022000CF93DF93CDB7DEB76B970FB6F894DEBFF1
:100230000FBECDBF8C018FEF94E10E94C8808BE18F
:10024000EFEFF4E1DE01119601900D928A95E1F74E
:10025000B801CE0101960E94D678CE0101960E9487
:10026000B2BF6B960FB6F894DEBF0FBECDBFDF9165
:10027000CF911F910F9108954F925F926F927F924D
:10028000AF92BF92CF92DF92EF92FF920F931F93A4
:10029000CF93DF931F92CDB7DEB78C017B015A015C
:1002A000C22EDB0159968D919C91F801928F818F1E
:1002B000CB010E94C880712CF70180859185A285B1
:1002C000B385418952896389748984179507A60784
:1002D000B70708F052C055E0B695A7959795879552
:1002E0005A95D1F7F82FFF70DF2ED70113968C9116
:1002F000823010F480E0DBC041E050E0BE016F5F6F
:100300007F4FC7010E948A7E0197A1F7F701808580
:100310009185A285B3854F96A11DB11D80879187D8
:10032000A287B387F0E2DF9EB00111246556704FBB
:1003300061157105F9F2DB018C91882341F0853E4E
:1003400009F04CC0772029F077247394B5CF711051
:100350000EC080919B1190919C11A0919D11B09124
:100360009E11F80184879587A687B787D08ADB011D
:100370008C918111E9CF772473948C2D827482340F
:1003800009F0B8CF772009F4A2C0F801D08861E065
:10039000C8010E941B7C009709F4ACCF20E2DC016D
:1003A0001D922A95E9F72BE0F501DC0101900D92F1
:1003B0002A95E1F721E238E2FC01318B208B40E005
:1003C00058E057874687338B228B318F208F578B8E
:1003D000468B0E94926F811109C08CCF4BE050E098
:1003E000C5010F945E3C892B09F066CFF0E2DF9ED9
:1003F000D00111249D012556304FF901838581716B
:1004000021F08C2D827109F001C1F801818D928D4E
:1004100040919B1150919C1160919D1170919E1182
:100420004487558766877787D08AFD01E556F04F68
:1004300044885588712C612C320155244424D801FC
:1004400055964D925D926D927C925897428D538D48
:1004500070E060E0442955296629772955964D9327
:100460005D936D937C935897D9011B962C912871BD
:1004700009F0BEC0848D958DA68DB78DF801818B56
:10048000928BA38BB48B81E083838C2D8F70F801CA
:100490008183148215821682178210861186128635
:1004A000138681E0C4FE03C0C8010E94A7F20F902A
:1004B000DF91CF911F910F91FF90EF90DF90CF9040
:1004C000BF90AF907F906F905F904F900895D7014D
:1004D00013968C911397823009F40CCF51968D911D
:1004E0009D910D90BC91A02D803E9F4FAF41B105D5
:1004F00008F000CFC7010E94207B882309F4FACEC0
:100500000E94926F882309F4F5CED7015996ED9198
:10051000FC915A9714964D905D906D907C90179732
:10052000B2E04B1A510861087108858504C0440C7B
:10053000551C661C771C8A95D2F786859785A089FD
:10054000B189480E591E6A1E7B1E81E08093A3115B
:1005500040929B1150929C1160929D1170929E113D
:10056000EBE9FFE080E092E0DF019C011D92215069
:100570003040E1F7DD24D394D7015996ED91FC91F9
:100580008481D816C0F48091A4119091A511DC014A
:10059000ED91FC910288F389E02D2BE93FE0B30156
:1005A000A2014D0D511D611D711D1995882309F47E
:1005B000A1CED394E1CF258580E092E0A0E0B0E029
:1005C00004C0880F991FAA1FBB1F2A95D2F7F701F5
:1005D0004189528963897489840F951FA61FB71FAB
:1005E000818B928BA38BB48B8BE99FE0D12CD6CEE1
:1005F000203161F498012F5E3F4F0E94667A882374
:1006000029F084E0D80113968C933FCFD80113963C
:100610001C9270CE2F923F924F925F926F927F9278
:100620008F929F92AF92BF92CF92DF92EF92FF9202
:100630000F931F93CF93DF93CDB7DEB7C354D10988
:100640000FB6F894DEBF0FBECDBF4C015B016A014F
:10065000222E19821C821C8E1F8E6115710521F5B8
:1006600010E0CE014C960E94B2BFCE0101960E94CE
:10067000B2BF812FCD5BDF4F0FB6F894DEBF0FBE48
:10068000CDBFDF91CF911F910F91FF90EF90DF9041
:10069000CF90BF90AF909F908F907F906F905F9022
:1006A0004F903F902F900895FC0183818111D8CF06
:1006B000FA0180818F32A1F18B01CE0101967C017C
:1006C0003C0180E2382E2E019CE1490E511C2396FC
:1006D000EFAE23972496FFAE249722963FAE229743
:1006E00021963FAE21973FAE3EAE3DAE3CAE3BAE17
:1006F0003AAE39AE38AE3FAA960190E047E0D90154
:100700008D91882309F447C08F3209F444C08E329A
:1007100009F54A3009F4A4CF98E04AE09D01EFCFF3
:10072000FB01838182508B01823060F0618D728D7C
:10073000CE014C960E94D07A8E01045E1F4F882312
:1007400009F48ECFC6016C010196F60120812F328B
:10075000D1F3B3CFE8E9F0E22491222321F03196DE
:100760008213FACF7DCF491708F47ACF813208F48B
:1007700077CF8F3709F474CF3FE9380F3A3108F457
:1007800020EEE7E3F0E0EC0FFD1FE90FF11D820F13
:1007900080839F5FC3CF8FA9803209F461CF690145
:1007A000F90180812F5F3F4F8F32C9F3882301F118
:1007B00021E0AE01495C5F4FB801C7010E943C8156
:1007C000882309F44DCF0A151B0519F0C8010E94B2
:1007D0003780942D852D6E147F0431F023969FADC4
:1007E000239724968FAD24978701E92EF82E75CF95
:1007F000222DAE01495C5F4FB801C4010E943C81CB
:10080000182F2FCF1F93CF93DF93CDB7DEB76D9700
:100810000FB6F894DEBF0FBECDBF1D8E1C8EAC018F
:10082000BE01645E7F4F80E00E945CF510E000979F
:10083000A9F019821C826C8D7D8D21E0AC01CE0166
:1008400001960E940A83182F882321F0CE01019679
:100850000E943780CE0101960E94B2BF812F6D9613
:100860000FB6F894DEBF0FBECDBFDF91CF911F91C1
:100870000895EF92FF921F93CF93DF9300D000D0A3
:1008800000D01F92CDB7DEB78091C41483FF0E94C1
:1008900062808091C41483FF3CC00E94A0BF81117C
:1008A00038C08091BA1490E08F969F938F938FE217
:1008B00092E29F938F93CE0101967C019F938F9339
:1008C0000F940B328091C4140F900F900F900F90E3
:1008D0000F900F9083FF1DC0C7010E940284182F44
:1008E0008823B9F00E94836FC7010E9447788091E6
:1008F000BA148F5F8093BA14812F2A960FB6F8949A
:10090000DEBF0FBECDBFDF91CF911F91FF90EF9063
:1009100008951092BA1410E0EFCF81E08093BA14DA
:100920000C943984CF939091C41493FF23C0909179
:10093000CC1491111FC02AE5811121E0C82F4AEF84
:1009400052E064EE74E189EC94E10E940A83811123
:1009500005C08AEF92E0CF910C943678C1110AC09D
:100960006AEF72E084E092E20E94E8DB8AE0CF91D5
:100970000C946AC7CF910895CF9321E04AEF52E0DB
:1009800064EE74E189EC94E10E940A83C82F882305
:1009900021F089EC94E10E9437808C2FCF9108954B
:1009A000FF920F931F93CF93DF93CDB7DEB76D9771
:1009B0000FB6F894DEBF0FBECDBF2091C41423FF45
:1009C0002DC0AC01BE01645E7F4F80E00E945CF5EB
:1009D0008C01009719F16C8D7D8D19821C8222E0AB
:1009E000AC01CE0101960E940A83811123C0F12C33
:1009F000CE0101960E94B2BFB801FF2081F183EDC4
:100A000091E20E94E8DB8AE00E946AC71092C0145B
:100A10001092C1141092C2141092C3146D960FB6A6
:100A2000F894DEBF0FBECDBFDF91CF911F910F9124
:100A3000FF900895CE0101960E94A7F28823B9F293
:100A400061E0CE0101960E941B7C009781F225EEA9
:100A5000FC0120831C820E94926FF82EC9CF8BEB81
:100A600091E20E94E8DB88EB91E20E9492C7D6CF28
:100A70000E94BC84882331F00E948ABF8AEF92E0F2
:100A80000C94D08408950F931F93CF93DF931F92FC
:100A90001F92CDB7DEB72091C41423FF32C08C0162
:100AA000BC0182E00E9434721092BB140E9440800C
:100AB000A801BE016F5F7F4F80E00E945CF58C0152
:100AC0000097F9F069817A8126E5AC0188E296E128
:100AD0000E940A838823E1F08091C414816080938E
:100AE000C414C8010E940E811092B814B80184E0A9
:100AF00092E20E94E8DB8AE00E946AC7C8010E9475
:100B0000F5F40F900F90DF91CF911F910F91089501
:100B1000C8010E943678F5CFCF92DF92EF92FF9214
:100B20000F931F93CF93DF931F921F92CDB7DEB722
:100B30002091C41423FF62C08C01613009F470C09D
:100B400008F467C0623009F4CFC00E944080A80159
:100B5000BE016F5F7F4F81E00E945CF58C010097C2
:100B600009F44CC069817A8121E0AC0188E296E108
:100B70000E940A83882309F4BEC08091391690919F
:100B80003A16A0913B16B0913C168093BC149093FA
:100B9000BD14A093BE14B093BF141092C014109251
:100BA000C1141092C2141092C314B80180E491E2EF
:100BB0000E94E8DBC090BC14D090BD14E090BE143D
:100BC000F090BF1488E391E20E9492C74AE0C70107
:100BD000B6010E9470778AE00E946AC789E291E2BA
:100BE0000E9492C7C8010E940E8180912212882320
:100BF00011F002E212E1C8010E94F5F40F900F908B
:100C0000DF91CF911F910F91FF90EF90DF90CF90E8
:100C10000895BC0182E00E9434721092BB1495CFFB
:100C20000E94C1C3811105C0B80181E00E943472E5
:100C30008CCF8091BB14882391F00E94F2DB61E09D
:100C400070E089E991E20E9459CA8AE00E946AC76D
:100C500040E070E060E088E891E20E94D0DE8BE442
:100C600095E00E94F07FE091BB1484E0E89FF001E2
:100C70001124E95BFA4F8091C0149091C114A091A6
:100C8000C214B091C31480839183A283B3830E9462
:100C9000F6DBB8018FE691E20E94E8DB6091BB14BD
:100CA00089E6689FB0011124655B7A4F84E691E282
:100CB0000E94E8DBC090C014D090C114E090C21430
:100CC000F090C3148EE591E20E9492C74AE0C701FA
:100CD000B6010E9470778AE00E946AC78091BB14B7
:100CE0008F5F8093BB1431CF0E94F6DB8EE491E2DC
:100CF0000E9492C72ACFC8010E9436787FCF6F9298
:100D00007F928F929F92AF92BF92CF92DF92EF929B
:100D1000FF920F931F93CF93DF93CDB7DEB7C356E8
:100D2000D1090FB6F894DEBF0FBECDBF5C018B01B9
:100D30006DB67EB67E0187E5E80EF11CBE016F5FE1
:100D40007F4FC5010E9482F118160CF0A4C08C855B
:100D50008871803109F076C08DB69EB6BE016F5F96
:100D60007F4FC7010E94C0780115110509F466C0C4
:100D7000F8018081882309F461C001900020E9F71F
:100D80003197CF01801B910B20E0F70101900020EB
:100D9000E9F73197EE19FF09E80FF91F32968DB781
:100DA0009EB78E1B9F0B0FB6F8949EBF0FBE8DBFD4
:100DB000EDB7FEB731966F01B801222311F061E063
:100DC00074E0C6010F949D3CB701C6010F94873CA7
:100DD00061E074E0C6010F94873C19A21CA221E0D7
:100DE000A701B501CE0181960E940A8381110AC034
:100DF0000E94F6DBB70188EA90E20E94E8DB8AE015
:100E00000E946AC78BE1FE01B196DE01DC9601907B
:100E10000D928A95E1F7B601CE01CC960E947F86AD
:100E2000CE01CC960E94B2BFCE0181960E94B2BF85
:100E30000FB6F8949EBE0FBE8DBE80CF21E081E03C
:100E400090E0A3CFCE0101960E94A578882309F4F3
:100E500075CFBE016F5F7F4F85E192E10E94C07840
:100E60000115110519F0C8010E94357C85E192E158
:100E70000E94357C80E20E946AC76D8D7E8D8F8DC9
:100E800098A14AE00E9470778DE00E946AC78AE0CC
:100E90000E946AC753CF0FB6F8947EBE0FBE6DBED8
:100EA000CD59DF4F0FB6F894DEBF0FBECDBFDF9137
:100EB000CF911F910F91FF90EF90DF90CF90BF9057
:100EC000AF909F908F907F906F900895CF93C82F91
:100ED0000E94F6DB84E50E946AC78C2F0E9474F1A1
:100EE00080E20E946AC786E890E2CF910C9492C794
:100EF0008F929F92AF92BF92CF92DF92EF92FF922A
:100F0000CF936B017C01B42E20E030E0A9010F9457
:100F1000743287FF07C08DE20E946AC7F7FAF09427
:100F2000F7F8F094C0E060E070E080E09FE3CB155C
:100F300041F02DEC3CEC4CEC5DE30F94DA32CF5FEA
:100F4000F6CFA70196010F9444396B017C010F94F1
:100F5000B73A4B015C014AE00E947077CC2379F1EB
:100F6000C501B4010F9479329B01AC01C701B601F0
:100F70000F9443396B017C018EE20E946AC7C15015
:100F8000F0F020E030E040E251E4C701B6010F94F8
:100F9000DA326B017C010F94B73A4B015C014AE0F5
:100FA0000E947077C501B4010F9479329B01AC01A6
:100FB000C701B6010F9443396B017C01E0CFCF919B
:100FC000FF90EF90DF90CF90BF90AF909F908F9069
:100FD0000895EF92FF920F931F93CF937C018B01A3
:100FE000C2E44F3F09F0C4E580E20E946AC78C2F3B
:100FF0000E946AC78AE30E946AC7F7016081718113
:101000008281938142E00E94788782E790E20E9489
:1010100092C7F801608171818281938142E00E94D0
:10102000788762E070E080E090E0CF911F910F91AF
:10103000FF90EF900C94F7731F93CF93DF9300D042
:1010400000D01F921F92CDB7DEB7182F609170129B
:1010500070917112072E000C880B990B0F947B3244
:101060006D837E838F83988760916E1270916F126B
:10107000072E000C880B990B0F947B3269837A83BF
:101080008B839C834AEFBE016B5F7F4FCE0101963D
:101090000E94E9876091051270910612072E000CDC
:1010A000880B990B0F947B326D837E838F83988797
:1010B0006091031270910412072E000C880B990B9B
:1010C0000F947B3269837A838B839C834FEFBE01BD
:1010D0006B5F7F4FCE0101960E94E98760910712F6
:1010E0001F3F39F085E11802F0011124E659FD4E49
:1010F000608570E08AE790E20E9459CA6091071209
:1011000070E085E790E20E9459CA28960FB6F894DD
:10111000DEBF0FBECDBFDF91CF911F9108952F92FB
:101120003F924F925F926F927F928F929F92AF9277
:10113000BF92CF92DF92EF92FF920F931F93CF93C4
:10114000DF93CDB7DEB763970FB6F894DEBF0FBE5F
:10115000CDBF898B81E080932D021A821B821C8275
:101160001D8219861A861B861C861D862CE32E87F7
:101170003CE13F8746E4488B312C212C50E85A8BC8
:101180008FEB8B8B198291E09887812C912C5401E5
:101190000091051210910612B801012E000C880B67
:1011A000990B0F947B326B017C01232D322D4A89E0
:1011B0005B890F947432882389F080910312909197
:1011C0000412A989A111E4C0B1E0B9830817190775
:1011D0000CF019823C2C2D2CEA8AFB8A0E942A747E
:1011E0006B017C01DC01CB0129853A854B855C854F
:1011F000821B930BA40BB50BB7FD2FC0D701C60103
:1012000088519C4FAF4FBF4F89879A87AB87BC8768
:1012100080E00E941C8882E890E20E9492C78114BC
:101220009104A104B10409F4DFC0C501B4016857F9
:101230007C4E8F4F9F4F6C197D098E099F0928EEB8
:1012400033E040E050E00F94B838CA01B9014AE0F9
:101250000E9471C78AE00E946AC780E00E94A1DFF5
:101260000E942A746093F9117093FA118093FB1114
:101270009093FC116091031270910412072E000CE0
:10128000880B990B0F947B326E837F838C019B01BB
:10129000AC01632D722D8A899B890F9443392B01F0
:1012A0003C0120E030E0A9010F94A43B87FF04C07B
:1012B00077FA709477F8709481149104A104B104C2
:1012C00009F096C020E030E040E85FE3C301B201DE
:1012D0000F94743287FF10C09885812C912C540193
:1012E000992331F082E8882E86E0982EA12CB12C2B
:1012F0008C0C9D1CAE1CBF1CA981AA2391F12A81D4
:101300003B814C815D81211531054105510541F03D
:10131000D701C601821B930BA40BB50BB7FD21C0EF
:101320002E813F81A8016D857E858F8598890F94D8
:10133000433920E030E040E85FE30F94743287FDEA
:101340002AC0D701C601805A9541AF4FBF4F8A834B
:101350009B83AC83BD839E819D87AF81AE870F87C2
:10136000188B80912D028823B1F081149104A1047F
:10137000B10461F0B8E8CB1AB3E1DB0AE108F10887
:10138000C818D908EA08FB08F7FE05C0188600CF80
:10139000081719071CF520912D022983222321F01B
:1013A00010922D020E942DF5898163960FB6F89454
:1013B000DEBF0FBECDBFDF91CF911F910F91FF9088
:1013C000EF90DF90CF90BF90AF909F908F907F90E5
:1013D0006F905F904F903F902F9008953C2C2D2C54
:1013E000EA8AFB8A1982FACE8FE30E946AC732CF5B
:1013F00020E030E040E450E4C301B2010F94A43B8C
:1014000018160CF079CF4601570176CF2F923F92F4
:101410004F925F926F927F928F929F92AF92BF9204
:10142000CF92DF92EF92FF920F931F93CF93DF93B0
:10143000CDB7DEB765970FB6F894DEBF0FBECDBF50
:101440008A8B6B8B20914605298B1092460581E093
:1014500080932D021A821B821C821D8219861A8695
:101460001B861C861D863CE33E874CE14F8756E475
:10147000588B312C212C80E88C8B9FEB9D8B198213
:10148000A1E0A887812C912C540100917012109139
:101490007112B801012E000C880B990B0F947B324E
:1014A0006B017C01232D322D4C895D890F947432A0
:1014B000882389F080916E1290916F12BB89B111CF
:1014C000E4C021E02983081719070CF019823C2C8D
:1014D0002D2CEC8AFD8A0E942A746B017C01DC01B0
:1014E000CB0129853A854B855C85821B930BA40B28
:1014F000B50BB7FD2FC0D701C60188519C4FAF4F28
:10150000BF4F89879A87AB87BC878A890E941C88CE
:101510008EE790E20E9492C781149104A104B10465
:1015200009F4E2C0C501B4016053784F8F4F9F4F5B
:101530006C197D098E099F0928EE33E040E050E0E8
:101540000F94B838CA01B9014AE00E9471C78AE015
:101550000E946AC780E00E94A1DF0E942A74609303
:10156000F9117093FA118093FB119093FC11609123
:101570006E1270916F12072E000C880B990B0F944E
:101580007B326E837F838C019B01AC01632D722DB6
:101590008C899D890F9443392B013C0120E030E078
:1015A000A9010F94A43B87FF04C077FA709477F8E1
:1015B000709481149104A104B10409F099C020E051
:1015C00030E040E85FE3C301B2010F94743287FF5B
:1015D00010C09885812C912C5401992331F08AE90F
:1015E000882E82E0982EA12CB12C8C0C9D1CAE1C58
:1015F000BF1CA981AA2391F12A813B814C815D8185
:10160000211531054105510541F0D701C601821B65
:10161000930BA40BB50BB7FD21C02E813F81A80110
:101620006D857E858F8598890F94433920E030E061
:1016300040EC5FE30F94743287FD2AC0D701C601E6
:10164000805A9541AF4FBF4F8A839B83AC83BD8344
:101650009E819D87AF81AE870F87188B80912D0269
:101660008823B1F081149104A104B10461F0B0EDBC
:10167000CB1AB7E0DB0AE108F108C818D908EA0874
:10168000FB08F7FE05C0188600CF0817190734F5C8
:1016900030912D023983332321F010922D020E94C4
:1016A0002DF5298920934605898165960FB6F89412
:1016B000DEBF0FBECDBFDF91CF911F910F91FF9085
:1016C000EF90DF90CF90BF90AF909F908F907F90E2
:1016D0006F905F904F903F902F9008953C2C2D2C51
:1016E000EC8AFD8A1982F7CE8FE30E946AC72FCF5A
:1016F00020E030E040E450E4C301B2010F94A43B89
:1017000018160CF076CF4601570173CF0F930FB721
:101710000F9300916E000B7F00936E0078940F93EF
:101720000BB70F930CB70F921F922F933F934F93CA
:101730005F936F937F938F939F93AF93BF93EF9339
:10174000FF9311240E94678CFF91EF91BF91AF919D
:101750009F918F917F916F915F914F913F912F91C9
:101760001F900F900CBF0F910BBF0F910460F89466
:1017700000936E000F910FBF0F91189520910512E5
:101780003091061221153105E9F0809103129091F4
:101790000412029624503109821793079CF4909307
:1017A0008F0680938E060E942A74605E70448D4F6F
:1017B0009F4F60939006709391068093920690934A
:1017C0009306089510929006109291061092920638
:1017D000109293060895CF93DF9310924605CAE6C0
:1017E000D2E11F821E820E94EFF018862C98CFEF64
:1017F000D1E11F821E820E94BE8B18868091020159
:10180000807280930001DF91CF910895EF92FF9253
:101810000F931F93CF93DF93C82F7B018A01809191
:1018200013068130A1F40E94F2DBC7010E9492C727
:101830008AE49FE10E9492C7C7FD33C08C2F0C2E13
:10184000000C990B0E947BF18AE00E946AC70E94FB
:10185000EB8BA89580916406811132C081E0809362
:10186000640680E8809313060E94EB8BD5E1D1508B
:10187000409AE1F069E170E080E090E00E94F77347
:10188000A895409868E270E080E090E00E94F773CD
:10189000A89568E270E080E090E00E94F773A89558
:1018A000E6CF86E49FE10E9492C7CECF6FE37FE14F
:1018B000CF3F11F063E47FE140E0C8010E94D0DE39
:1018C000DF91CF911F910F91FF90EF9008950F93AB
:1018D0001F93CF93DF93809122028F3708F442C089
:1018E0008F5790917212909398069923C9F12C9A70
:1018F0002091071220939706909102012111909553
:101900009072909300018F5F8093220280919606DF
:1019100091E089278093960680912102C1E0C80F4B
:1019200085300CF0C0E0823009F4D8C03CF5882343
:10193000D9F1813009F4C6C0C09321020E94EE3271
:1019400080913F0990914009009729F00197909369
:10195000400980933F09DF91CF911F910F91089526
:101960002C98C6CF90919806891708F02C989091E2
:101970009706891740F290910201C2CF843009F492
:10198000C5C00CF4BEC08530B9F690919506911192
:1019900002C08093950680919506815080939506AC
:1019A000882351F2C5E0C8CF809120028F5F80313B
:1019B0001CF480932002C0CF1092200280919406E4
:1019C000811113C080916A1290916B1290936D12E5
:1019D00080936C128091FF119091001290930212EB
:1019E0008093011281E08093940610926B12109202
:1019F0006A12109200121092FF1100916C12109155
:101A00006D128091701290917112D1E01816190622
:101A10002CF080917212811101C0D0E080912702D8
:101A200090912802081719073CF444E350E261E45E
:101A300070E280E00E94068CDD2371F08091250227
:101A400090912602801791073CF443E550E260E64E
:101A500070E280E00E94068C80910512909106123F
:101A6000D1E0181619062CF080910712811101C0DF
:101A7000D0E0209101123091021280919A0690914B
:101A80009B06281739073CF444E350E261E470E216
:101A90008FEF0E94068CDD2309F44ECF20910112B6
:101AA00030910212809123029091240282179307B1
:101AB0000CF042CF43E550E260E670E28FEF0E9407
:101AC000068C3ACF88E080937B0085E480937C008D
:101AD00080917A00806480937A002ECF80917A0082
:101AE00086FD27C0209178003091790080916A129C
:101AF00090916B12820F931F90936B1280936A12D6
:101B00001BCF88E080937B0086E4E0CF80917A0051
:101B100086FD11C020917800309179008091FF11ED
:101B200090910012820F931F909300128093FF11E7
:101B300003CFC2E001CFC4E0FFCE2F923F924F927D
:101B40005F926F927F928F929F92AF92BF92CF924D
:101B5000DF92EF92FF920F931F93CF93DF9300D00A
:101B6000CDB7DEB79B838A836B015A0129831801A5
:101B7000870181E090E02F3F11F090E080E025E0C8
:101B8000289FF001299FF00D1124E45CFA4F848115
:101B9000882309F48FC0EA81FB81148215821682A2
:101BA00017821086EA81FB8184818230B9F083300C
:101BB00009F400C1813009F067C025813681478171
:101BC0005085F60160817181828193810F94743216
:101BD00087FD5AC082E0EA81FB818483EA81FB8130
:101BE00085809680A780B084F601C080D180E28095
:101BF000F380B801110F880B990B0F947B322B01E6
:101C00003C0180911F028823F9F0F981F1111CC079
